:020000040800F2
:1000000000800120C96C02086D3C0208793C02089E
:10001000813C0208893C0208913C02080000000073
:10002000000000000000000000000000A103000824
:10003000A53C0208000000007D040008BD3C020849
:10004000116D0208116D0208116D0208116D020890
:10005000116D0208116D0208116D0208116D020880
:10006000116D0208C93C0208116D0208116D0208E9
:10007000116D0208116D0208116D0208116D020860
:10008000116D0208116D0208116D0208116D020850
:10009000116D0208116D0208116D0208116D020840
:1000A000116D0208116D0208116D0208116D020830
:1000B000116D0208116D0208116D0208116D020820
:1000C000116D0208116D0208116D0208116D020810
:1000D000116D0208116D0208116D0208116D020800
:1000E000E93C0208116D0208116D0208116D020849
:1000F000116D0208116D0208116D0208116D0208E0
:10010000116D0208116D0208116D0208116D0208CF
:10011000116D0208116D0208116D0208116D0208BF
:10012000116D0208116D0208116D0208116D0208AF
:10013000116D0208093D0208116D0208116D0208D7
:10014000116D0208116D0208116D0208116D02088F
:10015000893D0208116D0208593D0208116D02081F
:10016000116D0208116D0208116D0208116D02086F
:10017000116D0208116D0208116D0208116D02085F
:04018000116D0208F3
:1001880010B5054C237833B9044B13B10448AFF3C9
:1001980000800123237010BD041E00200000000011
:1001A80084010008084B10B51BB108480849AFF393
:1001B80000800848036803B910BD074B002BFBD02B
:1001C800BDE81040184700BF000000008401000887
:1001D800081E0020041E00200000000080B483B028
:1001E80000AF78607B6803F108027B685A607B681F
:1001F8004FF0FF329A607B6803F108027B68DA608F
:100208007B6803F108027B681A617B6800221A6028
:100218000C37BD465DF8047B704700BF80B483B0DF
:1002280000AF78607B6800221A610C37BD465DF824
:10023800047B704780B485B000AF786039607B6814
:100248005B68FB60FB685A683B685A607B685A6861
:100258003B689A60FB685B683A689A60FB683A6832
:100268005A607B683A685A603B687A681A617B68AA
:100278001B685A1C7B681A601437BD465DF8047BFE
:10028800704700BF80B485B000AF786039603B68C4
:100298001B68BB60BB68B3F1FF3F03D17B681B6978
:1002A800FB600CE07B680833FB6002E0FB685B687E
:1002B800FB60FB685B681A68BB689A42F6D9FB6802
:1002C8005A683B685A603B685B683A689A603B6862
:1002D800FA689A60FB683A685A603B687A681A61FB
:1002E8007B681B685A1C7B681A601437BD465DF82A
:1002F800047B704780B485B000AF78607B685B682A
:100308007A6892689A607B689B687A6852685A60D3
:100318007B681B69FB60FB685A687B689A4203D15B
:100328007B689A68FB685A607B6800221A61FB68E0
:100338001B685A1EFB681A601437BD465DF8047BBB
:10034800704700BF80B485B000AFF860B9607A60CC
:10035800FB68043BFB60FB684FF080721A60FB6827
:10036800043BFB60BA68FB681A60FB68043BFB60EF
:10037800FB6800221A60FB68143BFB607A68FB6824
:100388001A60FB68203BFB60FB6818461437BD46C3
:100398005DF8047B704700BF064B19680868B0E831
:1003A800F00F80F309884FF0000080F311884EF0B9
:1003B8000D0E7047341E002052480068006880F314
:1003C800088862B600DF00BF80B500AF0A4A0A4B52
:1003D8001B6843F47F031360074A074B1B6843F00D
:1003E8007F43136000F07CF8044B00221A60FFF78B
:1003F800E3FF0023184680BD20ED00E00000002048
:1004080080B400AFBD465DF8047B704780B400AF90
:10041800034B4FF080521A60BD465DF8047B70476D
:1004280004ED00E080B400AF4FF0BF0080F3118806
:10043800044B1B680133034A1360BD465DF8047B17
:10044800704700BF0000002080B400AF084B1B6855
:10045800013B074A1360064B1B68002B03D14FF082
:10046800000080F31188BD465DF8047B704700BF2B
:1004780000000020EFF309800C4B1A6820E9F00F08
:1004880010602DE908404FF0BF0080F3118801F09B
:100498008BFA4FF0000080F31188BDE80840196816
:1004A8000868B0E8F00F80F309887047341E002010
:1004B80080B582B000AF094B4FF080521A6000231C
:1004C8007B604FF0BF0080F3118801F0D7F94FF03F
:1004D800000080F311880837BD4680BD04ED00E0B8
:1004E80080B400AF044B054A1A60054B07221A6016
:1004F800BD465DF8047B704714E000E0BFD40100FE
:1005080010E000E008ED00E080B588B000AF78604A
:1005180000237B6101F080F8424B1B68002B04D15B
:1005280000F0DAF83F4B01221A607B68002B0ED0EE
:1005380008231A467B6813447B607B6803F0070333
:10054800002B04D07B6823F0070308337B607B68AB
:10055800002B56D07B68344A934252D8334BBB6148
:10056800324B1B68FB6104E0FB69BB61FB691B68DC
:10057800FB61FB695A687B689A4203D2FB691B6876
:10058800002BF1D1FB692A4A93423AD0BB691B6818
:10059800082213447B61FB691A68BB691A60FB690E
:1005A8005A687B68D31A08225200934222D9FA6902
:1005B8007B681344FB60FB695A687B68D21AFB6846
:1005C8005A60FB697A685A60FB685B68BB60174BC6
:1005D8003B6102E03B691B683B613B691B685A68E9
:1005E800BB689A42F6D33B691A68FB681A603B6994
:1005F800FA681A600F4B1A68FB695B68D31A0D4AD0
:1006080013607869796820F0A9FC01F013F87B6918
:10061800002B01D120F062FC7B6918462037BD46CB
:1006280080BD00BF301E0020F70F0700201E0020ED
:10063800281E00200400002080B586B000AF786036
:100648007B683B617B68002B2DD008235B423A69AD
:1006580013443B613B69FB6000F0DEFFFB685B68AD
:10066800BB60124B7B6102E07B691B687B617B6925
:100678001B685A68BB689A42F6D37B691A68FB689C
:100688001A607B69FA681A60FB685A68084B1B682D
:100698001344074A1360FB685B687868194620F0C2
:1006A8003BFC00F0C7FF1837BD4680BD201E002068
:1006B8000400002080B400AF034B1B681846BD46F9
:1006C8005DF8047B704700BF0400002080B400AFD1
:1006D800BD465DF8047B704780B483B000AF0D4B16
:1006E8007B600D4A7B6813600B4B00225A600B4BF2
:1006F8000B4A5A60094B00221A607B683B603B68D2
:10070800074A5A603B68054A1A600C37BD465DF8CF
:10071800047B704708000060201E0020281E00206F
:10072800F80F070080B582B000AF78603960FFF736
:1007380079FE7B681A687B68DB6B7968096C01FB5A
:1007480003F31A447B685A607B6800229A637B68CB
:100758001A687B689A607B681A687B68DB6B013B68
:100768007968096C01FB03F31A447B68DA607B68DB
:100778004FF0FF325A647B684FF0FF329A643B684F
:10078800002B0ED17B681B69002B14D07B681033BB
:10079800184601F083F90346012B0CD1FFF736FE0A
:1007A80009E07B6810331846FFF718FD7B6824338F
:1007B8001846FFF713FDFFF747FE012318460837D1
:1007C800BD4680BD80B588B000AFF860B9601346FB
:1007D800FB710023FB61FB68002B2AD05020FFF738
:1007E80093FEB861BB69002B23D0FB68BA6802FB93
:1007F80003F301337B617869FFF786FE0246BB6924
:100808001A60BB691B68002B10D0BB69FA68DA63F1
:10081800BB69BA681A64B8690121FFF783FFBB692D
:10082800FA7983F84D20BB69FB6102E0B869FFF7EC
:1008380003FFFB6918462037BD4680BD80B584B0EC
:1008480000AF0346FB715020FFF75EFEF860FB68BF
:10085800002B30D0FB6800225A60FB6800221A6027
:10086800FB6800229A60FB680022DA60FB680022BD
:100878009A63FB680122DA63FB6800221A64FB684A
:100888004FF0FF325A64FB684FF0FF329A64FB68FE
:10089800FA7983F84D20FB6810331846FFF79EFC61
:1008A800FB6824331846FFF799FCF86800210022FA
:1008B800002300F01BF8FB6818461037BD4680BDC2
:1008C80080B584B000AF7860396078680021022272
:1008D800FFF778FFF860FB68002B02D0FB683A68E6
:1008E8009A63FB6818461037BD4680BD80B588B04E
:1008F80000AFF860B9607A603B600023FB61FFF7E6
:1009080091FDFB689A6BFB68DB6B9A4216D2F8681C
:10091800B9683A6800F008FAFB685B6A002B09D0EE
:10092800FB682433184601F0B9F80346012B01D1BE
:10093800FFF76CFDFFF788FD012359E07B68002B6A
:1009480003D1FFF781FD002352E0FB69002B06D19C
:1009580007F11403184601F0F1F80123FB61FFF7D2
:1009680073FD00F059FEFFF75DFDFB685B6CB3F1AA
:10097800FF3F02D1FB6800225A64FB689B6CB3F10D
:10098800FF3F02D1FB6800229A64FFF75DFD07F183
:1009980014023B1D1046194601F0E6F80346002BE9
:1009A8001ED1F86800F0B8FA0346002B12D0FB6895
:1009B80003F110027B681046194601F03FF8F86809
:1009C80000F034FA00F036FE0346002B0FD1FFF793
:1009D8001DFD0CE0F86800F029FA00F02BFE8EE708
:1009E800F86800F023FA00F025FE002300E086E70F
:1009F80018462037BD4680BD80B586B000AFF86088
:100A0800B9607A603B6000233B614FF0BF0080F320
:100A18001188FB689A6BFB68DB6B9A4224D2F868F2
:100A2800B9683A6800F080F9FB689B6CB3F1FF3F46
:100A380012D1FB685B6A002B13D0FB68243318467D
:100A480001F02CF80346002B0BD07B68002B08D054
:100A58007B6801221A6004E0FB689B6C5A1CFB68E7
:100A68009A6401237B6101E000237B614FF0000061
:100A780080F311887B6918461837BD4680BD00BFD2
:100A880080B588B000AFF860B9607A603B60002339
:100A9800FB61FFF7C7FCFB689B6B002B3BD0FB6837
:100AA800DB68BB61F868B96800F09AF93B68002B0D
:100AB8001CD1FB689B6B5A1EFB689A63FB681B681A
:100AC800002B04D101F072FA0246FB685A60FB68F9
:100AD8001B69002B1BD0FB681033184600F0DEFFA3
:100AE8000346012B13D1FFF791FC10E0FB68BA69AC
:100AF800DA60FB685B6A002B09D0FB682433184670
:100B080000F0CCFF0346002B01D0FFF77FFCFFF776
:100B18009BFC012366E07B68002B03D1FFF794FC64
:100B280000235FE0FB69002B06D107F1100318468C
:100B380001F004F80123FB61FFF786FC00F06CFD6F
:100B4800FFF770FCFB685B6CB3F1FF3F02D1FB68F9
:100B580000225A64FB689B6CB3F1FF3F02D1FB682B
:100B680000229A64FFF770FC07F110023B1D104643
:100B7800194600F0F9FF0346002B2BD1F86800F066
:100B8800A1F90346002B1FD0FB681B68002B08D176
:100B9800FFF748FCFB685B68184601F017FAFFF797
:100BA80053FCFB6803F124027B681046194600F0E9
:100BB80045FFF86800F03AF900F03CFD0346002BC9
:100BC8000FD1FFF723FC0CE0F86800F02FF900F0D4
:100BD80031FD5EE7F86800F029F900F02BFD0023ED
:100BE80000E056E718462037BD4680BD80B586B080
:100BF80000AFF860B9607A6000233B614FF0BF0036
:100C080080F31188FB689B6B002B28D0F868B968C3
:100C180000F0E6F8FB689B6B5A1EFB689A63FB685A
:100C28005B6CB3F1FF3F12D1FB681B69002B13D03B
:100C3800FB681033184600F031FF0346002B0BD039
:100C48007B68002B08D07B6801221A6004E0FB68EF
:100C58005B6C5A1CFB685A6401237B6101E000232A
:100C68007B614FF0000080F311887B6918461837C4
:100C7800BD4680BD80B584B000AF7860FFF7D2FB79
:100C88007B689B6BFB60FFF7DFFBFB681846103740
:100C9800BD4680BD80B485B000AF78607B689B6B33
:100CA800FB60FB6818461437BD465DF8047B704747
:100CB80080B582B000AF78607B681B681846FFF784
:100CC800BBFC7868FFF7B8FC0837BD4680BD00BF9D
:100CD80080B483B000AF78607B6893F84C301846D6
:100CE8000C37BD465DF8047B704700BF80B483B005
:100CF80000AF78600B46FB707B68FA7883F84C206D
:100D08000C37BD465DF8047B704700BF80B483B0E4
:100D180000AF78607B6893F84D3018460C37BD46B5
:100D28005DF8047B704700BF80B584B000AFF86001
:100D3800B9607A60FB681B6C002B0CD1FB681B68E0
:100D4800002B45D1FB685B68184601F091F9FB68F8
:100D580000225A603CE07B68002B1AD1FB689A6835
:100D6800FB681B6C1046B9681A4625F0EBFAFB685D
:100D78009A68FB681B6C1A44FB689A60FB689A685F
:100D8800FB685B689A4223D3FB681A68FB689A6021
:100D98001EE0FB68DA68FB681B6C1046B9681A46E7
:100DA80025F0D0FAFB68DA68FB681B6C5B421A44D2
:100DB800FB68DA60FB68DA68FB681B689A4207D24E
:100DC800FB685A68FB681B6C5B421A44FB68DA6074
:100DD800FB689B6B5A1CFB689A631037BD4680BD45
:100DE80080B582B000AF786039607B681B68002BE3
:100DF80019D07B68DA687B681B6C1A447B68DA60F8
:100E08007B68DA687B685B689A4203D37B681A68F8
:100E18007B68DA607B68DA687B681B6C3868114627
:100E28001A4625F08FFA0837BD4680BD80B582B0D6
:100E380000AF7860FFF7F6FA14E07B685B6A002B76
:100E48000FD07B682433184600F028FE0346002B99
:100E580001D000F0CDFE7B689B6C5A1E7B689A64BB
:100E680000E003E07B689B6C002BE6DC7B684FF0BE
:100E7800FF329A64FFF7E8FAFFF7D4FA14E07B68C8
:100E88001B69002B0FD07B681033184600F006FE54
:100E98000346002B01D000F0ABFE7B685B6C5A1E4A
:100EA8007B685A6400E003E07B685B6C002BE6DC3F
:100EB8007B684FF0FF325A64FFF7C6FA0837BD4621
:100EC80080BD00BF80B584B000AF7860FFF7AAFA94
:100ED8007B689B6B002B0CBF01230023DBB2FB60FC
:100EE800FFF7B2FAFB6818461037BD4680BD00BF51
:100EF80080B485B000AF78607B689B6B002B0CBF1B
:100F080001230023DBB2FB60FB6818461437BD469B
:100F18005DF8047B704700BF80B584B000AF78608F
:100F2800FFF780FA7B689A6B7B68DB6B9A420CBF91
:100F380001230023DBB2FB60FFF786FAFB68184643
:100F48001037BD4680BD00BF80B485B000AF786063
:100F58007B689A6B7B68DB6B9A420CBF012300238A
:100F6800DBB2FB60FB6818461437BD465DF8047BAE
:100F7800704700BF80B58AB002AFF860B9603B60C7
:100F88001346FB80FB881846396B00F059FFB8619F
:100F9800BB69002B74D0BB691A6BFB8803F18043D3
:100FA800013B9B0013447B617B6923F007037B6152
:100FB800FB880093B869B968BA6A7B6B00F05CFE7D
:100FC8007869F9683A68FFF7BDF90246BB691A60A3
:100FD800FB6A002B02D0FB6ABA691A60FFF722FA93
:100FE800354B1B680133344A1360344B1B68002BA4
:100FF80009D1324ABB6913602F4B1B68012B0FD1F3
:1010080000F070FE0CE02E4B1B68002B08D12B4B18
:101018001B68DA6ABB6A9A4202D8284ABB6913601D
:10102800BB69DA6A274B1B689A4203D9BB69DB6A3A
:10103800244A1360244B1A68BB695A64224B1B6804
:101048000133214A1360BB69DA6A204B1B689A4254
:1010580003D9BB69DB6A1D4A1360BB69DA6A1346A8
:101068009B0013449B001A4A1A44BB690433104678
:101078001946FFF7DFF80123FB61FFF7E5F906E002
:101088004FF0FF33FB61F86AB9681FF027FFFB696F
:10109800012B0BD10A4B1B68002B07D0074B1B6891
:1010A800DA6ABB6A9A4201D2FFF7B0F9FB691846BF
:1010B8002037BD4680BD00BFF81E0020341E00202A
:1010C800081F0020001F00201C1F0020041F0020F4
:1010D800381E002080B584B000AF7860FFF7A2F911
:1010E8001D4B1B687A689A4201D100237B607B689C
:1010F800002B02D1184B1B6800E07B68FB60FB6883
:1011080004331846FFF7F6F8FB689B6A002B04D0F7
:10111800FB6818331846FFF7EDF8FB6804330F48EF
:101128001946FFF787F80E4B1B6801330C4A13600A
:101138000C4B1B6801330B4A1360FFF785F90A4B08
:101148001B68002B04D07B68002B01D1FFF75EF9E8
:101158001037BD4680BD00BF341E0020CC1E0020C5
:10116800E01E00201C1F0020081F002080B586B04C
:1011780000AF7860396000237B6100F04DFA7B682E
:101188001A683B6813443B617B681A681B4B1B68F1
:101198009A420CD97B681A683B699A4213D9174B53
:1011A8001B683A699A420ED901237B610BE07B6880
:1011B8001A683B699A4204D8104B1B683A699A42EC
:1011C80001D901237B617B683A691A607B69002B2E
:1011D80008D00B4B1B6804331846FFF78BF83869A7
:1011E80000F0F8FD00F026FAF860FB68002B01D14A
:1011F800FFF70CF91837BD4680BD00BFFC1E002064
:10120800341E002080B584B000AF78600023FB60F6
:101218007B68002B12D000F0FFF90C4B1A687B6832
:101228001344BB600A4B1B6804331846FFF762F887
:10123800B86800F0CFFD00F0FDF9F860FB68002BFE
:1012480001D1FFF7E3F81037BD4680BDFC1E002032
:10125800341E002080B584B000AF7860FFF7E2F854
:101268007B68002B02D1074B1B6800E07B68FB60A2
:10127800FB68DB6ABB60FFF7E7F8BB681846103706
:10128800BD4680BD341E002080B586B000AF7860B2
:10129800396000237B613B68032B01D903233B6042
:1012A800FFF7C0F8334B1B687A689A4201D10023D4
:1012B8007B607B68002B02D12E4B1B6800E07B68AB
:1012C8003B613B69DB6CFB60FA683B689A424CD037
:1012D8003A68FB689A4205D97B68002B07D001233E
:1012E8007B6104E07B68002B01D101237B613B69B2
:1012F800DA6C3B69DB6A9A4202D13B693A68DA6286
:101308003B693A68DA643B68C3F104023B699A6155
:101318003B695969FA6813469B0013449B00164AB7
:10132800134499421CD13B6904331846FEF7E2FF87
:101338003B69DA6A114B1B689A4203D93B69DB6A3D
:101348000E4A13603B69DA6A13469B0013449B00FC
:10135800094A1A443B69043310461946FEF76AFFE6
:101368007B69012B01D1FFF751F8FFF76DF81837AA
:10137800BD4680BD341E0020381E0020041F0020FA
:1013880080B584B000AF7860FFF74CF81E4B1B683F
:101398007A689A4201D100237B607B68002B02D1D6
:1013A800194B1B6800E07B68FB60FB680433184638
:1013B800FEF7A0FFFB689B6A002B04D0FB6818337C
:1013C8001846FEF797FFFB68043310481946FEF7E6
:1013D80031FFFFF739F87B68002B12D10C4B1B68E3
:1013E800002B02D0FFF712F80BE0084B1A68094BE4
:1013F8001B689A4203D1044B00221A6001E000F0F6
:10140800D3FA1037BD4680BD341E0020E41E0020EC
:10141800081F0020F81E002080B485B000AF786057
:101428000023FB607B68BB60BB685B690A4A934228
:101438000AD1BB689B6A094A934205D0BB689B6A7C
:10144800002B01D10123FB60FB6818461437BD4609
:101458005DF8047B704700BFE41E0020B81E002022
:1014680080B584B000AF78607B68FB60FB68002BB8
:1014780034D01C4B1B68FA689A422FD0FEF7D2FF73
:10148800F868FFF7C9FF0346012B25D1FB68043331
:101498001846FEF72FFFFB68DA6A134B1B689A425F
:1014A80003D9FB68DB6A104A1360FB68DA6A1346E3
:1014B8009B0013449B000D4A1A44FB6804331046F2
:1014C8001946FEF7B7FEFB68DA6A064B1B68DB6A4B
:1014D8009A4201D3FEF79AFFFEF7B6FF1037BD46D2
:1014E80080BD00BF341E0020041F0020381E0020CD
:1014F80080B586B000AF786000237B617B683B6174
:101508000023FB604FF0BF0080F311883869FFF7B4
:1015180083FF0346012B32D11D4B1B68002B28D1BA
:101528003B69DA6A1B4B1B68DB6A9A422CBF0123B2
:101538000023DBB27B613B6904331846FEF7DAFE11
:101548003B69DA6A144B1B689A4203D93B69DB6A28
:10155800114A13603B69DA6A13469B0013449B00E7
:101568000E4A1A443B69043310461946FEF762FED8
:1015780005E03B6918330A481946FEF75BFE4FF051
:10158800000080F311887B6918461837BD4680BD76
:101598000C1F0020341E0020041F0020381E0020CD
:1015A800B81E002080B586B004AF00230093002346
:1015B800019300230293002303930C480C498022D3
:1015C8000023FFF7D7FC78607B68012B0BD14FF025
:1015D800BF0080F31188074B01221A60064B0022D6
:1015E8001A60FEF7F1FE0837BD4680BD611C000891
:1015F80064260308081F0020FC1E002080B500AFE9
:101608004FF0BF0080F31188024B00221A60FEF7EA
:10161800F7FE80BD081F002080B400AF044B1B6894
:101628000133034A1360BD465DF8047B704700BF71
:101638000C1F002090B583B000AF00237B60FEF73D
:10164800F1FE314B1B68013B2F4A13602E4B1B6880
:10165800002B52D12D4B1B68002B4ED000233B6032
:1016680027E02B4BDB68DC6804F118031846FEF70B
:1016780041FE231D1846FEF73DFEE26A254B1B6816
:101688009A4202D9E36A234A1360E26A13469B002E
:1016980013449B00204A1A44231D10461946FEF79E
:1016A800C9FDE26A1D4B1B68DB6A9A4201D301231C
:1016B8003B60174B1B68002BD3D1194B1B68002BC1
:1016C8000DD006E000F0DAF8154B1B68013B144A10
:1016D8001360134B1B68002BF4D101233B603B685C
:1016E800012B03D00F4B1B68012B06D101237B6014
:1016F8000C4B00221A60FEF789FEFEF7A5FE7B68F8
:1017080018460C37BD4690BD0C1F0020F81E00205F
:10171800B81E0020041F0020381E0020341E0020A0
:10172800101F0020141F002080B582B000AFFEF704
:1017380079FE054B1B687B60FEF786FE7B681846C2
:101748000837BD4680BD00BFFC1E002080B483B0B2
:1017580000AF00237B604FF0BF0080F31188074B78
:101768001B683B604FF0000080F311883B68184607
:101778000C37BD465DF8047B704700BFFC1E002097
:1017880080B400AF034B1B681846BD465DF8047B68
:10179800704700BFF81E002090B585B000AF786094
:1017A800FFF73AFF7B6800221A707C68204628F011
:1017B80049FB034623442A4A1188927819809A7073
:1017C800284B1B680133FB60FB68013BFB60264923
:1017D800FA6813469B0013449B000B441B68002BBC
:1017E8000BD0FA6813469B0013449B001E4A13440F
:1017F80078681946522200F055FBFB68002BE3D1AC
:101808001A4B1B681B68002B06D0184B1B6878689E
:101818001946422200F046FB154B1B681B68002B3B
:1018280006D0134B1B6878681946422200F03AFB31
:10183800104B1B68002B04D078680E49442200F036
:1018480031FB0D4B1B68002B04D078680A495322E2
:1018580000F028FBFFF7EEFE1437BD4690BD00BF31
:101868006C260308001F0020381E0020B01E002030
:10187800B41E0020CC1E0020E41E002080B584B0D9
:1018880000AF404B1B68002B73D13F4B1B680133E3
:101898003D4A13603C4B1B68002B21D13B4B1B6816
:1018A800FB603B4B1B68394A1360394AFB6813607D
:1018B800384B1B680133374A1360344B1B681B686D
:1018C800002B04D1344B4FF0FF321A6008E02F4B45
:1018D8001B68DB68DB68BB60BB685B682E4A13600B
:1018E800294B1A682C4B1B689A4241D3274B1B681B
:1018F8001B68002B04D1284B4FF0FF321A6037E0E9
:10190800224B1B68DB68DB68BB60BB685B687B607D
:101918001D4B1A687B689A4203D21F4A7B68136082
:1019280026E0BB6804331846FEF7E4FCBB689B6AF4
:10193800002B04D0BB6818331846FEF7DBFCBB68E5
:10194800DA6A164B1B689A4203D9BB68DB6A134AEA
:101958001360BB68DA6A13469B0013449B00104A65
:101968001A44BB68043310461946FEF763FCBDE70A
:1019780004E00C4B1B6801330A4A13601037BD465C
:1019880080BD00BF0C1F0020FC1E0020B01E0020E0
:10199800B41E0020181F002008000020041F00208B
:1019A800381E0020101F002080B483B000AF1E4BEB
:1019B8001B68002B03D01D4B01221A602EE004E0A7
:1019C8001B4B1B68013B1A4A1360194B1A681949CB
:1019D80013469B0013449B000B441B68002BEFD05D
:1019E800134B1A6813469B0013449B00114A134477
:1019F8007B607B685B685A687B685A607B685A685A
:101A08007B6808339A4204D17B685B685A687B68B4
:101A18005A607B685B68DB68074A13600C37BD4611
:101A28005DF8047B704700BF0C1F0020141F0020C6
:101A3800041F0020381E0020341E002080B584B00A
:101A480000AF78603960124B1B6818337868194604
:101A5800FEF718FC0E4B1B6804331846FEF74AFCC9
:101A68003B68B3F1FF3F07D1094B1B6804330948B2
:101A78001946FEF7DFFB07E0074B1A683B6813447B
:101A8800FB60F86800F0A6F91037BD4680BD00BFBE
:101A9800341E0020E41E0020FC1E002080B584B007
:101AA80000AF78607B68DB68DB68BB60BB681833B5
:101AB8001846FEF71FFC1C4B1B68002B1DD1BB688A
:101AC80004331846FEF716FCBB68DA6A174B1B6826
:101AD8009A4203D9BB68DB6A144A1360BB68DA6AA6
:101AE80013469B0013449B00114A1A44BB680433F5
:101AF80010461946FEF79EFB05E0BB6818330D48F3
:101B08001946FEF797FBBB68DA6A0B4B1B68DB6A62
:101B18009A4202D30123FB6001E00023FB60FB68CB
:101B280018461037BD4680BD0C1F0020041F00203A
:101B3800381E0020B81E0020341E002080B483B058
:101B480000AF7860064B1A687B681A60054B1A6804
:101B58007B685A600C37BD465DF8047B704700BF50
:101B6800181F0020FC1E002080B584B000AF7860EC
:101B78003960FEF757FC3B681B68B3F1FF3F02D1A1
:101B88000023FB6029E07B681A68174B1B689A42A0
:101B980008D07B685A68154B1B689A4202D8012303
:101BA800FB601AE0114B1A687B685B68D21A3B68C5
:101BB8001B689A420FD20D4B1A687B685B68D31A70
:101BC8003A681268D21A3B681A607868FFF7B6FF5D
:101BD8000023FB6001E00123FB60FEF735FCFB6896
:101BE80018461037BD4680BD181F0020FC1E002077
:101BF80080B400AF034B01221A60BD465DF8047B38
:101C0800704700BF141F002080B485B000AF786013
:101C18007B68002B05D07B68BB60BB689B6CFB6056
:101C280001E00023FB60FB6818461437BD465DF8E9
:101C3800047B704780B485B000AF786039607B68FA
:101C4800002B04D07B68FB60FB683A689A64143701
:101C5800BD465DF8047B704780B582B000AF786000
:101C680000F07EF8034B1B68012B01D9FEF7CEFB71
:101C7800F6E700BF381E002080B584B000AFF860DA
:101C8800B9607A603B60FB6834331846B968102243
:101C980028F050F9FB68002283F843207B68032B67
:101CA80001D903237B60FB687A68DA62FB687A688B
:101CB800DA64FB6804331846FEF7B0FAFB68183399
:101CC8001846FEF7ABFAFB68FA681A617B68C3F13D
:101CD8000402FB689A61FB68FA685A621037BD46CD
:101CE80080BD00BF80B582B000AF00237B600CE0F0
:101CF8007A6813469B0013449B00114A1344184604
:101D0800FEF76CFA7B6801337B607B68032BEFD9A5
:101D18000C48FEF763FA0C48FEF760FA0B48FEF72A
:101D28005DFA0B48FEF75AFA0A48FEF757FA0A4BCB
:101D3800044A1A60094B044A1A600837BD4680BD38
:101D4800381E0020881E00209C1E0020B81E00207F
:101D5800CC1E0020E41E0020B01E0020B41E00206F
:101D680080B582B000AF184B1B68002B28D0FFF756
:101D780053FC164B1B68002B0CBF01230023DBB25E
:101D88007B60FFF757FC7B68002B19D1FEF74AFBF5
:101D98000E4BDB68DB683B603B6804331846FEF794
:101DA800A9FA0B4B1B68013B094A1360064B1B68D9
:101DB800013B054A1360FEF747FB386800F0E6F878
:101DC8000837BD4680BD00BFE01E0020CC1E0020A5
:101DD800F81E002080B582B000AF7860134B1B68F6
:101DE8007A685A60124B1B687A689A4209D2114B7A
:101DF8001A680E4B1B68043310461946FEF742FA60
:101E080010E00D4B1A68094B1B680433104619463D
:101E1800FEF738FA094B1B687A689A4202D2074AD9
:101E28007B6813600837BD4680BD00BF341E0020A4
:101E3800FC1E0020B41E0020B01E00200800002058
:101E480080B584B000AF03463960FB805020FEF7B0
:101E58005BFBF860FB68002B1FD03B68002B06D1AA
:101E6800FB889B001846FEF74FFB034600E03B68E3
:101E7800FA681363FB681B6B002B05D1F868FEF743
:101E8800DBFB0023FB6008E0FB681A6BFB889B0008
:101E98001046A5211A4627F051FCFB681846103752
:101EA800BD4680BDB0B58EB004AFF860B9601346CA
:101EB800FB71BB687B627B6A5B685A687B6A5A60A5
:101EC8007B6A5A687B6A08339A4204D17B6A5B68EA
:101ED8005A687B6A5A607B6A5B68DB683B62BB68EE
:101EE800FB61FB695B685A68FB695A60FB695A6861
:101EF800FB6908339A4204D1FB695B685A68FB693D
:101F08005A60FB695B68DB68BB61BB691B6B184681
:101F180000F024F80346FB82BB6903F1340597F906
:101F28000740BB69D96AFA8ABB695B6C0091019268
:101F38000293084808492A46234627F009FEF8680C
:101F4800044927F09BFEBA693B6A9A42C7D12837F1
:101F5800BD46B0BD201F00207026030890B482B093
:101F680000AF7860002405E07B6801337B6023467E
:101F780001339CB27B681B78A52BF5D0A3089CB2D3
:101F8800234618460837BD4690BC704780B582B0D6
:101F980000AF78607B681B6B1846FEF74DFB7868CE
:101FA800FEF74AFB0837BD4680BD00BF80B483B04A
:101FB80000AF054B1B687B607B6818460C37BD4635
:101FC8005DF8047B704700BF341E002080B584B0E4
:101FD80000AF78607B68FB60FB68DA6A214B1B689E
:101FE800DB6A9A423AD21F4B1B68DB6AC3F10402D0
:101FF800FB689A61FB685969FB68DA6A13469B00BB
:1020080013449B00184A1344994222D1FB680433B5
:102018001846FEF76FF9134B1B68DA6AFB68DA6239
:10202800FB68DA6A114B1B689A4203D9FB68DB6AC2
:102038000E4A1360FB68DA6A13469B0013449B0040
:10204800094A1A44FB68043310461946FEF7F2F8A9
:1020580004E0044B1B68DA6AFB68DA621037BD4695
:1020680080BD00BF341E0020381E0020041F002041
:1020780080B584B000AF78607B68FB607B68002B1C
:102088002CD0FB68DA6AFB68DB6C9A4226D0FB68C6
:1020980004331846FEF72EF9FB68DA6CFB68DA623F
:1020A800FB68DB6AC3F10402FB689A61FB68DA6AC1
:1020B8000C4B1B689A4203D9FB68DB6A094A136018
:1020C800FB68DA6A13469B0013449B00064A1A44CD
:1020D800FB68043310461946FEF7ACF81037BD46C6
:1020E80080BD00BF041F0020381E002080B485B0CA
:1020F80000AF78600023FB607B68FB6002E0FB6850
:10210800013BFB60FB68002BF9D11437BD465DF835
:10211800047B704780B500AF4FF00070012102F0DA
:102128004BFC4FF00070002102F046FC80BD00BF60
:1021380080B483B000AF78607B6801221A607B6846
:1021480000225A607B6800229A607B680022DA606D
:102158007B6800221A617B684FF480425A617B6871
:1021680000229A617B680022DA617B684FF4006282
:102178001A627B6800225A627B6800229A627B6836
:102188000022DA627B6800221A637B6800225A63A5
:102198007B6800229A637B680022DA637B684022AE
:1021A8001A647B6820225A647B6800229A647B68E0
:1021B8000022DA647B6800221A657B6800225A656F
:1021C8007B6800229A657B680022DA657B680022BA
:1021D8001A667B6880225A667B6800229A667B684A
:1021E8000022DA667B6800221A677B6800225A6739
:1021F8007B6800229A677B680022DA677B684FF069
:102208008062C3F880207B684FF00072C3F8842096
:102218007B680022C3F888207B684FF40012C3F85B
:102228008C207B680022C3F890207B680022C3F8CA
:1022380094207B680022C3F898207B680022C3F8AA
:102248009C207B680022C3F8A0207B684FF00072B6
:10225800C3F8A4207B684FF48032C3F8A8207B68B9
:102268004FF48002C3F8AC207B684FF40052C3F8E7
:10227800B0207B680022C3F8B4207B680022C3F832
:10228800B8200C37BD465DF8047B704780B58AB02E
:1022980000AF78600B467B8000233B6200237B62A3
:1022A800614BFB610023BB60604B1B697B627B6AEF
:1022B80023F01C037B6207F10C03184602F0D2FAE4
:1022C8003B69FB61FB695A4A934208D9FB69594A41
:1022D800934204D87B6A43F008037B6219E0FB69E8
:1022E800544A934208D9FB69534A934204D87B6AFB
:1022F80043F00C037B620CE0FB694F4A934204D91C
:10230800FB694E4A934200D803E07B6A43F004031A
:102318007B62464A7B6A13617B88184600214FF42A
:10232800004201F0D3F90346002B01D100236BE1F1
:102338004348FFF7DBFE7B681B68002B5FD0BB6858
:102348000133BB607B881846012101F06FF9034611
:1023580003F00403002B03D1BB683A4A9342EED939
:10236800BB68394A934201D100234DE10023BB6089
:102378007B88184600214FF4805201F0A7F90346E4
:10238800002B01D100233FE1BB680133BB607B8890
:102398001846012101F04AF9034603F02003002BF7
:1023A80003D1BB68274A9342EED9BB68264A9342B9
:1023B80001D1002328E10023BB607B881846102147
:1023C80001F034F903463B623B6A03F00403002B37
:1023D80004D07B684FF400621A6202E07B68002236
:1023E8001A623B6A03F00203002B03D07B680022C9
:1023F8005A612FE07B684FF480425A612AE07B687B
:102408001B6ADB089AB27B685B695B089BB2134363
:102418009BB27A88104600211A4601F057F9034604
:10242800002B13D10023EFE00087930300800240C4
:10243800FF2C3101BF0E1602FF869303FFE0F5055E
:10244800FFFF0F00FEFF0400FFFF04006FF07F4056
:10245800FFF74CFE6E4B1B687B627A6A6D4B13402C
:102468007B627B685A687B689B681A437B68DB6879
:102478001A437B681B691A437B685B691A437B684C
:102488009B691A437B68DB691A437B681B6A1A439A
:102498007B685B6A1A437B689B6A1A437B68DB6AC2
:1024A8001A437B681B6B1A437B685B6B13437A6A1E
:1024B80013437B62564A7B6A136055497B689A6B63
:1024C8007B68DB6B1A437B681B6C1A437B685B6C0D
:1024D8001A437B689B6C1A437B68DB6C1A437B68E6
:1024E8001B6D1A437B685B6D13434B60484A7B68DE
:1024F8009B6D9360464A7B68DB6DD360444B9B6958
:102508007B627A6A4FF6417313407B627B681B6E6D
:102518001A047B685B6E1A437B689B6E1A437B6860
:10252800DB6E1A437B681B6F1A437B685B6F134330
:102538007A6A13437B62364A7B6A936134497B68C3
:102548009A6F7B68DB6F1343CB61314B03F5805384
:1025580018331B687B627A6A2F4B13407B627B6857
:10256800D3F880207B68D3F884301A437B68D3F88B
:1025780088301A437B68D3F88C301A437B68D3F8C9
:1025880090301A437B68D3F894301A437B68D3F8A9
:1025980098301A437B68D3F89C301A437B68D3F889
:1025A800A03013437A6A13437B62194B03F58053B7
:1025B80018337A6A1A6016497B68D3F8A4207B68B6
:1025C800D3F8A8301A437B68D3F8AC301A437B6839
:1025D800D3F8B0301A437B68D3F8B4309B001A4361
:1025E8007B68D3F8B830134343F4000201F58053F5
:1025F8001A600749064B03F580531B6843F08002B5
:1026080001F580531A60012318462837BD4680BD5E
:10261800008002400F8120FF233FDEF880B500AF25
:10262800012000F00DF800F0DFFE012000F024F892
:10263800012000F009FF012000F02EFF80BD00BF3F
:1026480080B483B000AF0346FB71FB79002B06D042
:10265800084A084B1B6843F00803136005E0054A65
:10266800044B1B6823F0080313600C37BD465DF864
:10267800047B70470080024080B483B000AF0346FB
:10268800FB71FB79002B06D0084A084B1B6843F006
:102698000403136005E0054A044B1B6823F0040398
:1026A80013600C37BD465DF8047B7047008002401C
:1026B80080B483B000AF0023FB71094B9B6903F022
:1026C8000103002B02D00123FB7101E00023FB7101
:1026D800FB7918460C37BD465DF8047B704700BF90
:1026E8000080024080B400AF044A044B9B6943F069
:1026F80001039361BD465DF8047B7047008002408A
:1027080080B483B000AF0346FB71FB79002B06D081
:10271800084A084B9B6943F00103936105E0054AA9
:10272800044B9B6923F0010393610C37BD465DF8A8
:10273800047B70470080024080B485B000AF7860A9
:102748000023FB73084B9A6B7B681340002B02D065
:102758000123FB7301E00023FB73FB7B184614374E
:10276800BD465DF8047B70470080024080B485B0A8
:1027780000AF78600023FB73084B9A6B7B681340AB
:10278800002B02D00123FB7301E00023FB73FB7BCA
:1027980018461437BD465DF8047B70470080024038
:1027A80080B483B000AF78600B46FB70FB78002BD9
:1027B80007D00949084BDA6B7B68DB431340CB63CE
:1027C80005E00549044BDA6B7B681343CB630C3790
:1027D800BD465DF8047B70470080024080B485B038
:1027E80000AF786039603B6805331B781B023A6894
:1027F800043212781343FB607A68114B13441A466B
:10280800FB6813603B6803331B781A063B68023386
:102818001B781B041A433B6801331B781B021343C4
:102828003A6812781343FB607A68064B13441A46D9
:10283800FB6813601437BD465DF8047B704700BF22
:10284800408002404480024080B485B000AF786088
:1028580039607A68174B13441B68FB603B68053383
:10286800FA68120AD2B21A703B680433FA68D2B214
:102878001A707A68104B13441B68FB603B6803337B
:10288800FA68120ED2B21A703B680233FA68120C58
:10289800D2B21A703B680133FA68120AD2B21A70BF
:1028A800FB68DAB23B681A701437BD465DF8047BE2
:1028B800704700BF408002404480024080B483B02B
:1028C80000AF78600B46FB70FB78002B0BD07A6862
:1028D8000D4B134419467A680B4B13441B6843F09D
:1028E80000430B600AE07A68074B134419467A687C
:1028F800054B13441B6823F000430B600C37BD469F
:102908005DF8047B704700BF4080024080B483B00C
:1029180000AF786039603B68082B0BD07A680D4BA4
:10292800134419467A680B4B13441B6843F08043E1
:102938000B600AE07A68074B134419467A68054B1E
:1029480013441B6823F080430B600C37BD465DF8C9
:10295800047B70474080024080B483B000AF786049
:1029680039607A680C4B134419467A680A4B134449
:102978001B6823F07C530B607A68074B1344194695
:102988007A68054B13441A683B6813430B600C378D
:10299800BD465DF8047B70474080024090B486B025
:1029A80000AF786000237B610023BB600023FB60DD
:1029B80000233B61174B1B681A68174B13401B0C0D
:1029C800043B7B617B69BB60144B1B689B68012BD4
:1029D80005D9124B1B681B689B68FB6003E00D4B15
:1029E8001B689B68FB600B4B1B683B61094B1B68B2
:1029F800DB681A46074B1A607B681C4607F1080318
:102A080093E8070084E8070078681837BD4690BC4B
:102A1800704700BFE45000200000FF3F0C63002017
:102A280090B486B000AF78600023FB6000233B6160
:102A380000237B610023BB6077E0BB680133BB6088
:102A4800454B1B681B6803F40073002B16D0424BE0
:102A58001B681B6803F48073002B0FD13F4B1B6866
:102A68003D4A12681A603D4B1B6801229A603A4B36
:102A78001B68DB681A46384B1A6056E0364B1B68F1
:102A88001B6803F48073002B12D1334B1B681B683F
:102A980003F40073002B0BD1304B1B689A6801328A
:102AA8009A602D4B1B68DB681A462B4B1A603CE07A
:102AB8002A4B1B68284A12685A60284B1B689A6878
:102AC80001329A60254B1B689B68012B04D1234B6C
:102AD8001B68214A12681A601F4B1B681A68204B32
:102AE80013401B0C043BFB601C4B1B689B68012BB1
:102AF80005D91A4B1B681B689B683B6103E0164BA2
:102B08001B689B683B61144B1B687B61124B1B68FD
:102B1800DB681A46104B1A607B681C4607F10C03E9
:102B280093E8070084E8070010E00B4B1B681B685C
:102B3800002B03DBBB68022B7FF67FAF7B681C464C
:102B480007F10C0393E8070084E807007868183752
:102B5800BD4690BC704700BFE45000200C630020C5
:102B68000000FF3F80B487B000AF0346FB8000231E
:102B78007B610023BB6000233B61514B1B681B68D2
:102B8800002B01DA002395E04D4B1B68FB60FB88A6
:102B980040F2F452934217D9FB884A4AA2FB032316
:102BA8009B0A9BB27B61FB88464AA2FB0312920AEE
:102BB80040F2F45101FB02F29B1A9BB2002B05D0A4
:102BC8007B6901337B6101E001237B617B69012B18
:102BD8001CD13B4B1B683A4A1268126842F04052BB
:102BE8001A60374B1B68FA88C2F30C025A60344BE0
:102BF8001B68334A1268126842F000421A60304B70
:102C08001B68DB681A462E4B1A603DE000233B61C7
:102C180033E03B69002B07D1294B1B68284A12680F
:102C2800126842F080521A60FB6840F2F4525A600F
:102C38007B695A1E3B699A4213D1FB681B6843F0B3
:102C48000052FB681A60FA887B691F4901FB03F38D
:102C5800134403F2F453BB60BB68C3F30C02FB6874
:102C68005A60FB681B6843F00042FB681A60FB6807
:102C7800DB68FB603B6901333B613A697B699A42D7
:102C8800C7D30F4AFB681360104B03F58053143306
:102C98001B6803F00403002B0BD00C4B03F5805387
:102CA800143304221A60094B03F5805304330022BD
:102CB8001A60012318461C37BD465DF8047B70472F
:102CC800E85000200BB002AC0CFAFFFF0080024075
:102CD80080B487B000AFF860B9607A6000237B6188
:102CE800214AFB68136000237B612AE07B695B0152
:102CF800FA6813443B613B694FF000421A603B6934
:102D080044F2F4525A607B6940F2F45202FB03F336
:102D1800BA6813441A463B699A607B685A1E7B69F5
:102D28009A4208D97B6901335B01FA6813441A4651
:102D38003B69DA6002E0FA683B69DA607B69013373
:102D48007B617A697B689A42D0D3084BFA6803F5AD
:102D580080530C331A60064B064A1A601C37BD466E
:102D68005DF8047B704700BFE450002000800240FB
:102D78000C630020D850002080B400AF314B1B6892
:102D88001B68002B12DB2F4B1B681B6803F4807336
:102D9800002B0BD02C4B1B682A4A12685A602A4B0E
:102DA8001B689A6801329A60012345E0254B1B682D
:102DB8001B68002B21DB234B1B681B6803F4007383
:102DC800002B1AD01F4B1B681B6803F48073002B61
:102DD80013D11D4B1B681B4A12681A601A4B1B68DB
:102DE80000225A60184B1B6801229A60154B1B6819
:102DF800DB681A46134B1A601DE0124B1B681B68F0
:102E0800002B18DB0F4B1B681B6803F40073002BA7
:102E180011D10C4B1B681B6803F48073002B0AD17B
:102E2800094B1B689A6801329A60064B1B68DB687D
:102E38001A46044B1A6000231846BD465DF8047B09
:102E4800704700BFE45000200C63002080B487B0B6
:102E580000AFF860B9607A6000237B611D4AFB68A7
:102E6800136000237B6126E07B695B01FA681344E9
:102E78003B613B694FF480121A607B6940F2F4525F
:102E880002FB03F3BA6813441A463B699A607B68ED
:102E98005A1E7B699A4208D97B6901335B01FA683B
:102EA80013441A463B69DA6002E0FA683B69DA6063
:102EB8007B6901337B617A697B689A42D4D3064B7C
:102EC800FA6803F5805310331A601C37BD465DF865
:102ED800047B7047E85000200080024080B485B031
:102EE80000AF786039600023FB737B681A683B6821
:102EF8001340002B02D00123FB7301E00023FB7376
:102F0800FB7B18461437BD465DF8047B704700BF4D
:102F180080B483B000AF78607B681B6803F07803E7
:102F2800DB0818460C37BD465DF8047B704700BFC8
:102F380080B483B000AF78607B681B6843F00042C0
:102F48007B681A600C37BD465DF8047B704700BF8C
:102F580080B483B000AF78600B46FB70FB78002B21
:102F680006D07B681B6843F080427B681A6005E0E6
:102F78007B681B6823F080427B681A600C37BD466B
:102F88005DF8047B704700BF80B483B000AF786001
:102F980039607B681A683B681A437B681A600C378B
:102FA800BD465DF8047B704780B483B000AF78609D
:102FB80039607B681A683B681A437B681A600C376B
:102FC800BD465DF8047B704780B483B000AF78607D
:102FD8000B46FB70FB78002B06D07B681B6823F040
:102FE80000627B681A6005E07B681B6843F000623A
:102FF8007B681A600C37BD465DF8047B704700BFDC
:1030080080B483B000AF78600B46FB70FB78002B70
:1030180006D07B681B6843F480127B681A6005E061
:103028007B681B6823F480127B681A600C37BD46E6
:103038005DF8047B704700BF80B483B000AF786050
:103048000B46FB70FB78002B06D07B681B6823F0CF
:1030580080627B681A6005E07B681B6843F08062C9
:103068007B681A600C37BD465DF8047B704700BF6B
:1030780080B485B000AFF860B9607A60FB685A68C0
:103088007B681904BB680B431A43FB685A60143702
:10309800BD465DF8047B704780B485B000AF7860AA
:1030A80039600023FB737B681A683B681340002B68
:1030B80002D00123FB7301E00023FB73FB7B18465E
:1030C8001437BD465DF8047B704700BF80B485B0F7
:1030D80000AF786039600023FB737B681A693B682E
:1030E8001340002B02D00123FB7301E00023FB7384
:1030F800FB7B18461437BD465DF8047B704700BF5C
:1031080080B483B000AF78607B681B6843F00042EE
:103118007B681A600C37BD465DF8047B704700BFBA
:1031280080B483B000AF78607B681A68044B1340A2
:103138001B0C18460C37BD465DF8047B704700BF72
:103148000000FF3F80B483B000AF78600B46FB708F
:10315800FB78002B06D07B685B6823F000427B6815
:103168005A6005E07B685B6843F000427B685A6000
:103178000C37BD465DF8047B704700BF80B483B050
:1031880000AF786039603B68002B05D07B685A68CF
:10319800064B13401B0C03E07B685B68C3F30C030E
:1031A80018460C37BD465DF8047B70470000FF1FCA
:1031B80080B584B000AF78600023FB607B681B6833
:1031C800002B0FDB7B681B6803F40043002B09D13D
:1031D8007B681B6803F48073002B03D07868FFF7C3
:1031E8009FFFF860FB6818461037BD4680BD00BFDA
:1031F80080B483B000AF0346FB71FB79002B0AD083
:103208000C490C4B03F580531B6843F0800201F511
:1032180080531A6009E00749064B03F580531B6881
:1032280023F0800201F580531A600C37BD465DF823
:10323800047B70470080024080B400AF0649064B0B
:1032480003F580531B6843F0010201F580531A60AF
:10325800BD465DF8047B70470080024080B483B0AF
:1032680000AF0023FB710A4B03F580531B6803F082
:103278000103002B02D00123FB7101E00023FB7145
:10328800FB7918460C37BD465DF8047B704700BFD4
:103298000080024080B485B000AF78600023FB73E3
:1032A8000A4B03F5805314331A687B681340002BCC
:1032B80002D00123FB7301E00023FB73FB7B18465C
:1032C8001437BD465DF8047B704700BF008002409C
:1032D80080B483B000AF7860054B03F58053143396
:1032E8007A681A600C37BD465DF8047B704700BFEA
:1032F8000080024080B483B000AF78600B46FB705A
:10330800FB78002B0CD00F490E4B03F580531C3370
:103318001A687B681A4301F580531C331A600CE065
:103328000849084B03F580531C331A687B68DB4354
:103338001A4001F580531C331A600C37BD465DF8FE
:10334800047B70470080024080B485B000AF78608D
:103358000023FB730A4B03F5805314331A687B6808
:103368001340002B02D00123FB7301E00023FB7301
:10337800FB7B18461437BD465DF8047B704700BFD9
:103388000080024080B483B000AF7860054B03F53D
:10339800805314337A681A600C37BD465DF8047B95
:1033A800704700BF0080024080B400AF054B03F5B2
:1033B800805314331B6803F001031846BD465DF8BB
:1033C800047B70470080024080B400AF054B03F5D2
:1033D800805314331B6803F040031846BD465DF85C
:1033E800047B70470080024080B400AF0749074B58
:1033F80003F5805318331B6843F4801201F580539A
:1034080018331A60BD465DF8047B7047008002409F
:1034180080B483B000AF0023FB710A4B03F58053DF
:1034280018331B6803F48013002B02D00123FB71AF
:1034380001E00023FB71FB7918460C37BD465DF8A7
:10344800047B70470080024080B483B000AF03461D
:10345800FB71FB79002B0CD00E490E4B03F5805302
:1034680018331B6843F4005201F5805318331A606F
:103478000BE00849074B03F5805318331B6823F406
:10348800005201F5805318331A600C37BD465DF8B9
:10349800047B70470080024080B483B000AF0346CD
:1034A800FB71FB79002B0CD00E490E4B03F58053B2
:1034B80018331B6843F0020201F5805318331A6071
:1034C8000BE00849074B03F5805318331B6823F0BA
:1034D800020201F5805318331A600C37BD465DF8B7
:1034E800047B70470080024080B485B000AF7860EC
:1034F8000023FB73094B03F581531A687B6813405B
:10350800002B02D00123FB7301E00023FB73FB7B3C
:1035180018461437BD465DF8047B704700800240AA
:1035280080B400AF054B03F581531A68044B134070
:103538005B0C1846BD465DF8047B7047008002406E
:103548000000FE0F80B400AF044B03F581531B68E5
:103558009BB21846BD465DF8047B70470080024068
:1035680080B400AF044B03F5825308331B68184638
:10357800BD465DF8047B70470080024080B400AF10
:10358800044B03F582530C331B681846BD465DF89F
:10359800047B70470080024080B400AF044B03F501
:1035A800825310331B681846BD465DF8047B70478C
:1035B8000080024080B400AF044B03F582531433FB
:1035C8001B681846BD465DF8047B704700800240C2
:1035D80080B400AF044B03F58053043300221A6013
:1035E800BD465DF8047B70470080024080B400AFA0
:1035F800044B03F58053083300221A60BD465DF87A
:10360800047B70470080024080B483B000AF03465B
:10361800FB71054BFA7903F5815304331A600C37B3
:10362800BD465DF8047B70470080024080B485B0D9
:1036380000AF03460A46FB801346BB800023FB60AD
:103648000023BB601E4B1B69FB60FB6803F01C0377
:10365800FB60FB88DB029BB2FA681343FB60BB8804
:103668009B0103F4F863FA681343FB60FB6823F0DB
:103678000203FB60FB6843F00103FB60104AFB6830
:103688001361BB680133BB600D4B1B69FB60FB68B2
:1036980003F00103002B03D0BB680A4A9342F0D918
:1036A800BB68094A934201D1002302E0044B5B69DD
:1036B8009BB218461437BD465DF8047B704700BFBF
:1036C80000800240FEFF0400FFFF040080B485B0C4
:1036D80000AF0346FB800B46BB8013467B8000236C
:1036E800FB600023BB601F4B1B69FB60FB6803F09A
:1036F8001C03FB60FB88DB029BB2FA681343FB6088
:10370800BB889B0103F4F863FA681343FB60FB680A
:1037180043F00203FB60FB6843F00103FB60114ABE
:103728007B8853610F4AFB681361BB680133BB6038
:103738000C4B1B69FB60FB6803F00103002B03D0F3
:10374800BB68094A9342F0D9BB68084A934201D141
:10375800002300E0012318461437BD465DF8047BBA
:10376800704700BF00800240FEFF0400FFFF040016
:1037780080B584B000AF03460A46FB8013467B71D0
:103788000023FB81FB8818460021FFF74FFF034603
:10379800FB817B79002B04D0FB8943F48043FB81B8
:1037A80003E0FB8923F48043FB81FA88FB891046F8
:1037B80000211A46FFF78AFF0346002B01D0012398
:1037C80000E0002318461037BD4680BD80B400AF26
:1037D800044A044BDB6A43F00043D362BD465DF8FC
:1037E800047B70470080024080B485B000AF7860E9
:1037F8000023FB600023FB6009E00949FB689B008C
:103808007A6813441B688B62FB680133FB60FB68B2
:10381800072BF2D91437BD465DF8047B704700BF0B
:103828000080024080B483B000AF0346FB71FB798F
:10383800002B06D0084A084BDB6A43F40073D362B6
:1038480005E0054A044BDB6A23F40073D3620C37A6
:10385800BD465DF8047B70470080024080B485B0A7
:1038680000AF78600023FB73084BDA6A7B6813406B
:10387800002B02D00123FB7301E00023FB73FB7BC9
:1038880018461437BD465DF8047B70470080024037
:1038980080B483B000AF0346FB71FB79002B06D0E0
:1038A800084A084BDB6A43F00403D36205E0054A83
:1038B800044BDB6A23F00403D3620C37BD465DF882
:1038C800047B70470080024080B483B000AF034699
:1038D800FB71FB79002B06D0084A084BDB6A43F0E2
:1038E8000203D36205E0054A044BDB6A23F00203B6
:1038F800D3620C37BD465DF8047B704700800240F8
:1039080080B483B000AF0346FB71FB79002B06D06F
:10391800084A084BDB6A43F00103D36205E0054A15
:10392800044BDB6A23F00103D3620C37BD465DF814
:10393800047B70470080024080B400AF054A054B05
:10394800D3F8003143F03003C2F80031BD465DF8CA
:10395800047B70470080024080B400AF094A094BDD
:10396800D3F8003123F02003C2F80031054A054B93
:10397800D3F8003143F01003C2F80031BD465DF8BA
:10398800047B70470080024080B483B000AF0346D8
:10399800FB71FB79002B08D00A4A0A4BD3F8003197
:1039A80043F00803C2F8003107E0064A054BD3F894
:1039B800003123F00803C2F800310C37BD465DF82A
:1039C800047B70470080024080B483B000AF034698
:1039D800FB71FB79002B08D00A4A0A4BD3F8003157
:1039E80043F00403C2F8003107E0064A054BD3F858
:1039F800003123F00403C2F800310C37BD465DF8EE
:103A0800047B70470080024080B483B000AF034657
:103A1800FB71FB79002B08D00A4A0A4BD3F8003116
:103A280023F00203C2F8003107E0064A054BD3F839
:103A3800003143F00203C2F800310C37BD465DF88F
:103A4800047B70470080024080B400AF054A054BF4
:103A5800D3F8003143F00103C2F80031BD465DF8E8
:103A6800047B70470080024080B483B000AF786068
:103A78000B46FB707B6803F08053002B19D07B68E2
:103A880023F080537B60FB78002B09D01649164B36
:103A9800D3F80C217B68DB431340C1F80C311DE0DF
:103AA8001149114BD3F80C217B681343C1F80C3131
:103AB80014E0FB78002B09D00B490B4BD3F81021ED
:103AC8007B68DB431340C1F8103107E00649064B19
:103AD800D3F810217B681343C1F810310C37BD4669
:103AE8005DF8047B704700BF0080024080B485B059
:103AF80000AF78600023FB737B6803F08053002BD2
:103B080013D0174BD3F804217B681340002B09D03E
:103B1800134BD3F80C217B681340002B02D10123EF
:103B2800FB7315E00023FB7312E00D4BD3F808215B
:103B38007B681340002B09D0094BD3F80C217B6814
:103B48001340002B02D10123FB7301E00023FB7318
:103B5800FB7B18461437BD465DF8047B704700BFF1
:103B68000080024080B483B000AF78607B6803F1C6
:103B7800804303F520331B6818460C37BD465DF8B3
:103B8800047B704740F0BF60024B40F40030D860BF
:103B9800704700BF00ED00E0C27810B5037812B39B
:103BA800164A03F16043D1684278C943C1F3022140
:103BB800C1F10404E4B2A240D4B20F220A418178D0
:103BC80003F561430A4022431201D2B283F800236D
:103BD80003780122590903F01F0302FA03F3084A84
:103BE80042F8213010BD5A09012103F01F03994002
:103BF80002F12003024A42F8231010BD00ED00E054
:103C080000E100E021F0604121F07F01014B084311
:103C18009860704700ED00E0044B1A6909B1104341
:103C280001E022EA00001861704700BF00ED00E0E3
:103C3800044B04281A680CBF42F0040222F0040264
:103C48001A60704710E000E0036823F00103036086
:103C58000023036043608360C360036121234361E1
:103C6800294B984217D0294B98421BD0284B984291
:103C780020D0284B984225D0274B98422AD0274B52
:103C880098422ED0264B984232D0264B984236D0B6
:103C9800254B984203D13D2243F8082C7047234B0B
:103CA800984204D14FF4746243F8202C7047204B9B
:103CB800984204D14FF4741243F8382C70471D4BC6
:103CC800984204D14FF0746243F8502C70471A4B55
:103CD800984203D1194A43F8642C7047184B98420C
:103CE80003D1184A43F87C2C7047174B984203D1EC
:103CF800164A43F8942C7047154B984203D14FF05D
:103D08003D5243F8AC2C70471060024028600240D6
:103D18004060024058600240706002408860024083
:103D2800A0600240B860024010640240286402406B
:103D38004064024058640240706402403D00002024
:103D480088640240400F0020A064024000003D202B
:103D5800B86402400268134B10B51340CC680A6877
:103D680014434A6914438A691443CA6914430A6AA2
:103D780014434A6A14438A6A14434A6B14438A6B8D
:103D880022431343036043690C6B23F00702CB6A99
:103D98002343134343610B6943604B6883608B681B
:103DA800C36010BD3F801CF0002303604360836044
:103DB800C360036143618361C361036243628362D9
:103DC800C3620363436383637047036811B143F0BD
:103DD800010301E023F0010303607047036811B198
:103DE80043F4004301E023F4004303607047036891
:103DF80011B143F0200301E023F020030360704772
:103E080041607047406880B27047036812B143F45C
:103E1800002301E023F40023036001617047036875
:103E280011B143F4802301E023F480230360704739
:103E38000AB101617047C16070470068C0F3C040B3
:103E48007047006800F001007047406900F03800D2
:103E580070470A4B10B50A4A0A4CA04294BF18464C
:103E680010468B004CBF4368036821F0F02121F015
:103E78008211194214BF0120002010BD00600240C9
:103E8800006402400F64024010B5084A084B094C10
:103E9800A04294BF1846104611F0005F21F0F021AF
:103EA80021F0821114BFC160816010BD006402401E
:103EB800006002400F6402400B0611D543694AB105
:103EC80043F080038029436114D0036801F01E0188
:103ED80019430EE023F080038029436104D1704721
:103EE800802907D0002AF0D1036801F01E0123EAD7
:103EF800010101607047114A114B10B5114CA042E5
:103F080094BF1C46144621F0F02323F0C3122AB1B3
:103F1800006800F01E0000EAD12202E0406900F0CB
:103F2800800289004CBF6068206823F08213184023
:103F380002D0101C18BF012010BD00BF0064024051
:103F4800006002400F64024010B5084A084B094C53
:103F5800A04294BF1846104611F0005F21F0F021EE
:103F680021F0821114BFC160816010BD006402405D
:103F7800006002400F640240044B00221A605A603D
:103F88009A60DA60024A5A61704700BF003C0140FB
:103F9800FFFF7F00827970B501680379002A29D074
:103FA800CE43194A03F18043156803F59E33354023
:103FB80015605468344054601C68214319600368D4
:103FC8009468DD432C409460D1682940D1604179E0
:103FD800102909BF916801F180421943916015BF0A
:103FE80002F59E32D16811680B4316BF0B43D360AC
:103FF800136070BD03F1804303F59E331A6822EA0B
:104008000101196070BD00BF003C014000230C2273
:1040180003600371427183717047024A1369184340
:1040280010617047003C0140034B5B69184214BFA4
:1040380001200020704700BF003C0140014B58613F
:10404800704700BF003C0140054B1A685B6903409C
:1040580004D0104214BF0120002070471846704752
:10406800003C0140014B5861704700BF003C0140D3
:104078004FF0204318B943F2DB021A6003E043F221
:10408800D20243F82020800000F120406FF07043F6
:104098004360C0F8043170478168436830B541EA2D
:1040A8000302C368C46A1A430369082942EA03027F
:1040B8004369416B42EA030283698D6942EA03025C
:1040C800C36942EA0302036A42EA0302436A42EA14
:1040D8000302836A43EA0203026B43EA040343EAE6
:1040E800020302684FEA820202F12042136002BF13
:1040F800136843F0400313600B68B4F5804F43EA3C
:1041080005034D6843EA05138D6843EA0523CD6826
:1041180043EA05430D69496943EA055343EA0163E4
:10412800536010D1816B88690B680343486843EA80
:104138000013886843EA00230869496943EA005381
:1041480043EA016301E06FF07043C2F8043130BD07
:10415800022210B542604FF480524262416B4FF424
:104168000052826200230F22FF2403608360C36031
:10417800036143618361C3610362C36203630A60CD
:104188004A608C60CA600A614A618B61816B0A600F
:104198004A608C60CA600A614A618B6110BD800008
:1041A80000F1204019B1036843F0010302E00268FE
:1041B800014B134003607047FEFF0F0010280CBF2F
:1041C800054B064B4022182119605A604FF0FC320B
:1041D8009A60DA60704700BF600000A0800000A00D
:1041E8004268836830B51343C26843F008031A4332
:1041F8000369C46913434269616843EA42238269D7
:10420800056A43EA4233A2680068120442EA0122BE
:104218002168102842EA0102E168AC6842EA0161BB
:104228006A684FEA044444EA02242A6808BF064838
:1042380042EA0402EC6818BF044842EA04620360D8
:104248008160C26030BD00BF600000A0800000A097
:1042580010230360C269002343608360C360036165
:1042680043618361FC23136053609360D360026AE7
:10427800136053609360D360704739B110280CBF46
:10428800074A084A136843F0040306E010280CBFE5
:10429800034A044A044B11680B401360704700BF7F
:1042A800600000A0800000A0FBFF0F0039B11028BB
:1042B8000CBF074A074A136843F0400306E010287A
:1042C8000CBF034A034A044B11680B401360704744
:1042D800600000A0800000A0BFFF0F0010280CBFE6
:1042E800014B024B58697047600000A0800000A095
:1042F800054B18221A6000225A604FF0FC329A606F
:10430800DA601A61704700BFA00000A00368426825
:1043180043F0100343EA42238268154910B543EA83
:104328004233C4680B60A2686368120442EA03223D
:1043380023681343E268046943EA02638B60A26856
:104348006368120442EA0322236840691343E2685F
:1043580043EA0263CB6082684368120442EA03229C
:1043680003681343C26843EA02630B6110BD00BFD0
:10437800A00000A0C2680023036043608360FC23A0
:10438800136053609360D360026913605360936055
:10439800D3604269136053609360D3607047054BE4
:1043A80018B11A6842F0040202E01968024A0A4089
:1043B8001A607047A00000A0FBFF0F005AB1102838
:1043C80001D10C4A04E0B0F5807F0CBF0A4A0B4AC1
:1043D800536819430CE010286FEA010101D1054A1E
:1043E80004E0B0F5807F0CBF034A044A53681940C3
:1043F80051607047600000A0800000A0A00000A0ED
:10440800102801D1064B04E0B0F5807F0CBF054BA6
:10441800054B5B680B4214BF01200020704700BFAA
:10442800600000A0800000A0A00000A010286FEA93
:10443800010101D1054A04E0B0F5807F0CBF044AB0
:10444800044A536819405160704700BF600000A0DB
:10445800800000A0A00000A0102801D1084B04E0B3
:10446800B0F5807F0CBF074B074B5B6813EA010070
:1044780004D013EAD10314BF01200020704700BF05
:10448800600000A0800000A0A00000A010284FEA53
:10449800D10101D1054A04E0B0F5807F0CBF044A80
:1044A800044A536823EA010151607047600000A084
:1044B800800000A0A00000A008B52C4B984205D1B0
:1044C8000120014600F078FA012048E0284B984284
:1044D80005D10220012100F06FFA02203FE0254BB0
:1044E800984205D10420012100F066FA042036E044
:1044F800214B984205D10820012100F05DFA0820DF
:104508002DE01E4B984205D11020012100F054FAED
:10451800102024E01A4B984205D12020012100F0F8
:104528004BFA20201BE0174B984205D1402001216F
:1045380000F042FA402012E0134B984205D1802047
:10454800012100F039FA802009E0104B98420BD184
:104558004FF48070012100F02FFA4FF48070002191
:10456800BDE8084000F028BA08BD00BF00000240BE
:104578000004024000080240000C02400010024003
:104588000014024000180240001C024000200240B3
:10459800F0B50E6800220123934003EA060E9E45FB
:1045A8002AD155000323AB40DB4304681C40046058
:1045B8000C79076804FA05FC013C4CEA0707012C52
:1045C800076011D884684F791C4084608468AF40C4
:1045D80027438760446824EA0E0444608C7947685E
:1045E8009440A4B23C434460C4682340C360CB7980
:1045F800C468AB402343C3600132102ACBD1F0BD5D
:104608004FF6FF7303600023037143718371C37115
:10461800704782B04FF480330193019B0B430193A1
:10462800019BC361C161019BC361C3690193C369F4
:10463800019302B070470369194214BF012000209A
:104648007047006980B270474369194214BF01205E
:1046580000207047406980B27047018370474183EA
:1046680070470AB1018370474183704741617047C1
:10467800436959404161704701F00703C90800EBDD
:10468800810010B59B00046A0F21994024EA0101BA
:104698000162016A9A401143016210BD014B186022
:1046A800704700BF00300040014B5860704700BFA2
:1046B80000300040014B9860704700BF0030004058
:1046C8004AF6AA22014B1A60704700BF003000402A
:1046D8004CF6CC42014B1A60704700BF00300040D6
:1046E800034BDB68184214BF01200020704700BF4D
:1046F800003000400A4B00211A6842F001021A609B
:1047080099601A6822F0847222F480321A60054A8D
:104718005A601A6822F480221A60D960704700BF74
:104728000038024010300024024B00221A70187022
:10473800704700BF02380240034A136823F0F803A9
:1047480043EAC0001060704700380240014B18600F
:10475800704700BF00004742064B002201281A702C
:104768001A7002D0042802D07047187070470522CA
:104778001A70704770380240014B1860704700BFCC
:10478800800E474210B5029C5B0840EA0460014372
:10479800013B41EA821242EA0340014B586010BDD6
:1047A80000380240014B1860704700BF6000474264
:1047B8000907034B41EA8010C3F88400704700BF23
:1047C80000380240014B1860704700BF680047423C
:1047D800014B1860704700BF4C004742034A93687A
:1047E80023F0EC6319430843906070470038024097
:1047F800034A936823F0784319430843906070474D
:1048080000380240034A936823F00303184390607A
:10481800704700BF00380240024B986800F00C0057
:10482800704700BF00380240034A936823F0F00342
:1048380018439060704700BF00380240034A9368ED
:1048480023F4E05318439060704700BF00380240DB
:10485800034A936823F4604343EAC00090607047BA
:10486800003802401D4A10B5936803F00C03042B6E
:1048780003D0082B03D01A4B18E01A4B16E05168E6
:10488800536811F4800F516814BF164A144A03F094
:104898003F03B2FBF3F3114AC1F3881152684B434B
:1048A800C2F3014201325200B3FBF2F30B4A036038
:1048B80093680D49C3F30313CC5C0368E34043607A
:1048C8009468C4F382240C5D23FA04F4846092682B
:1048D800C2F342328A5CD340C36010BD0038024044
:1048E8000024F40040787D010C00002000F440739F
:1048F800094AB3F5407F01BF936820F0704123F463
:10490800F81321F4407104BF0B439360136FC0F395
:104918000B0018431067704700380240014B1860BD
:10492800704700BF3C0E4742014B1860704700BFFC
:10493800400E4742014B1860704700BF5C01474278
:10494800044B1A6B09B1104301E022EA0000186316
:10495800704700BF00380240044B5A6B09B110433E
:1049680001E022EA00005863704700BF00380240A7
:10497800044B9A6B09B1104301E022EA00009863E6
:10498800704700BF00380240044B1A6C09B110434D
:1049980001E022EA00001864704700BF00380240B6
:1049A800044B5A6C09B1104301E022EA0000586434
:1049B800704700BF00380240044B1A6909B1104320
:1049C80001E022EA00001861704700BF0038024089
:1049D800044B5A6909B1104301E022EA000058610A
:1049E800704700BF00380240044B9A6909B1104370
:1049F80001E022EA00009861704700BF00380240D9
:104A0800044B1A6A09B1104301E022EA0000186257
:104A1800704700BF00380240044B5A6A09B110437E
:104A280001E022EA00005862704700BF00380240E7
:104A3800044B1A6D09B1104301E022EA0000186521
:104A4800704700BF00380240044B5A6D09B110434B
:104A580001E022EA00005865704700BF00380240B4
:104A6800044B9A6D09B1104301E022EA00009865F1
:104A7800704700BF00380240044B1A6E09B110435A
:104A880001E022EA00001866704700BF00380240C3
:104A9800044B5A6E09B1104301E022EA000058663F
:104AA800704700BF00380240044B1A7809B1104320
:104AB80001E022EA00001870704700BF0D3802407C
:104AC8004209012A074B01D11B6803E0022A0CBFE7
:104AD8001B6F5B6F00F01F0023FA00F000F001006D
:104AE800704700BF0038024007B50023019331200A
:104AF800FFF7E6FF019B01330193019BB3F5A06F1C
:104B080001D00028F3D03120FFF7DAFF003018BFBA
:104B1800012003B05DF804FB024A536F43F0807331
:104B28005367704700380240034BDB68184214BFD4
:104B380001200020704700BF00380240014B187068
:104B4800704700BF0E38024008B540200121FFF72A
:104B58003FFFBDE8084040200021FFF739BF054B63
:104B68001A6810B142F0040201E022F004021A604F
:104B7800704700BF00080650014B9868704700BF97
:104B880000080650044B1A6810B142F0080201E010
:104B980022F008021A60704700080650034B5B6851
:104BA800184214BF01200020704700BF00080650BB
:104BB8006FEA0010014B5860704700BF00080650AC
:104BC800034B5B68184214BF01200020704700BFE8
:104BD80000080650C043024BC0B25860704700BF7F
:104BE8000008065008B5154B98420BD14FF4805079
:104BF8000121FFF711FFBDE808404FF48050002164
:104C0800FFF70ABF0E4B984207D14FF480400121AD
:104C1800FFF7F6FE4FF4804009E00A4B98420BD1AB
:104C28004FF400400121FFF7EBFE4FF40040002154
:104C3800BDE80840FFF7E4BE08BD00BF00300140F2
:104C480000380040003C004003884A8810B503F44F
:104C580041540B8813438A881343CA8813430A892B
:104C680013434A8913438A891343CA891343234345
:104C78009BB20380838B23F400631B041B0C838388
:104C88000B8A038210BD838BF0B523F47B6323F07A
:104C98000F031B041B0C8383022303848B68848B00
:104CA800022BA4B23AD02A4F8A88002ABA6814BFC5
:104CB8004FF0020E4FF0010E120242BFBA6822F402
:104CC8000002BA60D7F88460D7F884507A68C6F3CF
:104CD800881602F03F071F4AC5F30275B2FBF7F2C8
:104CE8005643B6FBF5F5CA88B2F5007F1CBF4FEAFC
:104CF8004E16B5FBF6F54FF00A0208BF2D0A6A43B7
:104D0800B2FBF3F305330A229BB2B3FBF2F303F0D1
:104D180001021202C3F34F0392B200E000229D1E6B
:104D2800ADB2FE2D24BF002202231343CA881343C9
:104D38009BB203840B888A881C434B8844F4006424
:104D4800234313438A8913439BB28383F0BD00BF77
:104D58000038024040787D0100230380438083802F
:104D6800C380038143818381C38107230382704702
:104D780000230222038043808380C3808260838172
:104D88007047038819B19BB243F0400303E023F056
:104D980040031B041B0C03807047838B19B19BB223
:104DA80043F4806303E023F480631B041B0C8383B8
:104DB8007047038823F400631B041B0C03800388DB
:104DC8009BB21943018070470388B1F5804F15BF26
:104DD80023F480439BB21B0443F4804318BF1B0C8D
:104DE800038070474FF6FF63994203880BBF23F493
:104DF80080739BB21B0443F4807308BF1B0C0380B1
:104E08007047838819B19BB243F0040303E023F091
:104E180004031B041B0C83807047838819B19BB261
:104E280043F0100303E023F010031B041B0C8380E2
:104E38007047808980B2704781817047038819B1B3
:104E48009BB243F4005303E023F400531B041B0CF0
:104E58000380704703889BB243F4805303807047F4
:104E6800012914BF008B808A80B27047008A80B203
:104E7800704783889BB20AB1194301E023EA010114
:104E880081807047090901238B409BB21AB182883F
:104E980092B2134303E0828892B222EA030383802A
:104EA80070470389194214BF012000207047C94385
:104EB80089B20181704710B584880389012201F005
:104EC8000F009BB202FA00F01840A4B205D00909FD
:104ED8008A40144214BF0120002010BD01F00F01C8
:104EE80001238B40DB439BB20381704708B54FF425
:104EF80080400121FFF790FDBDE808404FF4804055
:104F08000021FFF789BD014B186070470038014048
:104F180001F0030301F0FC0101F1804101F59C312E
:104F280010B59B008C680F229A4024EA02028A601E
:104F38008A68984002438A6010BD014B1860704728
:104F4800DC002742014B1860704700BF000427426D
:104F5800024B186AC0F30020704700BF00380140B8
:104F680008B5234B984205D110200121FFF754FDC5
:104F7800102037E01F4B984207D14FF40030012131
:104F8800FFF73EFD4FF4003009E01B4B98420BD170
:104F98004FF480200121FFF733FD4FF480200021DA
:104FA800BDE80840FFF72CBD144B984207D14FF4D9
:104FB80000200121FFF724FD4FF40020EFE7104BFC
:104FC800984207D14FF480100121FFF719FD4FF4E3
:104FD8008010E4E70B4B984209D120200121FFF70C
:104FE8001BFD20200021BDE80840FFF715BD08BDC6
:104FF800001001400044004000480040004C0040C0
:1050080000500040001401407FB50E460446038A54
:10501800CA889BB223F440531343038283890989C6
:105028009BB223F4B05323F00C02B3880B4371896D
:105038000B439BB213438381838AB2899BB223F4C7
:105048004073134383826846FFF70CFC194B9C425C
:1050580003D003F580639C4201D1039D00E0029DCB
:10506800A38919226A4331681BB2002BB4BF4D00D3
:105078008D00B2FBF5F56426B5FBF6F000010109D9
:1050880006FB1153A28912B2002AADBF1A01D9003A
:1050980032313232B5BFB1FBF6F2B2FBF6F302F0B1
:1050A800070203F00F03B4BF1043184380B22081F6
:1050B80004B070BD001001404FF4165303600C2279
:1050C80000238380C3800381428183817047038AE0
:1050D80010B59BB24C8823F470620B8823438C88EC
:1050E800C98823430B439BB21343038210BD00239B
:1050F800038043808380C3807047838919B19BB242
:1051080043F4005303E023F400531B041B0C838176
:105118007047038B03F47F430383038B9BB21943CC
:1051280001837047838929B16FEA43436FEA534388
:105138009BB201E0C3F30E0383817047838A19B1E0
:105148009BB243F4006303E023F400631B041B0CCD
:1051580083827047C1F30801818070478088C0F35B
:1051680008007047038A23F00F031B041B0C0382FB
:10517800038A9BB2194301827047838919B19BB294
:1051880043F0020303E023F002031B041B0C83819A
:105198007047838923F400631B041B0C8381838974
:1051A8009BB2194381817047038A23F020031B04B3
:1051B8001B0C0382038A9BB2194301827047038A3E
:1051C80019B19BB243F4804303E023F480431B04EA
:1051D8001B0C0382704783899BB243F001038381D0
:1051E8007047838A19B19BB243F0080303E023F0A8
:1051F80008031B041B0C83827047038BDBB20383F9
:10520800038B9BB243EA012101837047838A19B15A
:105218009BB243F0200303E023F020031B041B0C84
:1052280083827047838A19B19BB243F0100303E06D
:1052380023F010031B041B0C83827047838A23F01E
:1052480004031B041B0C8382838A9BB2194381824B
:105258007047838A19B19BB243F0020303E023F03D
:1052680002031B041B0C83827047838A9BB20AB11A
:10527800194301E023EA01018182704710B5C1F3A7
:105288004214012301F01F01012C03FA01F301D19B
:105298000C3003E0022C0CBF1030143012B102683D
:1052A800134302E0026822EA0303036010BD038887
:1052B800194214BF012000207047C94389B20180F8
:1052C8007047012310B5C1F3421401F01F029C423C
:1052D80003FA02F201D1838903E0022C0CBF038A8E
:1052E800838A9BB21340028892B23BB1090A012318
:1052F8008B40134214BF0120002010BD184610BD7A
:10530800090A01238B40DB439BB20380704700BF2F
:1053180008B5062004210022FBF754FA08BD00BF97
:1053280010B50446FBF7A6FC2046FBF7C1FC10BDF0
:10533800F0B583B0074602AC44F8041D4FF0FF36C1
:1053480000253846214632462B46FBF7CFFA01287E
:10535800F7D103B0F0BD00BF00B583B002AB43F88E
:10536800041D194600221346FBF7C0FA10F1FF305E
:1053780018BF4FF0FF3003B05DF804FB2DE9F04192
:1053880082B005460C461646FCF7CEF9804604B9AD
:1053980001AC8EB12846214632460023FBF770FB4C
:1053A800012804D1FCF7C0F9C8EB000013E0002382
:1053B80023604FF0FF300EE04FF0FF3700262846FD
:1053C80021463A463346FBF75BFB0128F7D1FCF749
:1053D800ABF9C8EB000002B0BDE8F08100B583B0BE
:1053E8000B4601B901AB194600221346FBF748FBEF
:1053F80010F1FF3018BF4FF0FF3003B05DF804FB29
:1054080038B50546012000210322FBF7DBF970B10E
:10541800044600210A460B46FBF768FA4DB92046B8
:10542800002101220B46FBF72BFB204638BD00204C
:1054380038BD204638BD00BFF8B504460D46FCF718
:1054480073F907465DB1204600212A460B46FBF753
:1054580017FB012812D1FCF767F9C01BF8BD00261D
:105468004FF0FF35204631462A463346FBF708FB06
:105478000128F7D1FCF758F9C01BF8BD4FF0FF30F1
:10548800F8BD00BF08B500210A460B46FBF72EFA07
:1054980008BD00BF08B5FBF70BFC08BD07490B1D8D
:1054A800CC3100221A6043F8042C08338B42F9D11E
:1054B8000022024BA3F8C820704700BF501F0020ED
:1054C80010B5FCF773FD0D4BB3F8C840A4B15B6889
:1054D80083420AD104E008325168814207D100E0D2
:1054E8000023064800EBC30010BD044A0023013323
:1054F800A342F0D1002010BD002010BD501F002095
:1055080070B586B0124CB4F8C840182C1DD80646A1
:1055180015460A9A009205AA01920024029403945F
:10552800084631469AB22B46FBF724FD0146084B44
:10553800B3F8C820501CA3F8C800059803EBC203B1
:105548005860012918BF204600E0002006B070BD51
:10555800501F002008B5FAF765FF012008BD00BFFD
:1055680008B5FAF771FF08BD08B5FAF75BFFFEE763
:1055780030B50D4687B0114600F0B8FB044698B127
:105588000C4B029001A801938DF80C5002F024FEF8
:1055980094F9083053B1E068FFF77CFF2069FFF702
:1055A800BFFE204604F000FF002000E0204607B0C0
:1055B80030BD00BF5B5C000810B5044686B050B132
:1055C800064B029001A8019302F006FE00236360D7
:1055D800204600F0CFFB002006B010BD395E000861
:1055E80010B5044686B068B161B15AB10748029453
:1055F800019001A8039104928DF8143002F0ECFD9B
:10560800207A00E0F62040B206B010BDAB6000087A
:1056180010B5044686B050B1074B029001A801931B
:105628000391ADF8102002F0D7FD207A00E0F620B3
:1056380040B206B010BD00BF995E000810B5044620
:1056480086B050B1074B029001A801930391ADF8C1
:10565800102002F0C1FD207A00E0F62040B206B02A
:1056680010BD00BFEB5E000810B5044686B038B127
:10567800054B029001A8019302F0AEFD207A00E0EC
:10568800F62040B206B010BD515F000810B50446C0
:1056980086B038B1054B029001A8019302F09CFD39
:1056A800207A00E0F62040B206B010BD735F000813
:1056B80013B5044690B1406980B101A9E269FFF7CA
:1056C8005DFE013002D10023019305E0E36A1BB1BE
:1056D80020460121002298470198FFE702B010BD3B
:1056E80030B5002589B00195044618B1006918B98C
:1056F800F8232372002058E094F908300433F9DBCA
:105708002378102B3DD16378022BF1D0284B988950
:1057180004F05CFF019008B9FF2320E0206902A98A
:10572800E269FFF72BFE013004D1019804F03CFE3A
:10573800FD23DEE7029A1AB11289238C9B1A23846F
:10574800E36A13B1204601219847029B4BB901989F
:1057580004F02AFE94F908000028CBD1F92323721B
:1057680023E0019A002113605360916091811B89A5
:10577800104A03A803920494ADF8143002F02CFDEB
:1057880012E001A9E269FFF7F9FD013008BF0195B0
:10579800019B4BB11B681A89238C9B1A2384E36AEB
:1057A80013B1204601219847019809B030BD00BFC8
:1057B800C82603085360000810B5044686B040B1F7
:1057C800064B029001A80193039102F005FD207A8F
:1057D80000E0F62040B206B010BD00BFFD5F000833
:1057E80010B529B1BDE810408A608B81FFF7E4BF8E
:1057F8006FF0080010BD10B5044686B070B100788F
:1058080010280DD108480294019001A803918DF841
:105818001430049202F0E0FC207A02E0F62000E066
:10582800F72040B206B010BD7D60000810B50446F0
:1058380086B038B1054B029001A8019302F0CCFC68
:10584800207A00E0F62040B206B010BD1F610008C3
:1058580070B50D4686B00646C8B1C1B10020FFF745
:10586800CFFD0446A8B10DF1070302A90122049057
:105878000A4805930296039502F044FC204605F079
:1058880017FB2046FFF706FE9DF8070002E0F6200A
:1058980000E0FF2040B206B070BD00BF3F610008C5
:1058A800D36811B9F721197004E000201870536803
:1058B800096819609068FFF7E5BD70B511460446A0
:1058C800A0B1006990B1237222B11689238C3344A8
:1058D800238400E01646FFF73FFD054640B9E36A1A
:1058E8003BB1204629463246984702E0F72500E0BA
:1058F800FF2568B270BDF8B50F4614460546002866
:1059080030D0036973B311890320002205F03DF8F4
:10591800064638B3214605F026F918B1304605F099
:1059280021F81FE0104B988904F050FE0446002827
:10593800F4D0736826600C336660A3603B7C214614
:10594800A3812869FFF708FD014618B1204600F039
:1059580017FC07E032892B8C13442B84EB6A0BB1BC
:10596800284698470020F8BDC826030810B54468A3
:105978000146204605F07BFC2046094905F079FCE4
:105988002046084905F078FC20460749042205F01E
:105998007BFC2046BDE81040044905F070BC00BF00
:1059A800C3580008215C00089D5B0008E159000805
:1059B80038B5054668B103780272102B02D10AB9CE
:1059C800FFF7D4FF0024E8686C70FFF75BFD204602
:1059D80000E0F72040B238BD0369002210B5044644
:1059E800426001723BB1C36A0BB111469847206906
:1059F8000021FFF79DFCE06830B16378032B03D1E9
:105A080000236370FFF73EFD63694BB1E36A1BB186
:105A1800002120460A46984760690021FFF788FC64
:105A28006378012B01D0042B06D100236370E06852
:105A3800BDE81040FFF726BD10BD70B5466A826A02
:105A4800B36804469B1AB3F5803F28BF4FF6FF732F
:105A5800406838BF9BB2B0F86E5071689D4228BF4D
:105A68001D461144337B2A4606F0B8FF00282FD183
:105A7800A36A626A2B44A36292689342636808BF70
:105A880060629A6F03BFA06260700126064662B129
:105A980093F8222012F0440F07D15A6F42B11168CF
:105AA80019B991891A8F914202D3184606F0E0FF7E
:105AB8002072A8B96368B3F86E2041F684439A420D
:105AC8000ED8E36A63B1204603212A46984707E0C7
:105AD800431C03D1606806F0CBFF07E0207200E0AA
:105AE80026B100236370E068FFF7CCFC002070BD8E
:105AF80010B504460021406805F0B9FB6068002134
:105B0800037C012B02D105F0BDFB12E005F0B1FBCF
:105B18006068002105F0B6FB6068002105F0ACFB69
:105B280060680021042205F0AFFB6068002105F0E1
:105B3800A6FB606805F010FD014690B9E36A607045
:105B48006060207213B120460A469847E36A1BB189
:105B58002046022100229847E068BDE81040FFF780
:105B680091BC6068084905F087FB60680749042212
:105B780005F08AFB6068064905F081FB60682146EC
:105B8800BDE8104005F073BB215C00089D5B000870
:105B9800E159000808B54378012B02D1FFF74DFF02
:105BA80003E0042B01D1FFF7A3FF002008BD2DE976
:105BB800F04116469846BDF81870044608B10369C6
:105BC80023B93046BDE8F04104F0CCBE114B9889AA
:105BD80004F0FCFC05460028F3D006604660C0F8D7
:105BE8000880878129462069FFF7B6FB014620B166
:105BF8002846BDE8F04100F0C3BA3289238C13442B
:105C08002384E36A1BB12046BDE8F0411847BDE88C
:105C1800F08100BFC826030838B543780446012B35
:105C2800154602D1FFF709FF03E0042B01D1FFF766
:105C38005FFF63685BB1B3F86E2041F684439A4214
:105C480005D9E36A1BB1204602212A46984700205D
:105C580038BD38B5036804465A68002A3BD11A7221
:105C680005682B7803F0F003202B12D0402B02D0CC
:105C7800102B2ED121E0007905F0CEF8686022685B
:105C8800506810B9FF23137225E0164905F064F82F
:105C980021E007F035FB686023685A6812B9FF22D3
:105CA8001A7218E01B781049222B04BF01231374C1
:105CB8002268506807F00CFB0DE005F0B9FD68603C
:105CC8002068436813B9FF23037204E0FFF74EFE10
:105CD80001E0F7232B722368D868BDE83840FFF746
:105CE800D1BB00BFFF580008B75B0008F8B5204BD0
:105CF8000646D8890F4604F069FC002504460028AA
:105D080033D005720670456006F0F000202806D0F2
:105D1800402806D0102808BF4FF4FA6501E04FF478
:105D2800FA650020FFF76CFB0646E06020B92046C4
:105D380004F03AFB3046F8BD2846FFF7E9FA054675
:105D4800206138B9E068FFF7A5FB204604F02CFB7A
:105D58002846F8BD00234FF0FF3263616370A261EB
:105D6800E76223846362A362E3612046F8BD00BF53
:105D7800C8260308036913B50446B3B1206901A90D
:105D8800FFF72CFB01300BD023780198102B04D19E
:105D98000028F3D004F0E6FDF0E700F0F1F9EDE7B4
:105DA8002069FFF7BDFA00232361636973B1606955
:105DB80001A9FFF713FB013003D00198FFF7FCFBA3
:105DC800F5E76069FFF7ACFA00236361E068FFF765
:105DD80061FB0023E360204604F0E6FA02B010BD40
:105DE800F8B5436905460F461446E3B10078E96AF9
:105DF800FFF77CFF0646C0B14760FFF7B7FD347276
:105E080068693146FFF7A8FA044628B10023736091
:105E18003046FFF7AFFF08E0EB6A3BB12846214662
:105E28002246984702E0F72400E0FF2460B2F8BD5C
:105E380010B5036804465868B0B11A7802F0F00249
:105E4800202A0CD0402A07D0102A0DD1BDE81040D6
:105E580004225A7018464BE604F0C9FF04E00022F9
:105E6800C261586807F037FA2068C36A13B1002185
:105E78000A4698472068C36A13B10221002298474E
:105E88002368D86818B1BDE81040FFF7FBBA10BD09
:105E980038B50568044695F9083004331BDB686893
:105EA800B8B12B7803F0F003202B0CD0402B06D090
:105EB800102B10D16168228905F0DAF807E06168D3
:105EC80004F040FF03E06168228907F01DF9287299
:105ED80001E0F7232B722368D868BDE83840FFF744
:105EE800D1BA38B505680446686808B9E86824E096
:105EF8002B7803F0F003202B15D0402B0FD0102B5C
:105F080017D103236B702846FFF730FD25686168B9
:105F1800686822890B4B05F09DFC287238BD6168C2
:105F280004F015FF03E06168228907F0A0F92872E0
:105F380001E0F7232B722368D868BDE83840FFF7E3
:105F4800A1BA00BFB9590008026810B51378044611
:105F580003F0F003202B02D1506807F0ADF9236855
:105F6800BDE81040D868FFF78DBA70B503680446DD
:105F780093F90820043234DB5868002831D01A78A5
:105F8800102A2ED1067C56BBFF2105F0D1F82368D4
:105F9800054608B9FF2223E0186918B1FFF7C0F9D0
:105FA80023681E612668736943B94FF4FA60FFF7E6
:105FB800AFF9706110B92368FF221A72236893F948
:105FC800082072B95D60216802225A70486805F09D
:105FD8004EF923680649586805F054F901E0F8229B
:105FE8001A722368BDE87040D868FFF74BBA00BF43
:105FF800E95D000838B50468054694F908300433AB
:106008001DDB6068D8B1237803F0F003202B0BD098
:10601800402B14D16B689A68196812B904F0E4FE31
:106028000CE004F09CFE09E06B689A68196812B9E4
:1060380007F019F902E09B8907F000F920722B6834
:10604800D868BDE83840FFF71DBA10B503680446A4
:1060580093F90820043207DB586828B11B78102B05
:1060680002D1A18805F0C9F82368BDE81040D868B6
:10607800FFF708BA036893F9082004320DDB5A6861
:106088004AB11A78102A06D101225A7000225862A1
:106098009A621846D1E4F7221A720368D868FFF7A3
:1060A800F1B910B503685A68002A2CD0047B4168FE
:1060B8000CB1126800E052680A601A7802F0F00227
:1060C800202A0AD0402A02D0102A1ED112E0027BD0
:1060D800CAB15B6882681B7C13E0017B5A6811B106
:1060E8008368528A04E0117C49070CD58368928A38
:1060F8001A800AE0017B82685B6809B11B8B00E0AB
:106108001B8C138001E0F8221A720368BDE8104066
:10611800D868FFF7B7B903685A6832B11A78102AF5
:1061280003D104225A701846E2E4F7221A7203686F
:10613800D868FFF7A7B938B50446C568234603C829
:10614800074A03F065F92870E36893F900300E33C5
:1061580004D0A068BDE83840FFF794B938BD00BF47
:10616800A958000808B5054B988904F02FFA20B102
:106178000023036043608360838108BDC826030849
:1061880010B5044658B1006820B104F0EBFB0023B9
:10619800636023602046BDE8104004F005B910BDD7
:1061A80038B50D46044608B9002038BD006808B166
:1061B80004F0D8FB00202946024604F0E6FB2060E4
:1061C8000028F1D06060406838BD10B5044630B191
:1061D800006808B104F0C6FB00236360236010BDAB
:1061E80070B50E461546044698B1006808B104F02B
:1061F800B9FB00200146022204F0C7FB206010B959
:106208006060FF2006E046600581458160600020EF
:1062180000E0F62040B270BD38B50D46044658B1CE
:1062280051B10068096804F071FC2368284663606E
:10623800BDE8384004F0B8B838BD50B149B142B1F2
:10624800436843B15B680B60436800205B89138037
:1062580002E0F62000E0FE2040B2704740B14368FB
:106268001B682BB143601868B0FA80F0400900E061
:10627800FF2040B2704708B103684360704700BF11
:1062880013B501A90446FFF7E3FA20B10C4BD2225B
:106298001A60002011E00B4B019803F114029A6177
:1062A8001A465861184642F81C4B5A6002229A60F6
:1062B8000422DA6003F118021A6102B010BD00BFAF
:1062C800586F00201C2000202DE9F74F0D9E8046B6
:1062D8000F4615461C4606B901AE0C9B3BB10C9AFD
:1062E80000231360B8F1000F01D007B10DB91623D0
:1062F80017E0404623F0A6FD00F1100294428246C2
:1063080001D222230DE0033525F0030505F1040B26
:1063180040465946FFF79CFA05F10C09044620B19E
:10632800A32333604FF0FF3016E0524648464146FB
:1063380020F008F82A462046022309F80A40C5F842
:1063480000B042F8084FBB600423FB600C9BC7F801
:1063580000907A603D611F6003B0BDE8F08F10B512
:1063680020B1C46904F020F82046F9E710BD2DE9F2
:10637800F74F0646914608469A460BB9CA2061E08F
:106388000023CAF800300EB909B956E049B121F026
:106398009BFD4FF6FE73421E9A4205464FD80EB932
:1063A8000DE00D46304601A9FFF752FA0028E5D165
:1063B800304623F047FD074600F1310806E0234840
:1063C80003F0ECF9374601904FF030081FFA88F0D7
:1063D80004F0FCF80446A0B34246002123F0AEF9CD
:1063E800019B4FF0020B6362102384F821B084F8FC
:1063F8002030A8B203F0CCF904F120086084C4F876
:1064080004B0B9F1000F05D0D9F80830A360D9F865
:106418000C30E3604EB104F130033A46A3611846EC
:1064280031461FF08FFF0022C25510232361C4F8A4
:1064380014800020CAF8004004E0C82002E0C92007
:1064480000E0CB2003B0BDE8F08F00BF0100007F63
:1064580080B500AF0120FEF7D3FF0246044B1A6057
:106468000120FEF7CDFF0246024B1A6080BD00BF37
:10647800082100200C21002080B485B000AF78608E
:106488007B68002B02DB7B68092B01DD00230EE013
:106498007A6813469B0013449B00084A1344FB6028
:1064A800FB681B68002B01D1002300E0FB6818463D
:1064B8001437BD465DF8047B704700BF3C200020C0
:1064C80080B584B000AF786039607868FFF7D4FF92
:1064D800F860FB681B683A68DA611037BD4680BD12
:1064E80080B584B000AF78607868FFF7C5FFF860C2
:1064F800FB681B681B7A5BB218461037BD4680BD27
:1065080080B584B000AF7860364B1B68184604F03D
:10651800CFFC0023FB6057E03349FA6813469B0021
:1065280013449B000B441B68002B4AD12E49FA6880
:1065380013469B0013449B000B447A681A602A494F
:10654800FA6813469B0013449B000B4400225A60D0
:106558002549FA6813469B0013449B000B440833F3
:1065680000221A802049FA6813469B0013449B00B6
:106578000B44083300225A801B49FA6813469B00D3
:1065880013449B000B44083301229A801649FA6889
:1065980013469B0013449B000B4408330022DA8007
:1065A8001149FA6813469B0013449B000B441033AF
:1065B80000221A600B4B1B681846FEF763FFFB6846
:1065C8000CE0FB680133FB60FB68092BA4DD054B7D
:1065D8001B681846FEF756FF4FF0FF331846103772
:1065E800BD4680BD082100203C20002080B590B029
:1065F80000AFF860B9607A60F868FFF73DFFF863AC
:10660800FB6B002B02D14FF0FF33B5E0FB6BDB894E
:1066180003F40063002B0AD0FB6B5B891BB2002BD1
:1066280005DCFB6B0B221A614FF0FF33A4E0FB6B18
:106638001B681846FFF73CF8B863BB6B002B15D1F5
:10664800FB6B1B681B7A5BB25B420E2B08D8FB6B9B
:106658001B681B7A5BB25B42494A52F8233000E060
:106668000523FA6B13614FF0FF3385E007F1280229
:1066780007F12603B86B11461A460023FEF7B0FF50
:10668800034687F8373097F93730002B14D0B86BAA
:10669800FEF792FF97F937305B420E2B06D897F931
:1066A80037305B42364A52F8233000E00523FA6B54
:1066B80013614FF0FF335FE0BB68002B22D007F176
:1066C800140318460021102223F038F810233B75D4
:1066D80002237B75FB8C184603F05AF80346FB82AD
:1066E800BB6ABB617B681B68102B02D97B681022D0
:1066F8001A607B681B6807F11402B86811461A46CD
:106708001FF020FEB86BFFF7FBFE38633B6BB3F15D
:10671800FF3F08D1B86BFEF74FFFFB6B17221A61DA
:106728004FF0FF3328E0BB6B164ADA623A6B134628
:106738009B0013449B00144A1344FB62134B1B68D1
:10674800184604F0B5FBFB6A5B899AB2BB6B9B6980
:106758009BB2D31A9BB2013B9BB29AB2FB6A5A8195
:10676800BB6B3A6B9A61094B1B681846FEF78AFEA9
:10677800FB6B00221A613B6B18464037BD4680BD53
:10678800842603082D7500083C20002008210020DD
:1067980090B589B000AFF860B9607A60F868FFF723
:1067A8006BFEF861FB69002B02D14FF0FF333CE030
:1067B8007B68102B03D1BB685B78022B05D00522C0
:1067C800FB691A614FF0FF332FE0BB685B687B61A0
:1067D800BB685B887B83FB691C687B8B184602F06F
:1067E800DAFF03461A4607F1140320461946FEF756
:1067F8000FFF03467B7697F91930002B11D097F9D4
:1068080019305B420E2B06D897F919305B42094ABA
:1068180052F8233000E00523FA6913614FF0FF3383
:1068280003E0FB6900221A61002318462437BD469D
:1068380090BD00BF8426030880B584B000AF78609F
:106848007868FFF719FEF860FB68002B02D14FF05B
:10685800FF3324E0FB681B681846FEF7ADFE124BB9
:106868001B68184604F024FBFB685B68002B04D007
:10687800FB685B681846FFF783FCFB6800225A60D8
:10688800FB6800221A81FB6800221A60FB6800225C
:106898001A61054B1B681846FEF7F4FD00231846DD
:1068A8001037BD4680BD00BF0821002090B589B0D3
:1068B80000AFF860B9607A60F868FFF7DDFDB8618D
:1068C800BB69002B02D14FF0FF3348E07B68102BE7
:1068D80003D1BB685B78022B05D00522BB691A611E
:1068E8004FF0FF333BE0BB685B78002B07D1BB69F7
:1068F8001B681846FEF7B8FE0346FB7715E0BB6831
:106908005B683B61BB685B88FB82BB691C68FB8A70
:10691800184602F040FF03461A4607F110032046C6
:106928001946FEF78BFE0346FB7797F91F30002BBD
:1069380011D097F91F305B420E2B06D897F91F30FC
:106948005B42094A52F8233000E00523BA69136113
:106958004FF0FF3303E0BB6900221A610023184699
:106968002437BD4690BD00BF8426030880B584B097
:1069780000AF786039607868FFF77EFDF860FB68E3
:10698800002B02D14FF0FF332DE03B68002B01DADA
:1069980000233B603B68FF2B01DDFF233B60FB6866
:1069A8001A683B68DBB210461946FEF76FFE0346CD
:1069B800FB7297F90B30002B11D097F90B305B4223
:1069C8000E2B06D897F90B305B42094A52F8233050
:1069D80000E00523FA6813614FF0FF3303E0FB681A
:1069E80000221A61002318461037BD4680BD00BF3B
:1069F8008426030880B58EB000AFF860B9607A606D
:106A08003B6000233B86002387F82B30F868FFF7AC
:106A180033FD78627B6A002B02D14FF0FF3312E11D
:106A28007B6A5B68002B03D07B6A5B687B6352E000
:106A38003B6803F00803002B05D17B6ADB8903F46C
:106A48000063002B12D07B6A5B891BB2002B0DDC24
:106A58003B8E002B04D07B6A00221A613B8EF2E049
:106A68007B6A0B221A614FF0FF33ECE07B6A1B68EC
:106A78001846FEF735FE78637B6A7A6B5A607B6B43
:106A8800002B28D13B8E002B04D07B6A00221A6190
:106A98003B8ED8E07B6A1B685B68002B04D07B6A5E
:106AA8001B681B7A002B11D07B6A1B681B7A5BB2B0
:106AB8005B420E2B08D87B6A1B681B7A5BB25B4271
:106AC800634A52F8233002E0052300E074237A6A0F
:106AD80013610023B7E07B6B1B681B897B847B6A8F
:106AE8001B897A8CD31A7B847A8C7B689A4202D26F
:106AF8007B8C7B8601E07B687B867B6B18683B8E92
:106B0800BA68D1187B6A1B897A8E04F076F83A8EB7
:106B18007B8E13443B867B6A1B681B78102B1BD12A
:106B28007B8E7A68D31A7B607B68002B10D07B6BD6
:106B38001B685B7B03F00103002B09D17B6A5B892F
:106B48001BB2002B04DD3B6803F00103002B06D0C9
:106B5800012387F82B3002E0012387F82B3097F8C0
:106B68002B30002B43D03B6C002B40D07B6C002B90
:106B78003DD07B6A1B681B78102B0ED107F11003E0
:106B88000433FB627B6A1A6807F120031046F96A2E
:106B98001A460023FEF724FD05E07B6B9B68FB6229
:106BA8007B6B9B893B8407F1100318460021102258
:106BB80022F0C4FD10233B7402237B743B8C1846DF
:106BC80002F0E6FD03467B82FB6A1B687B617B6CF7
:106BD8001B68102B02D97B6C10221A607B6C1B6817
:106BE80007F11002386C11461A461FF0ABFB3B68E0
:106BF80003F00103002B1DD17B6A1B681B78102B47
:106C08000FD17A8C7B8ED31A002B0ADD7B6A7A6BC4
:106C18005A607B6A1A897B8E13449AB27B6A1A81FE
:106C280008E07B6A00225A607B6A00221A81786B2E
:106C3800FFF7A6FA97F82B30002B3FF4F1AE7B6AEA
:106C480000221A613B8E18463837BD4680BD00BF0A
:106C58008426030880B586B002AFF860B9607A6010
:106C68000023009300230193F868B9687A68002329
:106C7800FFF7C0FE034618461037BD4680BD00BF6B
:106C880080B586B002AFF860B9607A603B600023D7
:106C9800009300230193F868B9687A683B68FFF7A6
:106CA800A9FE034618461037BD4680BD80B588B09A
:106CB80002AFF860B9607A603B60F868FFF7DCFB08
:106CC80078617B69002B02D14FF0FF3339E07B6993
:106CD8001B681B78102B0BD0002300930023019313
:106CE800F868B9687A683B6800F032F8034628E02B
:106CF8007B691A683B6803F01003002B01D003235B
:106D080000E001231046B9687A68FEF774FD03466F
:106D1800FB7497F913305B420E2B06D897F91330A2
:106D28005B420A4A52F8233000E005237A6913616E
:106D380097F91330002B01D17B6801E04FF0FF3346
:106D480000BF18461837BD4680BD00BF842603081B
:106D580080B58CB000AFF860B9607A603B60F868C5
:106D6800FFF78AFBB862BB6A002B02D14FF0FF33F2
:106D780077E0BB6A1B681B78102B07D1F868B968E5
:106D88007A683B68FFF792FF03466AE07B68FB84FA
:106D9800BB6B002B02D1FB6B002B0CD0FB6B102BB9
:106DA80003D1BB6B5B78022B05D00522BB6A1A6145
:106DB8004FF0FF3355E000237B617B693B61BB6B80
:106DC800002B0FD0BB6B5B683B62BB6B5B881846C4
:106DD80002F0E1FC0346BB8407F12003BB61BB8CD6
:106DE800BB8307E000233B620023BB840023BB6115
:106DF8000023BB8307F11002FB8C1046B9681A46C2
:106E0800FFF7EEF9034687F82F3097F92F30002B5C
:106E18000AD1BB6A1A6807F1100310461946FEF733
:106E2800CBFC034687F82F3007F110031846FFF70D
:106E3800CCF997F92F305B420E2B06D897F92F30F3
:106E48005B420A4A52F8233000E00523BA6A13610C
:106E580097F92F30002B01D1FB8C01E04FF0FF3365
:106E680000BF18463037BD4680BD00BF84260308E2
:106E780080B586B000AFF860B9607A60BB68022B55
:106E88000DD0032B02D0012B16D01CE07B68DBB29F
:106E9800402019461B4AFEF76BFB786116E07B68B9
:106EA800882B01D1212300E0202318460021154A10
:106EB800FEF75EFB786109E010200021114AFEF719
:106EC80057FB786102E04FF0FF3317E07B69002B36
:106ED80002D14FF0FF3311E07869FFF711FB3861F9
:106EE8003B69B3F1FF3F05D17869FEF765FB4FF0C9
:106EF800FF3303E07B693A699A613B6918461837A2
:106F0800BD4680BD2D75000880B584B000AFF8601F
:106F1800B9607A60F868B9687A680023FFF7C6FE36
:106F2800034618461037BD4680BD00BF80B596B0F1
:106F380000AFF860B9607A603B6000233B6507F1F9
:106F48002403BB640023FB6407E0BB6C5A1CBA64CF
:106F580000221A70FB6C0133FB64FB6C072BF4D91D
:106F680007F11C033B6400237B6407E03B6C5A1C5D
:106F78003A6400221A707B6C01337B647B6C072BAC
:106F8800F4D907F11403BB630023FB6307E0BB6B71
:106F98005A1CBA6300221A70FB6B0133FB63FB6B4C
:106FA800072BF4D900237B6569E07B6D5A09BB6820
:106FB80053F822207B6D03F01F0342FA03F303F01A
:106FC8000103002B27D0786DFFF756FAF862FB6AA9
:106FD800002B20D0FB6A5B68002B04D1FB6A5B891D
:106FE8001BB2002B17DD7B6D5A09930007F158017E
:106FF8000B4453F8341C7B6D03F01F03012000FA87
:1070080003F31943930007F15802134443F8341C5F
:107018003B6D01333B657B6D5A097B6853F8222031
:107028007B6D03F01F0342FA03F303F00103002B07
:1070380022D0786DFFF720FAF862FB6A002B1BD08C
:10704800FB6A9B89002B17D07B6D5A09930007F1C7
:1070580058010B4453F83C1C7B6D03F01F030120BF
:1070680000FA03F31943930007F15802134443F855
:107078003C1C3B6D01333B657B6D01337B657A6D51
:10708800FB689A4291DBBB681A4607F1240393E830
:10709800030082E803007B681A4607F11C0393E8A3
:1070A800030082E803003B683B6300237B6307E03F
:1070B8003B6B5A1C3A6300221A707B6B01337B636B
:1070C8007B6B072BF4D93B6D18465837BD4680BDFE
:1070D80080B5ACB000AFF860B9607A603B6000235F
:1070E8003B61BB687B617B68BB613B68FB610023DC
:1070F8003B62BB4B1B68184603F0DAFEBB68002BEB
:1071080007D0BA6807F1380392E8030083E8030060
:1071180017E007F13803C7F89C300023C7F8A03000
:107128000BE0D7F89C305A1CC7F89C2000221A7034
:10713800D7F8A0300133C7F8A030D7F8A030072B14
:10714800EFD97B68002B07D07A6807F1300392E803
:10715800030083E8030017E007F13003C7F8943011
:107168000023C7F898300BE0D7F894305A1CC7F8BA
:10717800942000221A70D7F898300133C7F8983055
:10718800D7F89830072BEFD93B68002B07D03A681F
:1071980007F1280392E8030083E8030017E007F1EA
:1071A8002803C7F88C300023C7F890300BE0D7F8D5
:1071B8008C305A1CC7F88C2000221A70D7F89030EF
:1071C8000133C7F89030D7F89030072BEFD907F183
:1071D800380107F1300207F12803F868FFF7A6FE27
:1071E800C7F8AC00D7F8AC30002B40F06C81D7F86A
:1071F800B830002B54D0D7F8B8301B68002B4FD1CB
:10720800D7F8B8305B68002B4AD1754B1B68184615
:10721800FEF738F9BB68002B16D0BB68C7F8843076
:107228000023C7F888300BE0D7F884305A1CC7F819
:10723800842000221A70D7F888300133C7F88830C4
:10724800D7F88830072BEFD97B68002B13D07B68E1
:10725800FB670023C7F8803009E0FB6F5A1CFA6708
:1072680000221A70D7F880300133C7F88030D7F879
:107278008030072BF1D93B68002B0FD03B687B6728
:107288000023BB6707E07B6F5A1C7A6700221A70DD
:10729800BB6F0133BB67BB6F072BF4D900233AE1FF
:1072A8000020FEF7ADF803467B624E4B1B683B613E
:1072B8004C4A07F110031360494B1B681846FEF748
:1072C800E1F8D7F8B830002B03D10023C7F8A8306D
:1072D8001BE0D7F8B8301B684FF47A7202FB03F250
:1072E800D7F8B8305B6803F5FA733F4981FB0301AF
:1072F8008911DB17CB1A1344C7F8A830D7F8A83080
:10730800002B02D10123C7F8A8307B6A1846D7F8AA
:10731800A81003F04CFE3864314B1B68184603F084
:10732800C7FD304B1A6807F110039A4203D13B6935
:107338002C4A136019E02B4B1B68C7F8A43010E0E7
:10734800D7F8A4301A6807F110039A4204D13A69B1
:10735800D7F8A4301A6008E0D7F8A4301B68C7F83B
:10736800A430D7F8A430002BEAD11D4B1B6818466F
:10737800FEF788F87B6A1846FEF78CF83B6C002B02
:1073880041D1BB68002B0FD0BB68FB6600233B676D
:1073980007E0FB6E5A1CFA6600221A703B6F013335
:1073A8003B673B6F072BF4D97B68002B0FD07B68BA
:1073B8007B660023BB6607E07B6E5A1C7A66002258
:1073C8001A70BB6E0133BB66BB6E072BF4D93B68E2
:1073D800002B16D03B68FB6500233B660EE000BF20
:1073E8000C21002004210020D34D6210FB6D5A1C93
:1073F800FA6500221A703B6E01333B663B6E072B21
:10740800F4D9002387E0BB68002B07D0BA6807F1DE
:10741800380392E8030083E8030010E007F138031B
:107428007B650023BB6507E07B6D5A1C7A650022EB
:107438001A70BB6D0133BB65BB6D072BF4D97B6834
:10744800002B07D07A6807F1300392E8030083E83D
:10745800030010E007F13003FB6400233B6507E0FD
:10746800FB6C5A1CFA6400221A703B6D01333B65B1
:107478003B6D072BF4D93B68002B07D03A6807F11E
:10748800280392E8030083E8030010E007F12803CB
:107498007B640023BB6407E07B6C5A1C7A6400227F
:1074A8001A70BB6C0133BB64BB6C072BF4D907F1B2
:1074B800380107F1300207F12803F868FFF736FDB5
:1074C800C7F8AC0004E0164B1B681846FDF7DAFF56
:1074D800BB68002B07D0BB681A4607F1380393E84E
:1074E800030082E803007B68002B07D07B681A46FC
:1074F80007F1300393E8030082E803003B68002BA0
:1075080007D03B681A4607F1280393E8030082E88E
:107518000300D7F8AC301846B037BD4680BD00BF71
:107528000C21002080B586B000AF78600B46FB7058
:1075380013463B807B68002B2CD07B689B697B6162
:107548007B69002B1EDA5E4B1B68184603F0B0FC03
:107558007B689B69002B0DDAFB78002B04D17B68D4
:107568009B695A1E7B689A61554B1B681846FDF744
:1075780089FFA1E07B689B697B61514B1B681846BA
:10758800FDF780FF7869FEF777FFF860FB68002B4E
:1075980001D191E090E04B4B1B68184603F088FC42
:1075A800FB78032B26D801A252F823F0C5750008F2
:1075B800D9750008ED750008F5750008FB685B894A
:1075C8009BB29BB201339BB29AB2FB685A8112E01C
:1075D800FB685B899BB29BB2013B9BB29AB2FB688A
:1075E8005A8108E0FB6801229A8104E0FB680022C6
:1075F8009A8100E000BF334B1B681846FDF742FF35
:10760800304B1B68184603F053FC2F4B1B683B613B
:1076180037E03B691B69002B30D13B695B68002B65
:1076280014D03B695B687A69520953F822207B6958
:1076380003F01F0342FA03F303F00103002B05D004
:10764800FB685B891BB2002B00DD1DE03B699B6872
:10765800002B13D03B699B687A69520953F82220A2
:107668007B6903F01F0342FA03F303F00103002BC5
:1076780004D0FB689B89002B00D005E03B691B68A0
:107688003B613B69002BC4D13B69002B0DD03B69A2
:1076980001221A613B695B691846FDF7F3FE094B45
:1076A8001B681846FDF7EEFE05E0064B1B681846FA
:1076B800FDF7E8FE00E0A3E71837BD4680BD00BF30
:1076C800082100200C2100200421002080B582B070
:1076D80000AF786039607868FFF7AEF8034618465F
:1076E8000837BD4680BD00BF80B58AB000AFF860DE
:1076F800B9607A60FB70F868FEF7BEFE78627B6A54
:10770800002B02D14FF0FF3330E007F11403184685
:107718000021102222F012F810233B7502237B75FA
:107728007B6A186807F1100107F114039A1CFB78AB
:10773800FDF756FFFB8A184602F02AF80346FB823B
:107748003B69BB617B681B68102B02D97B681022E0
:107758001A607B681B6807F11402B86811461A465C
:107768001EF0F0FD7B6A00221A61002318462837B4
:10777800BD4680BD80B584B000AFF860B9607A605E
:10778800F868B9687A680023FFF7AEFF0346184621
:107798001037BD4680BD00BF80B584B000AFF8602B
:1077A800B9607A60F868B9687A680123FFF79CFFC6
:1077B800034618461037BD4680BD00BF80B58EB061
:1077C80000AFF860B9607A603B60002387F8373013
:1077D800F868FEF751FE38633B6B002B02D14FF07F
:1077E800FF33B9E03B68002B02D03B6C002B05D17E
:1077F8003B6B0E221A614FF0FF33ADE0BB68062BDE
:1078080056D040F6FF72934202D0002B3ED068E07B
:107818007B68202B13D0202B04DC022B0FD0082BE5
:107828000DD02EE041F2060293422ADB41F2080213
:10783800934204DD41F20A02934209D021E03B6CF5
:107848001B68032B03D8162387F837301DE01CE08C
:107858003B6C1B68032B02D8162387F837303B6B29
:107868001B681B78202B07D13B6B1B685B681B7C54
:1078780003F00203002B03D06A2387F8373004E0B3
:1078880003E06D2387F837302EE02DE07B68013B5D
:10789800012B08D83B6C1B68032B03D8162387F8E9
:1078A800373004E003E06D2387F837301CE01BE035
:1078B8003B6C1B68032B03D8162387F8373013E07B
:1078C8003B6B1B681B78102B01D0002344E07B68BE
:1078D800013B012B03D96D2387F8373004E000BF43
:1078E80002E06D2387F8373097F93730002B06D040
:1078F80097F937203B6B1A614FF0FF332CE03B6B55
:107908007B61BB68FB617B683B623B687B623B6C6D
:10791800BB6297F8373087F82C3007F1140310480A
:107928001946012200F0EEFB3B6B1B68DB6818462A
:107938000021FDF781FD97F82C3087F8373097F94B
:1079480037203B6B1A6197F93730002B02D04FF084
:10795800FF3300E0002300BF18463837BD4680BD1E
:107968006D79000880B588B000AF78607B68FB61EE
:10797800FB691B68BB61FB695B687B61FB699B6892
:107988003B61FB69DB68FB60FB691B69BB603B69AA
:10799800062B00F0998040F6FF72934202D0002B2C
:1079A8007BD0B1E0FB6841F2060293425FD041F21E
:1079B8000602934206DC082B11D0202B0FD0022B95
:1079C8000DD0A1E041F20802934212D041F2080220
:1079D80093422DDB41F20A0293424ED094E0BB69F8
:1079E8001B685B681B891A46FB681A40BB681A60EB
:1079F80052E0BB691B681B7803F0F003202B0CD006
:107A0800402B02D0102B04D00BE0BB6803221A6075
:107A18000DE0BB6801221A6009E0BB6802221A6007
:107A280005E0BB691B681B781A46BB681A6033E01F
:107A3800BB691B69002B12D1BB691B681B7A5BB23F
:107A48005B420E2B08D8BB691B681B7A5BB25B4292
:107A5800324A52F8233000E00523BA691361BB6942
:107A68001A69BB681A60BB6900221A6114E0BB6915
:107A78001B68DA69BB681A600EE0BB691B685B6843
:107A88001B7C03F00103002B14BF01230023DBB28E
:107A98001A46BB681A6000BF36E0FB68012B0AD0A3
:107AA800022B00D030E0BB691B685B68DB7A1A46A2
:107AB800BB681A6007E0BB691B685B689B7A1A465B
:107AC800BB681A6000BF1FE0FB68012B02D0022BC5
:107AD80010D018E0BB691B685B6893F8223003F08C
:107AE8004003002B14BF01230023DBB21A46BB68F6
:107AF8001A6008E0BB691B685B68D3F894301A46C3
:107B0800BB681A6000BF00BFBB691B68DB6818460A
:107B1800FDF7B8FC2037BD4680BD00BF84260308AA
:107B280080B58EB000AFF860B9607A603B60F868E5
:107B3800FEF7A2FC386300237B633B6B002B02D16A
:107B48004FF0FF33A0E03B68002B05D13B6B0E22C2
:107B58001A614FF0FF3397E0BB68062B47D040F619
:107B6800FF72934202D0002B32D056E07B68202B64
:107B78000DD0202B02DC082B09D025E041F20602AB
:107B8800934204D041F20A02934207D01CE03B6CB6
:107B9800032B02D816237B6319E018E03B6C032BF8
:107BA80001D816237B633B6B1B681B78202B07D1FE
:107BB8003B6B1B685B681B7C03F00203002B02D045
:107BC8006A237B6303E002E06D237B6327E026E002
:107BD8007B68013B012B06D83B6C032B02D816238C
:107BE8007B6303E002E06D237B6318E017E03B6CE6
:107BF800032B02D816237B6311E03B6B1B681B78B1
:107C0800102B01D000233FE07B68013B012B02D9F8
:107C18006D237B6303E000BF01E06D237B637B6B17
:107C2800002B05D03B6B7A6B1A614FF0FF332BE0CA
:107C38003B6B7B61BB68FB617B683B623B687B623B
:107C480007F14003BB627B6BDBB287F82C3007F18E
:107C580014030F481946012200F054FA3B6B1B68C5
:107C6800DB6818460021FDF7E7FB97F82C305BB27C
:107C78007B633B6B7A6B1A617B6B002B02D04FF0F6
:107C8800FF3300E0002300BF18463837BD4680BDEB
:107C98009D7C000880B588B000AF78607B68FB6188
:107CA800FB691B68BB61FB695B687B61FB699B685F
:107CB8003B61FB69DB68FB60FB691B69BB603B6977
:107CC800062B75D040F6FF72934202D0002B58D095
:107CD8009DE0FB68202B0DD0202B02DC082B09D05F
:107CE80095E041F20602934228D041F20A029342FB
:107CF8002AD08CE0BB681B68002B0ED0BB691B68C0
:107D08005B68BA6912685268128991B2FA6892B2CD
:107D18000A4392B292B21A8132E0BB691B685B686F
:107D2800BA6912685268128991B2FA6892B2D2435B
:107D380092B20A4092B292B21A8121E0BB691B68E2
:107D4800BA681268DA611BE0BB681B68002B0BD0AD
:107D5800BB691B685B68BA6912685268127C42F09A
:107D68000102D2B21A740AE0BB691B685B68BA697F
:107D780012685268127C22F00102D2B21A7400BF53
:107D880045E0FB68012B0AD0022B00D03FE0BB691D
:107D98001B685B68BA681268D2B2DA7207E0BB691E
:107DA8001B685B68BA681268D2B29A7200BF2EE08C
:107DB800FB68012B02D0022B20D027E0BB681B6890
:107DC800002B0DD0BB691B685B68BA6912685268E2
:107DD80092F8222042F04002D2B283F8222015E025
:107DE800BB691B685B68BA691268526892F82220FE
:107DF80022F04002D2B283F8222007E0BB691B6858
:107E08005B68BA681268C3F8942000BF00BFBB69FA
:107E18001B68DB681846FDF735FB2037BD4680BD7B
:107E280080B588B000AFF860B9607A60F868FEF78E
:107E380023FBB8610023FB82BB69002B02D14FF002
:107E4800FF3356E0BB682D4A934232D02C4A934206
:107E58004AD17B68002B05D1BB6916221A614FF005
:107E6800FF3346E0BB691B681B8CFB83B7F91E30E8
:107E7800002B01DA0023FB83FA8B7B681A80BB692D
:107E88005B68002B10D0BB695B681B681B89FB8291
:107E9800BB691B89FA8AD31AFB827B681A88FB8A1A
:107EA80013449AB27B681A80BB6900221A610023C6
:107EB8001FE07B68002B0BD07B681B68002B07D06A
:107EC800BB69DB8943F400639AB2BB69DA8106E0D7
:107ED800BB69DB8923F400639AB2BB69DA81BB69A9
:107EE80000221A61002304E0BB6958221A614FF08E
:107EF800FF3318462037BD4680BD00BF7E6604802C
:107F08007F66044008B503F0ABFB084B1B6813B948
:107F1800074B1B6833B1BDE80840FA200549002229
:107F280002F0EFBF044A136008BD00BF6C6F002069
:107F3800806F00200D7F00081021002013B500225B
:107F48004FF47A70274902F0DCFF41F28830264965
:107F5800002202F0D6FF4EF660202449002202F0EB
:107F6800D0FF234C4FF4FA702249002202F0C9FFD7
:107F78004FF47A702049002202F0C3FF63680BB106
:107F8800A0689847E06801A902F066FF019B1A788B
:107F9800042AF7D8DFE802F0030713171D009868D2
:107FA80003680430EDE7D968986891F831209306A2
:107FB80002D505F039FC10E001F036FD0DE09A68B5
:107FC800D868904709E003F1080007C802F099FF54
:107FD80003E0D868196902F0C5FF019802F0E4F9D6
:107FE800D0E700BF75800008598000083D80000870
:107FF80010210020218000080580000808B501F044
:10800800F9F9BDE808404FF47A700249002202F0FD
:1080180078BF00BF0580000808B500F063FFBDE821
:1080280008404FF4FA700249002202F06ABF00BF0C
:108038002180000808B500F0CDFEBDE808404EF6E6
:1080480060200249002202F05CBF00BF3D800008AA
:1080580008B505F019FABDE8084041F28830024930
:10806800002202F04EBF00BF5980000808B501F099
:10807800D1FEBDE808404FF47A700249002202F0B0
:1080880040BF00BF7580000802F06CBC084B1A683E
:1080980062B9084A126812B9074A126832B1012255
:1080A8001A60FA200549002202F02BBF704700BF72
:1080B800102100206C6F0020806F00200D7F0008C9
:1080C800F8B50E4D0746EB680E4693B10C4B588A2F
:1080D80002F07CFA044670B1012303708760C66021
:1080E8002146E868FDF738F930B1204602F05CF91E
:1080F80001E0F72000E0FF2040B2F8BD1021002089
:10810800C82603082DE9F041124D8046EB680F465A
:108118001646C3B1104B188A02F058FA0446A0B1AB
:1081280002230370C0F80880C7602146E8681EB1C2
:10813800FDF7FEF8002009E0FDF70EF930B1204602
:1081480002F032F901E0F72000E0FF2040B2BDE87C
:10815800F08100BF10210020C8260308F8B50D4C97
:108168000746E3680E4615467BB10B4B188A02F0AA
:108178002DFA014658B1032202708760C660056176
:10818800E068FDF7D5F8002002E0F72000E0FF20C6
:1081980040B2F8BD10210020C826030870B50C4C69
:1081A8000646E3680D4673B10A4B188A02F00EFAC8
:1081B800014650B104220270C6600561E068FDF70F
:1081C800B7F8002002E0F72000E0FF2040B270BDC1
:1081D80010210020C826030830B50B4B0546D86887
:1081E80087B068B1002401A98DF804400395FDF714
:1081F8009FF86B682146D868FDF71EF9204600E015
:10820800F72040B207B030BD1021002073B50D46ED
:1082180006460A4C01F08AF905206660A560FDF75C
:1082280077F80123E0600093054900224FF420739A
:108238000448FDF765F902B070BD00BF10210020A9
:10824800457F000840830308014600220148FFF7E4
:1082580059BF00BF91800008014600220148FFF77E
:1082680051BF00BFB1A30008837C8B421EBF00230F
:108278008174C3747047838B30B584695D1C234453
:10828800858383F8F010838B81695C1C0B4484839D
:1082980083F8F02030BD10B5838B82695C1C1344D1
:1082A800848383F8F01010BD838B826910B55C1C41
:1082B80013440A0A848383F8F020838B82695C1C48
:1082C8001344848383F8F01010BD838B826910B542
:1082D8005C1C13440A0E848383F8F020838B826924
:1082E8005C1C1344C1F30742848383F8F020838B1A
:1082F80082695C1C1344C1F30722848383F8F0204D
:10830800838B82695C1C1344848383F8F01010BD4E
:10831800C268F0B50546002A3BD0078A0FB938462F
:10832800F0BD00231C46BB4202D3B4B92046F0BDC1
:10833800D65CD018FF2EF8D0342E05D1981C80B208
:1083480003339BB2145CEEE78E4225D0581C80B2F2
:10835800105C023303449BB2E5E7012CAB6802D101
:108368006C33802405E0022C03F12C030CBF40245D
:10837800C02400229D5C9818FF2D0CD08D420BD094
:10838800501C80B2185C0230024492B2A242F1D36F
:1083980001E01046F0BD0020F0BDF8B50646002803
:1083A80075D0046A002C74D000204FF49A710246EC
:1083B80002F0EBFA606100286DD0E27C374B12B90D
:1083C8001A6801321A601B68426823600123A2619F
:1083D8001370A26900255370A36906229A70A369D5
:1083E800DD702068A76901F0D9F9A36978601D726A
:1083F8005D729D72DD721D735D739D73DD73A27C6A
:108408000A2A02D0043A012A01D87268DA600022E6
:108418001A745A749A74DA741A755A759A75DA75E0
:108428001A765A769A76DA7696F82A0091B28842BF
:10843800A36984BFB11891F82B10134402F101020B
:1084480098BF0021102A1977EED10022A369991844
:1084580001320023402A81F82C30F7D1A269002587
:108468001A440133802B82F86C50F7D10C48A66966
:1084780001F094F92B46C6F8EC00A583A2691A44CA
:1084880082F8F0300133442BF8D1002004E0F620C4
:1084980002E0F72000E0FF2040B2F8BD1C000020F9
:1084A8006353826310B540B1046A34B1606908B19E
:1084B80002F058FA00236361A36110BD38B5054680
:1084C800046A08212046FFF7CFFE284604F1280158
:1084D800002205F0DBF8E37C0133E3740123E38336
:1084E80038BD37B50546002854D0046A002C51D051
:1084F800A36C591C0BD03C221E33B3FBF2F34FF68E
:10850800FF72934228BF134603B901232384E36C07
:108518005A1C0BD03C221E33B3FBF2F34FF6FF720A
:10852800934228BF134603B901236384E06A00908D
:1085380078B901F0C1F9000E030602D44FF07F406C
:1085480004E0BF2894BF14486FF0FF0001F026F93B
:108558000090236B01934BB9A36A009A0120134042
:10856800019301F01BF9019B18430190284604F17F
:10857800280102F043F92846694602F09FF901A94B
:10858800284602F097F9284602F0A2F920460A2167
:10859800FFF76AFE03B030BD0000FFFF10B50446C8
:1085A800806818B101F000FF0023A360E06820B1E3
:1085B80001F0FAFE0023E360238210BD90B1838BA3
:1085C8008269591C81831344FF2283F8F020838B2E
:1085D800432B05D88269591C818313440022F4E790
:1085E8009A07F7D17047F7B50646046A0421204672
:1085F800FFF73AFE3046FFF7D0FE0546002838D18F
:10860800012220463521FFF736FE20460321FFF7D9
:1086180042FE204639210222FFF72DFE2046318DE9
:10862800FFF742FE776A9FB92046FFF7C7FFA18B85
:108638006069F03189B202F037FA009660686169C2
:10864800184A432304F08AFD3046FFF72BFF10E059
:10865800384621F0F7FB0C21C2B22046FFF70BFE8B
:10866800013F17F8011F0029DED02046FFF713FE4F
:10867800F7E7E37C28460133DBB2092BE3748FBFAD
:1086880042F21073C3EB431203EB8203DB0098BF83
:108698009BB24FF4FA7203F2F31393FBF2F3E38302
:1086A80003B0F0BDC026030873B506462E4B046A16
:1086B8001B682046A3620621FFF7D6FD3046FFF768
:1086C8006CFE0546002839D1012220463521FFF7E6
:1086D800D2FD20460121FFF7DEFD02222046392186
:1086E800FFF7C9FD2046318DFFF7DEFD0422204645
:1086F8003721FFF7C0FD20460121FFF7CCFD2046BA
:108708000321FFF7C8FD20461C21FFF7C4FD062101
:108718002046FFF7C0FD2046FFF750FFA18B606998
:10872800F03189B202F0C0F90096606861690F4AB9
:10873800432304F013FD3046FFF7B4FEE27C2846DD
:108748000132D2B2052A8FBF4EF660234FF47A73F6
:1087580093409BB2E27403F2F3134FF4FA7293FB63
:10876800F2F3E38302B070BDC4260308C0260308F1
:10877800F7B50646046A01212046FFF775FD304625
:10878800FFF70BFE0546002865D10122204635215A
:10879800FFF771FD20460321FFF77DFD02222046E9
:1087A8003921FFF768FD2046318DFFF77DFD042252
:1087B80032212046FFF75FFDA06A01F07DF80146EF
:1087C8002046FFF782FD042236212046FFF753FD9D
:1087D800606A01F071F801462046FFF776FD042231
:1087E80020463721FFF747FD20460121FFF753FDBB
:1087F80020460321FFF74FFD20461C21FFF74BFDC4
:1088080020460621FFF747FD776A9FB92046FFF704
:10881800D5FEA18B6069F03189B202F045F9009666
:1088280060686169174A432304F098FC3046FFF7F3
:1088380039FE10E0384621F005FB0C21C2B2204673
:10884800FFF719FD013F17F8011F0029DED0204668
:10885800FFF721FDF7E7E27C28460132D2B2052A6C
:108868008FBF4EF660234FF47A7393409BB2E27445
:1088780003F2F3134FF4FA7293FBF2F3E38303B0BA
:10888800F0BD00BFC026030873B50646046A03217D
:108898002046FFF7E9FC3046FFF77FFD054688BB19
:1088A800012220463521FFF7E6FC20460321FFF789
:1088B800F2FC022220463921FFF7DDFC20464FF466
:1088C8001071FFF7F1FC042232212046FFF7D3FC98
:1088D800A06A00F0F1FF01462046FFF7F6FC2046AB
:1088E800FFF76CFEA18B6069F03189B202F0DCF809
:1088F800009660686169104A432304F02FFC3046F3
:10890800FFF7D0FDE37C28460133DBB2092BE37483
:108918008FBF42F21073C3EB431203EB8203DB00F9
:1089280098BF9BB24FF4FA7203F2F31393FBF2F37E
:10893800E38302B070BD00BFC02603082DE9F047ED
:1089480017467B8906462B2B056A52684CD9137843
:10895800022B49D196F82A3000F12A012A3302F174
:108968001B003344994206D011F801EF10F8014F6B
:10897800A645F7D038E0506800F09EFF2B68984273
:1089880032D12846FFF70AFE3889F02808D9F0388E
:1089980080B2288201F01AFEE86008B9288223E034
:1089A800F02001F013FE0446A86030B9E868D8B199
:1089B80001F0FAFCEC602C8216E021463846F022E1
:1089C800002302F01AF9E968B1B138462A8AF0237F
:1089D80002F013F910E04046704900F0B9FC00239A
:1089E800EB833046FFF76AFD2846FFF7D7FD384688
:1089F800BDE8F04701F0B6BF28463521FFF788FCEF
:108A08000028F1D08378052B40F08480AB7C012BC3
:108A180076D1346A0023E3622363636320463321FB
:108A2800FFF776FC18B102301EF0FEF860642046AD
:108A38003A21FFF76DFC20B102301EF0F5F8A06472
:108A480002E0636C5B08A36420463B21FFF760FCEF
:108A580020B102301EF0E8F8E06401E0636CE364E2
:108A6800A268204612F1100318BF13690121A362FE
:108A7800FFF74EFC28B102301EF0D6F800F08EFE4B
:108A8800E06220460321FFF743FC28B102301EF0C4
:108A9800CBF800F083FE206320461C21FFF738FC4A
:108AA80028B102301EF0C0F800F078FE606320465E
:108AB8000621FFF72DFC8246002890D043789B08BA
:108AC800022BA36384BF0223A36300235FFA83F806
:108AD80003F10109A36B9845BFF47DAF0AEB880049
:108AE80002301EF0A1F800F059FE08F10E0104EB67
:108AF800810141F8040F404600F02AFC4B46E5E7A7
:108B0800033B022B3FF670AF0023EB833046FFF7A1
:108B1800E8FC69E7062B20D1AB7CDA1E022A02D9D1
:108B2800012B7FF461AF0023EB833046346A01F0F8
:108B3800DEFE3046194901F061FE3046174901F062
:108B4800B9FE3046154901F0B9FE20460C21FFF761
:108B58008BFB3046FFF7A8FD46E7022B7FF444AFB6
:108B6800AB7C062B7FF440AF346A0023EB832046AE
:108B78003621FFF7CDFB00283FF436AF02301EF058
:108B880053F800F00BFEA268606212F1100318BFE0
:108B980013693046A362FFF7EBFD25E7C4260308F7
:108BA80073B50546502001F011FD0446002844D055
:108BB8000021502220F0C2FD04F0A2FB60600028D2
:108BC80035D02E6A28462C62FFF7E7FB48BB012206
:108BD80020463521FFF74FFB20460821FFF75BFBB6
:108BE800022220463921FFF746FB298D2046FFF750
:108BF8005BFB2046FFF7E2FCA18B6069F03189B28C
:108C080001F052FF0E494422606804F07DFA009595
:108C1800606861690B4A432304F0A0FA2846FFF70D
:108C280041FC606804F057FB002363602E62204615
:108C380002B0BDE8704001F0B7BB02B070BD00BF24
:108C4800C4260308C026030838B5056A0446C5B11A
:108C5800AB7C033B0A2B0FD8DFE803F00606060EB1
:108C68000E0E0E060E0E130001F041FE0023EB74EB
:108C78002046BDE8384007E60023EB74BDE83840DD
:108C880012E538BD37B5054600283ED0046A002CE9
:108C98003BD0A37C082B38D10A68A36A9A4234D106
:108CA80020460C21FFF7E0FA2846FFF776FB38BB91
:108CB800012220463521FFF7DEFA20460421FFF77E
:108CC800EAFA042232212046FFF7D5FAA06A00F01A
:108CD800F3FD01462046FFF7F8FA2046FFF76EFC41
:108CE800A18B6069F03189B201F0DEFE0095606801
:108CF8006169074A432304F031FA2846FFF7D2FB9B
:108D0800E37C0133E3741423E38303B030BD00BF75
:108D1800C0260308F7B50646046A05212046FFF772
:108D2800A3FA3046FFF739FB0546002839D101225E
:108D380020463521FFF79FFA20460321FFF7ABFABB
:108D4800204639210222FFF796FA2046318DFFF797
:108D5800ABFA776AA7B92046FFF730FCA18B6069A8
:108D6800F03189B201F0A0FE00966068616904F1F3
:108D78002402432304F0F2F93046FFF793FB10E096
:108D8800384621F05FF80C21C2B22046FFF773FA8B
:108D9800013F17F8011F0029DDD02046FFF77BFAB5
:108DA800F7E7E37C28460133DBB2092BE3748FBF76
:108DB80044F62063C3EB431203EB82031B0198BF05
:108DC8009BB24FF4FA7203F2F31393FBF2F3E383CB
:108DD80003B0F0BD134B10B51C6814B3236AF3B18C
:108DE8005A8C511E012A59840AD19B7C03F0FB023C
:108DF800012A01D00A2B12D12046FFF7F4FB0EE01E
:108E08001A8C511E012A198409D19B7C03F0FB029C
:108E1800012A01D00A2B02D12046FFF77BFF2468E4
:108E2800DBE710BD646F002073B50546046A0D21A9
:108E38002046FFF719FA00236362E362A3626363C3
:108E48002363E364A3646364A3632846FFF7A5FA76
:108E58000646E0B9012220463521FFF70CFA072122
:108E68002046FFF718FA2046FFF7A8FBA18B606998
:108E7800F03189B201F018FE00956068616904F16B
:108E88002402432304F06AF92846FFF70BFBE37C2E
:108E980028460133DBB2092BE3748FBF42F210730B
:108EA800C3EB431203EB8203DB0098BF9BB24FF482
:108EB800FA7203F2F31393FBF2F3E38301F017FD65
:108EC8002846074901F09AFC2846054901F0F2FCBA
:108ED8002846034901F0F2FC304602B070BD00BFDD
:108EE800C4260308254B10B51C68002C45D0236AFE
:108EF800002B40D0DA8B012A02D9013ADA833AE012
:108F080039D10022DA839A7C0C2A27D0062A25D068
:108F1800012A06D1DB7C2046052B1DD8FFF728FC4B
:108F280029E0082A09D1DB7C2046012B02D8FFF76B
:108F3800C5FA20E0FFF7D5FA1DE0052A03D120463F
:108F4800FFF7E8FE17E0042A0AD1DB7C2046082B4D
:108F580002D8FFF748FB0EE0FFF766FF204608E05F
:108F6800032A08D1DB7C2046012B02D8FFF78CFCB2
:108F780001E0FFF799FB2468B7E710BD646F002094
:108F880038B590F83130056A23F00803044680F8B4
:108F9800313055B1686818B104F09DF900236B6051
:108FA800284601F001FA0023236238BD70B5044653
:108FB800002843D090F83130056A23F0080380F880
:108FC8003130038DB3F5107F2FD335B9502001F020
:108FD800FDFA054648B3206203E0686808B104F06A
:108FE8007AF900215022284620F0A8FB04F088F9DD
:108FF8000646686020B9284601F0D6F9266214E0D2
:109008001049442204F080F80E494322686804F0AD
:109018002EF968680C49224604F05AF92046FFF7F1
:1090280043FB20B12046FFF7ABFFFF2007E094F891
:10903800313043F0080384F8313000E0F62040B2C4
:1090480070BD00BFC4260308458900082DE9F0411A
:10905800064600200F4690464FF48871024601F0FC
:1090680094FC054600284BD0446800210C22204679
:1090780020F064FB404600F08BFB20800120A070AC
:1090880000F086FB04F10C03A080791E5F1C3C46AF
:10909800481C0178E21B2E29D2B205D11A70037838
:1090A80001463BB12346F1E70029F7D004F8011B3C
:1090B8000130EEE72370012000F06AFB074601202B
:1090C80000F066FBA4F80170A4F803006968053491
:1090D800611A0D4C284604EB860689B201F0E4FCBF
:1090E8003146A068352204F0C2F8A0682946324605
:1090F800352304F0A3F80446284601F033FC00E0C9
:10910800FF2460B2BDE8F081202100204FF48C716B
:10911800F8B54143264E04467218177B02F10C033A
:10912800022F35460BD0032F3AD0012F3FD1022012
:109138001073002058709F70D87011462BE09A78F1
:10914800013AD2B29A7092BBDA7858780132D2B228
:10915800042ADA701DD130B9726822B101225A701E
:109168009A70D870F8BD4FF48C736343EA18D2F83C
:109178001C612EB10F4800211844D2F82021B047B5
:109188004FF48C7303FB045400232373C4F81C317D
:10919800F8BD9A7031442246BDE8F840183155E7C9
:1091A8005369013B536113B91373C2F81C31F8BDFD
:1091B80020210020382100202DE9F74F91461289FF
:1091C800A2F11A03B3F5F37F6CD85D4C002348462F
:1091D80004F50F7101F011FDB9F80830834261D12F
:1091E800B4F83C0200F0D4FAC7B2012F5AD84FF4B1
:1091F8008C757D4363191A7B03F10C06022A51D141
:1092080003221A7394F83F3203F00F037371B4F812
:10921800400200F0BDFA8046B4F8420200F0B8FA05
:1092280094F93E32002B0EDB4FF48C737B43E2182B
:10923800D2F81C5102F58E7665B3424800211844D5
:109248007268A84726E07379002BEDD15FFA88F899
:10925800B8F1010FE8D104F10C010D440C352A4690
:1092680004F5127300915E1C1B7803F0C001C0293D
:109278001ED0D11833468A4207D092F800E01E78F3
:10928800B645D1D101330132F5E719780132002909
:10929800E9D10DE04FF48C7303FB074400232373DB
:1092A800C4F81C31484603B0BDE8F04F01F05ABB82
:1092B800C6B225481DF0C3FC0430002EB4D01DF002
:1092C800BEFC4388D0F804B0B0F808A080460088F7
:1092D800019300F060FA0128019B28D1184600F09C
:1092E8005AFA012823D1504600F055FA04281ED115
:1092F800584600F0E1FA4FF48C7303FB0742134918
:109308005F438842506188BF5161009A07F58473B2
:10931800D8F80A001A4450602744D7F81C31111DA8
:10932800002BBFD02846D7F820219847BAE75046E7
:1093380000F02EFA013E0A304044F6B2BDE700BF05
:10934800202100203821002068230020803A0900CD
:10935800012807D8044B9A6822B119B10A680AB1E2
:1093680043F82020704700BF2021002037B50D4862
:1093780000F096FA0C4D0190AC6884B903F0C0FF78
:10938800A86060B10949224603F0BEFEA8680849F2
:10939800224603F09DFF204601A9FFF7D9FF03B03D
:1093A80030BD00BF4783030820210020C4260308DE
:1093B800C1910008012895BF0C4B0D4B53F82000B4
:1093C800186882B001909DF80430002063F307000C
:1093D8009DF8053063F30F209DF8063063F31740BE
:1093E8009DF8073063F31F6002B07047202100200A
:1093F800C426030808B5054B9B6833B10020FFF766
:1094080085FEBDE80840012080E608BD2021002037
:109418002DE9F8431E46424B17469A680546894689
:109428009846002A76D0002974D0002872D0037894
:10943800002B6FD020F006FDFF286BD8284600F0DF
:109448002FFA431C0446C9F8000001D0002064E04C
:1094580098F80C30032B05D1284608F118011CF0A8
:10946800E7FF48B198F82431032B0BD128462D4942
:109478001CF0DEFF30B901204FF48C7303FB008031
:10948800D0F81841C9F800400134DFD198F80C40F1
:1094980098F83C246CB1032C06D1214B1B7CD31AC1
:1094A800002B01DDDBB200E0002398F8241131B96C
:1094B80001241D4A4FF48C7000FB042015E0032999
:1094C80008D1174991F82841141B9C42D4BF0024A5
:1094D800012400E000244FF48C70604308EB000383
:1094E8001B7B032B18D1104B18440123037098F8E9
:1094F8003C34C0F810715A1C0371C0F81461294635
:109508000C3088F83C2420F03FFC2046FFF7FEFD95
:10951800F22002E0F72000E0FF2040B2BDE8F88327
:1095280020210020502200202C21002008B5FBF724
:10953800B5FF00F0FBFEFCF78BFFBDE80840FFF726
:1095480015BF2DE9F7430646894690460120242198
:10955800002201F01AFA054668B344683768002308
:1095680084F8009084F8018023716371A371E3711A
:1095780041683368083103F11C0253F8040B934225
:1095880041F8040BF9D100266989A670E6702046D7
:1095980000F0FDF9012360803146019300962846CA
:1095A80007F10C02FF2300F083FB284603B0BDE857
:1095B800F04301F0D7B903B0BDE8F0832DE9F04FCF
:1095C800456887B004462888884600F0E4F8C0F368
:1095D80003208600C6F100092046494601F096F9A5
:1095E800002840F08F802389032B40F28B8063682A
:1095F8001B78082B40F08680AA464FF070405AF836
:10960800107F00F059F905904FF0604000F054F9D0
:1096180041468346504600F067FB059B002871D100
:109628001F405F456ED02389072B6BD9204600F079
:10963800B4F9002866D120462221B6B201F066F9B5
:10964800F0B12046314601F061F90246002859D1AF
:109658000220218901F099F90746002852D02146B5
:1096680001F081FA00284DD1384649467D6801F05D
:109678004DF9002846D1204601F074F93C4605E032
:1096880020466FF0210101F041F9D8BBEB6867680B
:109698002A692B610023EA604FF2FF703B70B7F82C
:1096A800029000F075F881454FF4006003D300F094
:1096B8006FF8013001E000F06BF87B88184478807F
:1096C800288900F068F860F0FF0080B200F060F8C8
:1096D80000232881AB72EB721421284600F057F959
:1096E80031466881204601F011F9024650B901233C
:1096F80000900193CDF80880204605F10C01FF2366
:1097080000F066FA204607B0BDE8F04F01F02AB92C
:109718000A460430032114E70A4604300B2110E7F7
:1097280073B5019019480DF103040DF1070614F8FB
:10973800011F00230A22B1FBF2F502FB15110DF1FE
:10974800080E5A1C3031734403F8081CD2B215F0C5
:10975800FF011346EED121700146013AD2B2FF2A29
:1097680006D002AD154415F8085C01F8015BF4E772
:1097780003442E22B44203F101001A70D7D100230A
:1097880000F8013C014802B070BD00BF6025002010
:1097980040BA80B2704740BA80B2704700BA70478A
:1097A800F0B585B00C466A466F460378A3F13001E0
:1097B80009296FD8302B0BD1437803F0DF015829E2
:1097C8000DBF837801300826023008BF102600E05C
:1097D8000A26451C0020A3F13001092905F1FF3CA8
:1097E80003D806FB0030303815E0102E16D123F0D0
:1097F80020014139C9B2A3F1610E05295FFA8EFE35
:109808000CD8BEF11A0F03F10A0334BF61214121BC
:109818005B1A43EA00102B780135DCE72E2B09D1BF
:1098280003AB9A4236D042F8040B9CF801300CF195
:109838000100BBE713F0DF0F02D0093B042B29D846
:10984800D21B92100132042A1FD8DFE802F0261E2C
:10985800030A1300B0F1807F1CD2009B40EA03602A
:1098680013E0B0F5803F15D2009B019A1B0643EA2E
:10987800024309E0FF280DD8009B019A1B0643EA22
:109888000243029A43EA022318432CB1FFF786FFEA
:10989800206001E0002200E00122104605B0F0BD82
:1098A80007B501A9FFF77CFF08B1019801E04FF067
:1098B800FF3003B05DF804FBFFF770BFF0B54E084A
:1098C80000EB4604431C033400220233A34207D0B2
:1098D80013F8037C13F8025C45EA07252A44F4E7E9
:1098E800CB0748BF10F81630BDE8F04048BF02EB80
:1098F800032293B203EB1240030C1CBF80B2C018C2
:1099080080B2FFF745BF2DE9F84300250646884693
:1099180091461F462C46AEB170687189FFF7CEFF9D
:109928007389204484B2DB0704EB104441BF23024F
:10993800C5F101059BB2C4F3072444BFEDB21C4333
:109948003668E8E725B1210289B2C4F307240C433D
:10995800D8F80000D9F8003082B202EB10409AB271
:10996800104400EB134004443846FFF711FF044449
:10997800BDF82000FFF70CFF204484B204EB104030
:1099880083B203EB1040C04380B2BDE8F88308B54A
:10999800FFF794FFC04380B208BD70B500250646A6
:1099A8002C46AEB170687189FFF788FF738920442F
:1099B80084B2DB0704EB104441BF2302C5F1010563
:1099C8009BB2C4F3072444BFEDB21C433668E8E7F2
:1099D80025B123029BB2C4F307241C43E04380B2A1
:1099E80070BD000038B505460D4B1C685CB12046BB
:1099F80000F086FF28B12A6863685340A2681342C2
:109A08000CD02468F2E7074C206808B9002038BD5C
:109A180000F076FF0028F9D0206838BD204638BD10
:109A2800646F0020686F00202DE9F84344680546FC
:109A380020880F46FFF7AFFEC0F30F30042803D08D
:109A4800284600F08FFFBAE02088FFF7A4FEC0F395
:109A580003204FEA80086088FFF79DFE6B89064661
:109A68004345EDD32B898342EAD320464146FFF78D
:109A78008EFF0028E4D13146284601F015F83E460D
:109A88004FF00109304600F03BFF28B9B9F1000F4B
:109A980012D04C4B1E6810E0331DF7D07368002BB2
:109AA800F4D022699A4270D004F11000314600F0D7
:109AB8001BF90028EAD068E03668BE4208BF36685D
:109AC8004FF00009002EDDD12089FFF764FEC0B2F7
:109AD80011285AD1A044B8F80200FFF75CFE4428C8
:109AE80053D13E46002EABD043F6FF70E688FFF711
:109AF8004FFE304206D0284600F0A0F9054600285F
:109B08005DD04468DFF8C4802F4E28463946C8F82F
:109B18000070346001F0E0F890BB2089FFF73BFE4D
:109B2800C0B206280DD0112806D001280ED128462B
:109B38003946FFF743FD23E02846394603F022FA69
:109B48001EE02846394602F063F919E004F11000D6
:109B5800394600F0C9F880B94FF070402769FFF71F
:109B6800ABFE07404FF06040FFF7A6FE874204D0E7
:109B78006C6028460221FFF7CBFD284600F0F2FE74
:109B88000023C8F80030336019E0E368002BA9D03F
:109B980004F10C00394600F0A7F800287FF450AF14
:109BA8004FF07040D4F80C80FFF786FE00EA0808F2
:109BB8004FF06040FFF780FE804593D140E70020DA
:109BC800BDE8F883646F0020606F00205C6F0020A0
:109BD8002DE9F74F0E9E074689469B469DF8308033
:109BE8009DF834A01546002A44D0142100F08EFEBA
:109BF8000190002855D17C682089FFF7CCFD6BF3D4
:109C08001F20FFF7C5FD2081FFF7C5FD00F47F4049
:109C180040EA0A00FFF7BCFD2A682081226148F467
:109C28008A40FFF7B5FD20803889FFF7B1FDDFF8DE
:109C38007C80019B6080A371E371B8F80000FFF796
:109C4800A7FDB8F80030A0800133A8F80030B9F1BA
:109C5800000F02D0D9F8003013B9331D18BF73684C
:109C6800E3600023A372E37220461421FFF78FFEFE
:109C7800608101E045681035338D53B13A899A42C5
:109C880007D9384631462A4603B0BDE8F04F00F000
:109C980041BA304639462A46736903B0BDE8F04FE9
:109CA80018476FF0010003B0BDE8F08F7025002061
:109CB800F0B5074685B010460E4614461D46FFF718
:109CC80091FE68B19DF82830029000939DF82C30E1
:109CD80038460193314622462B46FFF779FF00E0CC
:109CE800FC2040B205B0F0BD0268531E033314D8FF
:109CF80091F8313003F0020303F0FF0083B14B68A1
:109D08009A420CD088685340034208D1C34303EAFF
:109D18000200C31A5842584170470120704700207A
:109D2800704700002DE9F041456804466B680F460E
:109D38009A88BAB91A6800F11C01426000F1080259
:109D480052F8040B8A4243F8040BF9D12846012142
:109D5800FFF7E2FC284600F0CCFE0646284600F055
:109D680001FE00E0002665685DB16B682846D3F8FF
:109D7800008000F0BEFE0644284600F0F3FD45468C
:109D8800F2E7084D20462B68A342236814BF3B60C6
:109D98002B6000F009FBAB8830469B1BAB80BDE80D
:109DA800F08100BF74250020F8B506460F4600254F
:109DB800002421462046164B1B68F3B1D6F80CE068
:109DC8005A69724509D1D6F810E09A69724504D1EA
:109DD800B3F80CE0B288964509D0013430B193F855
:109DE8001FE0C27F964598BF184600E018461A68DB
:109DF800002A18BF19461346DFE710B1FFF792FF94
:109E08000544BD4201DA012CD2DC2846F8BD00BF6A
:109E18007425002038B5084B0024186858B1C37F52
:109E280005681BB1013BC377044602E02146FFF7F2
:109E380079FF2846F2E738BD742500202DE9F74F51
:109E4800446806462088FFF7A6FCC0F303200528CF
:109E58004CD1E088FFF79FFC01906088FFF79BFCDE
:109E680083462088FFF797FC0746304600F041FEFE
:109E7800A64D8046AB8803440A2B04DC0023D5F8A2
:109E88000090009312E020464146FFF78DFF68B32B
:109E9800AB8843440A2BF1DD28E0E268D9F81410B6
:109EA800914207D0CDF80090D9F80090B9F1000F91
:109EB800F3D10AE02269D9F818109142F2D1B9F821
:109EC8000C10A2889142EDD114E0914BB3F80AA08E
:109ED800504600F07BFB8146002840F0F180204688
:109EE8004146FFF761FF404580F2E380304600F0CD
:109EF80039FD07E1E088FFF74EFCC0F30C0088B994
:109F0800B9F80E00FFF747FCC0F30C0050B1224629
:109F180009F1080104F1140052F804EB824241F8F7
:109F280004EBF9D1AA889044A5F80480E088FFF7EB
:109F380032FC820412D499F81E20019B42F00102DF
:109F480089F81E20C7F30327C3F30C020BEBC20BDF
:109F5800C7EB87370BEB870BA9F81CB074686088D0
:109F6800FFF719FC80462088FFF715FC0746E088B4
:109F7800FFF711FCC0F30C00C400C7F3032704EB80
:109F88000800C7EB8737716800EB87070022B8B273
:109F9800D9F804300A704A708A70CA708C80C880F8
:109FA8000127002B00F0A580D3F804C0BCF804807A
:109FB800444509D20B60AAB1B2F806E0A6452BD8F1
:109FC800404529D816600FE026D0BCF806E0A64523
:109FD80022D81AB1D288424518BF0027DCF80030D1
:109FE8006246DEE7C9F8046099F81E20D30740F1FD
:109FF8008980002F00F08680D9F804205468A28850
:10A00800002A7FD10A6872B15068C9888288914253
:10A0180078D102680146F6E7304600F06AFDAB8861
:10A02800181AA88062E72146B9F81C20266814325D
:10A03800A9F81C2009F11C0009F1080252F8047B58
:10A04800824241F8047BF9D1B9F81C00FFF7A0FB64
:10A0580000226080A271E271A272E272204614218D
:10A06800FFF795FC6081D9F804405EB17768304607
:10A078006FF0130100F04AFC3146204600F046FD1F
:10A088003E68F2E72A6848464A4519BF009BD9F856
:10A098000020D9F800101D4A14BF1A60116000F0A2
:10A0A80083F9204600F025FDAB88181AA8802046C1
:10A0B80029E0504600F08AFA814600283FF416AF9E
:10A0C8000021202248461FF039FB032289F81F206F
:10A0D8002A6809F10801C9F800202246C5F800904D
:10A0E80004F1140052F804EB824241F804EBF9D170
:10A0F80018E7002A3FF476AF1660D288A24218BF4C
:10A10800002771E7002003B0BDE8F08F7425002018
:10A11800C82603082DE9F04F824689B0022006922E
:10A12800B1F828908B460246002100F02EFC064626
:10A13800002800F096804D4DA0F80A9025F0030500
:10A148002A464560DAF80430A0F8089003F11007B1
:10A15800144618685968083303C4BB422246F7D12D
:10A1680018682060E888FFF716FBC0F30C0300F4BA
:10A178000050019383B204930822A9F1140393FBBE
:10A18800F2F39BB2BAF808400393DB009BB2143C8D
:10A1980005931423A4B20293002C5DD0019BA9F16E
:10A1A800130CA445C3F30C08049BD4BF4FF0000C58
:10A1B8004FF0010C43EA0808BCF1000F03D148F442
:10A1C8000058059F00E0274605F114013A46029B16
:10A1D8005046CDF81CC000F010FD029B184483B215
:10A1E80040460293FFF7D4FAE88007F1140080B2E2
:10A1F800FFF7CEFA002368806B8128461421FFF709
:10A20800C6FBDDF81CC06881BCF1000F05D004F165
:10A218001401304689B200F047FC002102200A46AA
:10A2280000F0B3FB804698B1314600F080FCDBF8C3
:10A238001430069A414658469847404600F092FB2B
:10A24800019B039AE41B13449BB2A4B20193A3E7B6
:10A25800304600F087FB04E0304600F083FB2046E0
:10A2680000E0FF2040B209B0BDE8F08F7D25002056
:10A2780080B485B000AF7860294B1B687A68128873
:10A288001344FB607A68FB689A421FD0FB681B790D
:10A29800002B1BD1234B1B68FA689A4216D0224B1D
:10A2A8001A68FB689A4202D11F4A7B681360FB68F0
:10A2B8001A887B681A801A4B1B68FA68128813443C
:10A2C8007A6817490968521A92B25A80144B1B6867
:10A2D8007A6852881344BB60BA687B689A421AD07D
:10A2E800BB681B79002B16D10F4B1A687B689A4202
:10A2F80002D10D4ABB6813607B681A88BB681A8054
:10A30800074B1B687A6812881344BA6804490968BD
:10A31800521A92B25A801437BD465DF8047B7047D2
:10A328005C2B0020602B0020642B002080B582B0BD
:10A3380000AF184B184A1A60164B1B687B607B6885
:10A348004FF470421A807B6800225A807B68002292
:10A358001A71104B1B6803F57043104A13600F4BBA
:10A368001B6801221A710D4B1B684FF470421A804A
:10A378000A4B1B684FF470425A800120FBF740F8E3
:10A388000246074B1A60034B1B68064A13600837DE
:10A39800BD4680BD5C2B002000100760602B0020AC
:10A3A800682B0020642B002080B584B000AF786053
:10A3B8007B68002B00D131E01A4B1B687A689A42FF
:10A3C800184B1B687A689A4204D3174B1B687A6843
:10A3D8009A4200D322E0154B1B6818460021FBF770
:10A3E8002BF87B68083BFB60FB6800221A71104B56
:10A3F8001B68FA689A4202D20D4AFB681360FB6830
:10A40800084A12689B1A1A460A4B1A60F868FFF73E
:10A418002FFF064B1B681846FBF734F81037BD466C
:10A4280080BD00BF5C2B0020602B0020682B002023
:10A43800642B00209050002080B586B000AF786073
:10A448000B467B807B8803339BB223F003037B801E
:10A458007B880B2B01D80C237B807B88B3F5704F4E
:10A4680001D90023A5E0554B1B687A689A42534BE3
:10A478001B687A689A4204D3514B1B687A689A42DF
:10A4880001D37B6895E07B68083B7B617B694B4A1D
:10A4980012689B1A7B827B691A887B8AD31A9BB2C3
:10A4A800083B3B827A883B8A9A4201D9002380E0A4
:10A4B8007A883B8A9A4201D17B687AE0414B1B68D3
:10A4C80018460021FAF7B8FF3C4B1B687A691288D6
:10A4D8001344FB60FB681B79002B32D1FB681B8897
:10A4E8007B817A8A7B8813449BB208333B81364B45
:10A4F8001A68FB689A4205D1304B1A683B891344A5
:10A50800314A13602D4B1A683B891344FB60FB6882
:10A5180000221A71FB687A891A80FB687A8A5A8045
:10A528007B693A891A80FB681B88B3F5704F07D09E
:10A53800224B1B68FA68128813443A895A8032E021
:10A5480031E07B8803F114023B8A9A422BD87A8A3D
:10A558007B8813449BB208333B81184B1A683B89AC
:10A568001344FB60184B1B68FA689A4202D2164AD9
:10A57800FB681360FB6800221A717B691A88FB6804
:10A588001A80FB687A8A5A807B693A891A80FB6844
:10A598001B88B3F5704F06D0084B1B68FA68128801
:10A5A80013443A895A80074B1B681846FAF76AFF22
:10A5B8007B6818461837BD4680BD00BF5C2B00205D
:10A5C800602B0020682B0020642B002080B586B00B
:10A5D80000AF0346FB80FB88002B01D10023A7E0D6
:10A5E800FB8803339BB223F00303FB80FB880B2B10
:10A5F80001D80C23FB80FB88B3F5704F01D90023E9
:10A6080096E04D4B1B6818460021FAF715FF4B4B97
:10A618001B681A464A4B1B68D31AFB827BE0484BDF
:10A628001A68FB8A13443B613B691B79002B6CD188
:10A638003B691B881A46FB8AD31AA3F10802FB88D8
:10A648009A4262D33B691B881A46FB8AD31AA3F144
:10A658000802FB8814339A4227D3FA8AFB881344EA
:10A668009BB20833FB81364B1A68FB891344BB60E5
:10A67800BB6800221A713B691A88BB681A80BB68DC
:10A68800FA8A5A803B69FA891A803B6901221A7151
:10A69800BB681B88B3F5704F0AD0294B1B68BA6892
:10A6A80012881344FA895A8002E03B6901221A7120
:10A6B800224B1B683A699A4218D107E0204B1B6865
:10A6C8001E4A1268128813441C4A13601B4B1B68ED
:10A6D8001B79002B05D0194B1A681A4B1B689A4234
:10A6E800ECD1164B1A68174B1B689A42124B1B6821
:10A6F8001846FAF7C7FE3B69114A12689B1A1A46B0
:10A70800114B1A603B69083312E00D4B1A68FB8A3B
:10A7180013441B88FB82FA8AFB88C3F570439A426C
:10A72800FFF67DAF044B1B681846FAF7ABFE002313
:10A7380018461837BD4680BD682B0020642B0020C2
:10A748005C2B0020602B00209050002080B584B046
:10A7580000AF03460A46FB801346BB80FB88BA88D5
:10A7680002FB03F39BB21846FFF730FFF860FB6863
:10A77800002B08D0FB88BA8802FB03F3F868002195
:10A788001A461EF0DBFFFB6818461037BD4680BD31
:10A79800A8B10B4A1368834203D10368136008E029
:10A7A80013462BB11A688242FAD102681A6000E097
:10A7B8007047044B1A68824204BF00221A6070472F
:10A7C800646F0020686F002010B5A0B182780A4B32
:10A7D800303AD2B21B686BB193F834109142F9D178
:10A7E800047893F832108C42F4D1447893F83310FB
:10A7F8008C42EFD1184610BD646F00200A68436888
:10A8080070B59A4204460D4602D12B68636070BD4C
:10A818000C4B186848B102686368C6689A4202D14E
:10A82800012100F02FFF3046F4E7074B1B68002B8F
:10A83800EBD01A6822B161688A4204BF2A681A609C
:10A84800DB68F4E76C6F0020746F002070B5154664
:10A8580006461C46FFF7D2FF05B12D68B56004B166
:10A868002468F46070BDF8B50446069E0F4FC661B3
:10A878003E78002506F1010E80F83460089E456098
:10A888008560C56080F831500562066187F800E090
:10A89800FFF7DCFF2046079B984728B9044B204662
:10A8A8001A6822601C60F8BD2846F8BD6C2B002091
:10A8B800646F002001B10968C160704701B109687F
:10A8C80081607047014B1860704700BF686F0020B7
:10A8D80090F831300146DA0708D443F001029B06AC
:10A8E80080F8312002D5043102F083BE704790F819
:10A8F8003130DA0744BF23F0010380F83130704764
:10A9080090F8310000F00100704700BF10B529B37E
:10A9180038B3002905DA4A42438992B2934201D2F8
:10A928001EE08AB2047B43680CB1032C05D15B1A84
:10A9380000F11002934209D212E0013C012C0FD819
:10A9480000290DDA448994420AD35B1A436043898B
:10A9580089B20B444381038919440181002010BD49
:10A96800012010BD38B578B10024E2B220B1C38906
:10A97800013B9BB2C3810BB1104638BD0568013459
:10A98800FFF712FD2846F0E738BD2DE9F0410D46E6
:10A998001646032800F28380DFE800F00204070B64
:10A9A800142400E00024143400E000240E34A4B27F
:10A9B80000E00024032E72D8DFE806F0465E5E024F
:10A9C800384B1E8B3046FFF701FE0746002866D03D
:10A9D80003230373002303600319033424F00304DF
:10A9E800C4F5BB640434AC42A8BF2C46804613337C
:10A9F80023F003034360012344810581C3812C1B99
:10AA0800002C45DD3046FFF7E1FD0023054628B957
:10AA18003846FFF7A7FF2846BDE8F0814373036077
:10AA280040F2DC5303220273A2B2934228BF1346BA
:10AA3800C8F80000028100F110024260012243813F
:10AA4800C281E41A8046DBE704F11300EB1C23F013
:10AA5800030320F00300184480B2FFF7B7FD074650
:10AA6800E8B10319133323F003034360002305817E
:10AA78004581036003730BE00A4BD88AFFF7A6FDF4
:10AA8800074660B100234360058145810360067372
:10AA98000123FB8100237B733846BDE8F081002049
:10AAA800BDE8F081C826030838B503890D469942E8
:10AAB8001ED2CA1A43899D4206D9ED1A0389ADB23E
:10AAC800134403810068F5E7027B044642B99D42BE
:10AAD80006D04168091A294489B2FFF7ADFC04463B
:10AAE80020686581258108B1FFF73CFF00232360BA
:10AAF80038BD03460022D0B201320BB11B68FAE719
:10AB0800704710B1C3890133C381704730B568B14C
:10AB180001B930BD05680C8925B10289A3180381E4
:10AB28002846F7E7038901602344038130BD10B547
:10AB38000C46FFF7EBFF2046BDE81040FFF7E1BFEA
:10AB480010B504680CB9002010BD428903899B1A0E
:10AB580023810023036002812046FFF703FF0028BA
:10AB6800F1D1204610BD2DE9F0410D4604460028DC
:10AB78003DD000293BD002890B899A4237D34FF048
:10AB88000008474663896E89DB1BC8EB0606B3429B
:10AB980060686968B4BF9EB2B6B238444144324670
:10ABA8001BF0D0FB37446389BFB2BB4246446B8974
:10ABB8001FFA86F804BF24680027434503D82D6888
:10ABC8004DB14FF000086A892B899A4201D12B6850
:10ABD8007BB914B9D6E76CB1A846628923899A4231
:10ABE80001D123682BB9002DCCD12C4602E0F624E4
:10ABF80000E0F72460B2BDE8F0812DE9F84388460B
:10AC08009146064628B331B300242746B9F1000F10
:10AC180024D01EB32BB171898B4202D35B1A9BB22D
:10AC280015E072897168D21A95B24D4528BF4D4614
:10AC380008EB070019442A462C442F44C5EB0905A4
:10AC48001BF080FBA4B2BFB21FFA85F90023366857
:10AC5800DCE7BDE8F8830846BDE8F8832046BDE890
:10AC6800F8832DE9F04188461446054608B90020C6
:10AC780018E00029FBD00389934212D30026002C48
:10AC8800F5D06F896868A74228BF274608EB0601F8
:10AC98003A46E41B3E441BF055FBA4B2B6B22D68FD
:10ACA800EDE7F62040B2BDE8F08138B50368044608
:10ACB8000BB9204638BD084600222189FFF765FEFA
:10ACC80005460028F5D02146FFF74DFF2046FFF73F
:10ACD80049FE284638BD00BF2DE9F047D0F804905A
:10ACE8008046B9F80800FEF756FD154E5FFA80FA5F
:10ACF80034680027F4B1237C534512D1656985B1C6
:10AD0800A0692146424609F10C03A84768B157B12A
:10AD1800E3680120FB6033684FF00008E3603460AB
:10AD280003E0002001E0B8460120E368274620B987
:10AD38001C46DFE72046BDE8F0870120BDE8F08724
:10AD4800702B002001B1096801600020704701B133
:10AD58000968416000207047416182617047F0B521
:10AD6800044685B00E46084614211746FFF7CEFD67
:10AD780060B1002101200A46FFF707FE054608B921
:10AD8800FF202EE03146FFF7D2FE07E030466FF095
:10AD98001301FFF7BBFD0028F2D135463846FEF710
:10ADA80021FE28B9B54219D02846FFF7DBFD15E08A
:10ADB80021460CB1236803B9011DA27AE37A0092F7
:10ADC800227C0290019228463A46FEF701FFB542DE
:10ADD800044605D02846FFF7C5FD01E0FC2000E049
:10ADE800204640B205B0F0BD021DFFF7B8BF094AC2
:10ADF8001368834209D1C368136008E0DA681AB19E
:10AE0800824204BFC268DA60DB68002BF6D1FFF724
:10AE1800CBBA00BF702B002038B50A4B05461888FE
:10AE2800FFF7D4FB044650B11C2200211EF086FC1B
:10AE3800FF23E372044B25741A681C60E260204605
:10AE480038BD00BFC8260308702B002001230380EB
:10AE580043681868FAF716BBF8B505460E46FAF7C0
:10AE68002FFB044608B1036833B928463146BDE8CC
:10AE7800F8400022FAF782BA5A685AB9206803687B
:10AE8800C76823608468FFF78FFA002CE7D038463C
:10AE9800A047E4E728463146FAF770FA431CEDD09C
:10AEA80022685368984234BF1B1A00235360F8BDC8
:10AEB80070B50546FAF704FB044608B103682BB9D8
:10AEC8002846BDE870400021FAF7B6BA596859B962
:10AED80020680368C66823608468FFF765FA002C59
:10AEE800E8D03046A047E5E72846FAF7A5FA431C1C
:10AEF800EED022685368984234BF1B1A002353606F
:10AF080070BDF8B5164B0546988A0F461646FFF7EA
:10AF18005DFB044610B3002303608760C66045608C
:10AF2800FAF7CEFAD0B103682BB15A68AA4208D909
:10AF3800521B5A6023600460F8BD5068884208D8E4
:10AF4800134662685968511A1A686160002AF4D178
:10AF580001E0411A516022601C60F8BDF8BD00BFD5
:10AF6800C826030870B505460E46FAF7A9FAE8B1EF
:10AF78000368DBB100229968A94212D1D968B142AD
:10AF88000FD119680AB9016000E011601A681AB196
:10AF980050685968014451601846BDE87040FFF791
:10AFA80003BA1C681A460CB12346E4E770BD1FB506
:10AFB80004AB43F80C0D03930023ADF8083021B11E
:10AFC800084602AA0949FFF79CFF0198FFF770FF9E
:10AFD800BDF908302BB9054802A9FFF7C3FF0120C6
:10AFE80000E0002005B05DF804FB00BF55AE000886
:10AFF80038B505460020FAF703FA04462946FFF754
:10B00800D6FF2046BDE83840FAF744BA6FF004008E
:10B01800704770B5124B134A19681468124B134ADB
:10B02800188815680A46013080B210F4004F18BF1E
:10B038004FF4805022B1168B8642F3D0D268F9E7DC
:10B04800224622B1168B8642ECD0D268F9E72A460E
:10B0580022B1168B8642E5D0D268F9E7188070BD18
:10B068006C6F0020806F002020000020746F00208B
:10B07800F8B5037C05460C46002B4CD112B9FFF7F6
:10B08800C8FF0246264B1B6873B1198B914209D140
:10B098001868002841D0002C3FD0216800293CD0F6
:10B0A80088423AD0DB68EFE71E4B1B685BB1198B0F
:10B0B800914206D1186880B37CB3216869B388428D
:10B0C8002BD0DB68F2E718490F680E463B465BB1A8
:10B0D800198B914206D11868F8B1F4B12168E1B131
:10B0E80088421AD0DB68F2E7104B1B6843B1198B12
:10B0F800914203D12168186888420ED0DB68F5E7D1
:10B1080014B1236803B12B602A83EF603560FCF724
:10B11800BDFF002002E0F32000E0F52040B2F8BDBA
:10B12800746F00206C6F00207C6F0020806F0020FF
:10B1380038B5037C05460BB1002038BD1C4BD888B8
:10B14800FFF744FA04460028F6D06B69194A4361B0
:10B158002B8B0383012303742B8943F002030381A0
:10B16800EB7AC372AB7A83722B6803601368AB42C5
:10B1780001D1EB680BE0104A136043B1D968A942CA
:10B1880003D11360EA68DA6002E00B46F5E7136062
:10B1980000232846EB60FFF707F9084BE361084BEB
:10B1A8001A681C60E260FCF771FF204638BD00BFDA
:10B1B800C82603087C6F0020786F002015B00008AF
:10B1C800746F002070B5C16A068D446A731A058FC2
:10B1D8000246181941F64C539D4294BF431BC31AAB
:10B1E800002B01DB568570BD631A002B4FF0000061
:10B1F800D6BF091B5085518570BD038D10B5194404
:10B2080043F6982389B299428CBF03850185044689
:10B21800FFF7D8FF40F6A56398420ADD94F822307C
:10B22800204643F0020384F82230BDE8104001F0C4
:10B238001FBC10BD38B5054640B1406808B1FFF7DE
:10B2480091FB04462846FFF7AFF800E00446204685
:10B2580038BD38B5002430B10568FFF7EBFF20444E
:10B26800C4B22846F7E7204638BD417470474161AB
:10B278007047C0F884107047C0F880107047C0F855
:10B2880090107047C1617047C0F88C1080F8352065
:10B298007047037C10B5012B044610D90A2B0ED039
:10B2A800C06F18B1FFF75EFB0023E367606FFFF71D
:10B2B800D0FFA06FFFF7CDFF00236367A36710BD22
:10B2C8002DE9F743874F4FF000093B6801333B6096
:10B2D800854B98461C68002C00F0E580217C94F88A
:10B2E8004A20022901D1062A51D00C2A4FD094F8BD
:10B2F8009C30C3B17D49D4F89820194411F8011C39
:10B3080001328A42C4F898203FD3062B4FF000023E
:10B3180098BF0133C4F8982098BF84F89C30204621
:10B3280001F0DAFD31E0E38E18045CBF0133E386F7
:10B33800A36F53B3B4F93600B4F94830984224DB0C
:10B3480002290BD0B4F94410B4F9463003EBE103F9
:10B3580066490A44D2799340A4F848300023B4F8E7
:10B368005220E386B4F85C302046934228BF134647
:10B37800228F5B089342A4F854303CBF5300A4F8D2
:10B388005430A4F8522001F012FD002500E00125F8
:10B39800237C062B06D13A68216B521A282A84BFCF
:10B3A8000135EDB2268906F00806B6B246B3042B7D
:10B3B80001D0072B23D13B68216B4FF4FA70591A3F
:10B3C800D4F8943003F5242202F6B842B2FBF0F226
:10B3D800914203D90135EDB2012611E094F89D2080
:10B3E800434E06FB0233B3FBF0F3994207D92046DC
:10B3F80001F043FD94F89D30013384F89D30002618
:10B40800237C032B07D13B68226B9B1A282B09D975
:10B418000135EDB206E0092B04D13B68226B9B1A7B
:10B42800F02B00D81DB32046FFF733FFE368B9F1CE
:10B43800000F02D0C9F80C3001E0C8F80030D4F889
:10B4480090301BB160696FF0040198474EB1238BAF
:10B4580022460093238C0193A06D616A231D01F09D
:10B4680049FC2046E568FEF79FFF4C4618E094F833
:10B47800343094F835200133DBB29A4284F8343002
:10B488000DD8D4F88C3084F834501BB9204601F01C
:10B49800EFFA04E06069214698470028F6D0E5688D
:10B4A800A1462C4617E7134B98461D68BDB13B686B
:10B4B8002A6B9B1AF02B10D92846FFF7EAFEEB6897
:10B4C8000CB1E36001E0C8F800302846EE68FEF7EA
:10B4D8006BFF25462C463546E8E7EE68FAE703B0E9
:10B4E800BDE8F083706F00206C6F0020E42603082D
:10B4F800F8240100806F0020036810B58B420C46C9
:10B5080002D1CB6803600CE0124A136043B1D968DA
:10B51800A14203D11360E268DA6002E00B46F5E766
:10B5280013600023E3602046FFF7B3FE237C0A2B59
:10B538000CD0012B0AD094F82230DA0706D543F054
:10B54800020384F82230204601F092FA0023237483
:10B5580010BD00BF786F0020037C10B50446072B90
:10B5680034D8DFE803F0041A1C242433332A194A98
:10B578001368834201D1C3680BE0174A136043B1D3
:10B58800D968A14203D11360E268DA6002E00B4691
:10B59800F5E713600023E36005E0104800E0104879
:10B5A8002146FFF7A9FF2046FEF7FEFE0EE0012127
:10B5B80001F008FA58B9052304E0012101F002FA64
:10B5C80028B909232374204601F052FA002040B21A
:10B5D80010BD00BF7C6F0020786F0020746F0020C2
:10B5E8006C6F002010B50846144632B11189FFF778
:10B5F80004FE2046FFF7B6F904E01BB9BDE8104089
:10B60800FFF7AABF002010BD38B5144B1C681CB347
:10B61800E26F72B1D4F8845025B1606921460023E5
:10B62800A84704E0284621462B46FFF7DBFF00B970
:10B63800E06794F82230DA070CD543F0020384F867
:10B648002230204601F014FA94F8223023F0030344
:10B6580084F82230E468DAE738BD00BF6C6F002058
:10B6680008B5FFF7D1FF064A13780133DBB2137030
:10B67800DB0703D5BDE80840FFF722BE08BD00BFC1
:10B68800742B00202DE9F04F037C85B00A2B04466B
:10B698008A4607D11C482146FFF72EFF2046FEF7B1
:10B6A80083FE2EE00368876D03934368466AB0F80B
:10B6B8001890B0F82080D0F89050D0F814B02146F7
:10B6C80012480293FFF718FFA06F08B1FFF7C1FDFA
:10B6D800606F08B1FFF7BDFD2046FEF765FE1DB19E
:10B6E80058466FF00401A847BAF1000F09D0CDF809
:10B6F8000090CDF804803846314603AA02AB01F029
:10B70800F9FA05B0BDE8F08F806F00206C6F00205B
:10B71800034A044B1868536818445060704700BFC8
:10B7280020000020706F0020F8B53B4B07469D882D
:10B738003A4E2846FEF74AFF0446002834D1384BD3
:10B7480031681B683BB11A6B8A1AA24224BF18469B
:10B758001446DB68F6E710B10121FFF793FF28468E
:10B76800FEF734FF0446F8B92E4BD6F800C01B6824
:10B778004FF07F0E73B1597CB94209D8714507D88B
:10B788001A6BC2EB0C02A24222BF8E461446184620
:10B79800DB68EFE710B10121FFF774FF2846FEF7D9
:10B7A80015FF0446002835D00021A02220461DF0B0
:10B7B800C5FF43F6081240236374E3724FF406731F
:10B7C80023870623A4F84830A4F846304FF6FF73C1
:10B7D800A4F86E2043F698220025E3860123A4F8F6
:10B7E8005230A4F8705022856285A572A4F844509E
:10B7F800FFF78EFF3368606623630B4BA065C4F8C0
:10B8080084300A4BE064A06684F83450C4F894305D
:10B8180084F89D502046F8BDC8260308706F0020A4
:10B82800806F00206C6F0020EDB5000800DD6D0012
:10B838004020FFF779BF10B504460846FEF7D2F856
:10B8480030B1038D23B1283B9BB29C4228BF1C46D4
:10B85800204610BD73B51E46037C04460D46002BDA
:10B8680053D1002953D00868238B6060228413B910
:10B87800FFF7CFFB2083FFF74BFF43F69823A06524
:10B8880001380022E064A0664FF4067062622385E6
:10B898006385E262A4F85C3020872946FFF7CBFF76
:10B8A800012320871D4A00EB80009840A4F85230FD
:10B8B800022323741368A4F85400A342C4F88860D0
:10B8C80001D1E3680BE0164A136043B1D968A1427D
:10B8D80003D11360E268DA6002E00B46F5E7136013
:10B8E800104B1A681C60E260FCF7D0FB00210123B2
:10B8F8008DE80A0020460A46022300F08EFE05461F
:10B9080038B9204601F0B4F803E0F32002E0F7204C
:10B9180000E0284640B202B070BD00BF7C6F002036
:10B92800786F00206C6F0020024B03EB800080686A
:10B93800704700BF200000202DE9F041B44D0446B7
:10B948002B78DE0640F14481016E6B68B0F85C60CC
:10B95800426EC81A00280DDB994203D1A968511A12
:10B96800002907DBA9688A4212D1A949C968C9898F
:10B97800B1420DD9E968C9892366AB68A4F85C109F
:10B98800636629B194F89C3013B1002384F89C3085
:10B99800A968E06C0B1A002B30DC0023A4F86C308B
:10B9A8009B4B1B8A002B40F0EB81B4F85C70636EF4
:10B9B80032443B44934240F0E381B4F93630002BE3
:10B9C800C0F2DE81884240F0DB8194F850300133C8
:10B9D800DBB2032B84F850300AD9B4F85220238FF5
:10B9E80013449BB2934240F2C780A4F85230C3E09C
:10B9F80040F0C280204601F015FABDE0A26D8A1A17
:10BA0800002A79DC94F82220B4F94460500742BF38
:10BA180022F0040284F82220B4F854209BB248BFD4
:10BA2800A4F85220B4F84620A4F86C3002EBE602E1
:10BA3800A4F84820B4F86E2000201344A4F86E300F
:10BA4800237C84F84A00032B84F85000E16445D92C
:10BA5800B4F85220B4F854309342238F9CBF5B4310
:10BA680093FBF2F313449BB2934237D9A4F85230B4
:10BA780034E01B695868FDF71FFFA36F06469F89CE
:10BA88001B699889FDF787FEAB6810F0030018BFA3
:10BA98000120F61A38443044002822DCA66F3368A7
:10BAA8007068A367FFF725F8B4F86C305BB13369A9
:10BAB8009889FDF770FEC30742BFB4F86C3003F1F4
:10BAC800FF33A4F86C307068FFF713F8B4F87030DF
:10BAD800181AA4F870003046FFF7ACFBA36F002BD0
:10BAE800C7D1A26F00231AB94FF6FF72E28600E0B1
:10BAF800E38684F834303FE00023A4F86C303BE060
:10BB08001B69AE685868FDF7D7FE636F80469F894A
:10BB18001B69C8EB06069889FDF73DFE10F0030087
:10BB280018BF01203844361A002E28DB384BA26D86
:10BB38009B689B1A002B22DC666F3368706863670A
:10BB4800FEF7D7FFB4F86C305BB133699889FDF71D
:10BB580022FEC70742BFB4F86C3003F1FF33A4F8E4
:10BB68006C307068FEF7C5FFB4F87030181AA4F886
:10BB780070003046FFF75EFB636F002BC0D1E16BAE
:10BB880031B3236CAA689B1A002B21DA214AB4F836
:10BB980044301268521A43F3CC01521A92B291B24D
:10BBA8000804134444BF524291B2B4F846209BB2F1
:10BBB80042F38D00121A0A4492B2A4F8443043F3B7
:10BBC800CC031344A4F848300023A4F84620E363C8
:10BBD8000F4E2F8A626A7368002F00F0BD80D11A59
:10BBE80001292CD4501CC01AC01B002827DCB669B8
:10BBF8000B4672898A4211DA3289521A92B27189D5
:10BC0800994209DA5B1A0021328171813668F6E7B8
:10BC1800782B0020706F0020594200E0494209B299
:10BC28003046FEF773FE73686968EB612B8C626AB5
:10BC38000B449B1A2B846B6A6A605A600BE09B1A50
:10BC4800002B08DA94F82230204643F0020384F8E7
:10BC5800223000F00DFF6A68616A4C4E531A002BBF
:10BC680075DB531C208D5B1A1B1A002B6FDC91426D
:10BC78006DD1736A378C9889FDF78DFD10F003003C
:10BC880018BF01203844238D80B28342308233D2DA
:10BC9800736A9889FDF77FFDC70710D5736A4FF659
:10BCA800C0709F89FDF774FD766A0740B089FDF77B
:10BCB80072FD00F03E00FDF76BFD3843B081238D27
:10BCC800324E2B846B6A9889FDF765FD800748BF63
:10BCD800338CA86944BF03F1FF333384298CFEF702
:10BCE800E3FE6B6A2E8C9889FDF755FD10F0030072
:10BCF80018BF012030442882298A238D6A685B1A7C
:10BD08000A44626223852046FFF75CFAAB691F4E3E
:10BD18001A8912B1B3620023B3616B6A1B4E98890A
:10BD2800FDF739FDC10742BF96F82C3043F02003D8
:10BD380086F82C3094F82230DA0702D523F0010374
:10BD480015E043F0010384F82230BDE8F081204675
:10BD5800BDE8F04100F057BE991A002905DB013310
:10BD68009B1A228D9B1A002B0EDD94F8223043F08B
:10BD7800020384F822302046BDE8F04100F078BE86
:10BD8800002384F85030F7E6BDE8F081782B0020D6
:10BD9800F8B51E4E0446F568A889FDF7FCFCC0F30B
:10BDA8000F30052831D9F36814359889FDF7F3FC6D
:10BDB800000B0538800080B20023834225D2EA5C5C
:10BDC800012A05D021D3022A05EB030102D017E08E
:10BDD800013318E04A78042A17D1DA1C824214DAAF
:10BDE8008E78CA7840F2B35742EA062240F2B45637
:10BDF800511E89B2B94288BF32460433228002E01C
:10BE08004A7812B113449BB2D7E7F8BD782B0020CB
:10BE18002DE9F3474468B84D074620880E462C6341
:10BE2800FDF7B9FC2B6BC0F3032004EB80041888E2
:10BE3800EC60FDF7B0FCC0F30320810049423846AE
:10BE4800FEF764FD10B93B89132B05D8384602B0BC
:10BE5800BDE8F047FEF786BD286B31461030FDF788
:10BE680043FF0028F2D12B6B4FF070401C69FDF79F
:10BE780023FD04404FF06040FDF71EFD8442E5D0ED
:10BE88002A6B3B8902F10C010093384610320623D5
:10BE9800FDF739FD0028D9D1EB689889FDF77BFCBF
:10BEA800000BC0EB8030810009B23846FEF72EFD4A
:10BEB80006460028CAD1EC68DFF84C822088FDF7D6
:10BEC8006AFC2080EC686088FDF765FC6080EC689F
:10BED8006068FDF7F1FC6060EC686860A068FDF7D9
:10BEE800EBFCA060EC68A860E089FDF754FCEB6807
:10BEF800E0819889FDF74FFCD8F800905FFA80FE42
:10BF08004C4630461EF00302B7F808C018BF01229D
:10BF18000EF03F0362442B7092B2E9682B6B2A82C1
:10BF280004B3B4F820A00E88B24518D1B4F818A00C
:10BF38004E88B24513D1D3F80CA0666856450ED189
:10BF4800D3F810A02668564509D1002800F0DE80F5
:10BF5800E368C8F80040C360C4F80C90D6E02046F7
:10BF6800E468DDE76548006800283AD0048C0E884C
:10BF7800A64234D1048BB1F802C0A4452FD1D3F81E
:10BF88000C9044684C452AD1D3F8109004684C456D
:10BF980025D11EF0040F7FF459AF1EF0020F0ED00A
:10BFA8006968446A0C1B10D4058D641B002C0CDCDA
:10BFB8005148CDF800C00196806811443AE01EF05F
:10BFC800010F1EBF4E4B1B680363002A3FF43EAFB0
:10BFD80090F8223043F0020380F8223031E0C06844
:10BFE800C2E7484CD4F80090A4464E4605E0D3F882
:10BFF80010A0544507D03046F668002E00F0AE82F7
:10C008003468002CF3D14C88B6F818A0A245F2D1B8
:10C0180028B1F368CCF80060C360C6F80C901EF035
:10C02800100F11D0A8682B6B6D6800940988013037
:10C038000191511903F110020C3300F05BFE05E782
:10C04800204600F015FD01E71EF0020F3FF4FEAE9A
:10C05800707CFFF769FB044600283FF4F7AE2B6BB2
:10C0680013F1100218BF1A690260328B028313F1B0
:10C078000C020CBF1346DB68EA68436051781378FA
:10C0880043EA01230384032303746B680025591CC6
:10C098004162C162013BD28903667369A0F85C20E2
:10C0A8004361F369A0F85420C361338923F0660320
:10C0B800DB05DB0D0381D8F80030C8F80000C36049
:10C0C800FBF7E4FF04F13800FFF762FE211D208F23
:10C0D800FFF7B1FB012320872946019300952046ED
:10C0E8002A46122300F099FA0028A9D020462946AA
:10C0F800FFF7C8FAAAE600BF782B0020806F00205F
:10C10800706F0020746F00206C6F00207A68002325
:10C11800EA61E26F6B61A5F820C0AF616962AB624A
:10C1280085F82C307AB1D4F884601EB16069214654
:10C13800B04704E0304621463346FFF753FA00285B
:10C148007FF484AEE0672B78AE4E59073460AE4A70
:10C1580013D5237C022B05D19268A36D9A4240F037
:10C16800A3810CE25368626A9B1A00F19D81228DBB
:10C178009B1A002B00F3988101E29F0703D5237CCB
:10C18800023B012B6AD8A14B04F138001B682363DA
:10C19800002384F89D30FFF7FBFD237C023B072B2F
:10C1A80000F28281DFE813F008007600C000D300B7
:10C1B8000D01C000360169012B78934F03F012037B
:10C1C800122B55D1A36FD7F808801B695868FDF763
:10C1D80073FB013080454BD1B4F86E30F9680133F8
:10C1E800A4F86E307B68208F5A1C6262E262BA68DB
:10C1F800013BE2648A7BC97B236642EA012204236D
:10C208002374E118A4F85C20FFF715FB00EB80030A
:10C218005B00A4F85430B4F852302087012B04BFD7
:10C22800400080B2B4F87030A4F85200A06F013B0F
:10C23800A4F870300368A3671BB94FF6FF73E38651
:10C2480003E00023E38684F84A30FEF7F3FFD4F8CE
:10C2580088301BB1606921460022984794F8223043
:10C26800204643F0020384F8223000F001FC1BE171
:10C278002B78654AD80640F11781D068178AB0F83C
:10C2880002E05168136BCDF800E000883944019052
:10C29800906836E02B785C4AD90638D5E36C90680C
:10C2A800DB43C34224D4A36DC31A002B20DC042330
:10C2B8002374E3694BB1606921460022984720B195
:10C2C80020460121FFF7DEF93FE12046B4F852701D
:10C2D800FFF732FBB4F86C3013B1013BA4F86C30B3
:10C2E800238F012F04BF5B009BB2A4F852301EE0DD
:10C2F800EA682F8A51882B6B0091128801926A682C
:10C30800B91803F110020C3300F0F4FCCCE09F07DD
:10C3180040F1CA80636A5268013B9A4240F0C48087
:10C32800204600F05BFDBFE02046FFF705FB95F8CF
:10C338002C30980640F1B88094F82230204643F01B
:10C34800020384F8223000F093FB07232FE02046F5
:10C35800FFF7F2FA95F82C302B4A13F0200F2B78C0
:10C3680027D013F0100F94F8223043F0020318D0AE
:10C378009168A26D914214D184F82230204600F0D1
:10C3880077FB2046FEF785FFD8F80030A34259D046
:10C398001F4A1360002B66D0D968A14259D00B46BA
:10C3A800F8E784F82230204600F062FB0823237463
:10C3B8007AE0D90678D59268A36D9A4274D106239B
:10C3C800F5E72046FFF7B8FA95F82C309B066BD5B1
:10C3D80094F82230204643F0020384F8223000F01B
:10C3E80047FB2046FEF755FFD8F80030A34229D076
:10C3F800074A1360002B36D0D968A14229D00B46D2
:10C40800F8E700BF846F0020782B0020706F0020B1
:10C41800786F00202046FFF78FFA2A7802F0100282
:10C4280002F0FF0322B15E4B9B68003318BF012363
:10C43800A26D934238D12046FEF72BFFD8F8003082
:10C44800A34203D1E268574B1A600DE0564A1360C5
:10C4580007E01360E268DA6006E0D968A142F8D024
:10C468000B46002BF9D113600A2323744F4B1A682B
:10C478001C60E260FBF70AFE16E02046FFF75CFA54
:10C488002A7802F0100202F0FF0322B1444B9B68A5
:10C49800003318BF0123A26D934202BF95F82C30D8
:10C4A80043F0100385F82C3095F82C301F0707D57A
:10C4B800D4F8903033B160696FF00501984701E016
:10C4C800D80607D537482146FFF716F82046FDF766
:10C4D8006BFF3AE0B4F86C202AB1D4F8803013B17D
:10C4E800606921469847AA6ABAB12D4B1B7819078B
:10C4F80042BF537B43F001035373D4F8847027B1D0
:10C50800606921460023B84704E0384621463B4687
:10C51800FFF768F808B1AB6AE36795F82C309A061C
:10C528000ED5D4F884702FB10022606921461346D5
:10C53800B84705E0384621463A463B46FFF752F8E9
:10C5480000232046336000F093FAA8690024346081
:10C5580010B3FEF707FA124B9C611DE08889FDF7BE
:10C568001AF943073FF572ACEA682C8A5088696863
:10C578002B6B0090128821440192A8685AE595F81F
:10C588002C3043F0080385F82C3094F8223023F03F
:10C59800010384F8223087E702B0BDE8F08700BFC6
:10C5A800782B00206C6F0020786F0020806F0020AF
:10C5B80070B50546008B0C461646FDF7E9F8208055
:10C5C800288CFDF7E5F866606080686AFDF7E6F894
:10C5D800A0604FF6C070A689FDF7DAF80640102073
:10C5E800FDF7D6F83043A081688DFDF7D1F8002615
:10C5F800E081A674E674A089FDF7CDF800F03F004D
:10C6080040F4A040FDF7C4F86A8D6B6AA08113441A
:10C61800267466742046EB6270BD2DE9F04F8BB02E
:10C628009A469DF85030064606939DF85430059179
:10C638000293914642B91BB91AF0030F00F0B38177
:10C64800059B002B40F0AF81B6F86E304B4506D203
:10C6580096F8223063F07F0386F82230A7E1029B28
:10C66800029A13F0010302F0020118BF0423002903
:10C6780014BF0C210021B6F87080CB180093B36E5C
:10C68800B8F57A7F0493E3D20027CB463A46009B5D
:10C69800C3F3870305331B039BB20793059B0193E1
:10C6A8000892338F009A9B1A5B45A8BF5B46039399
:10C6B800B64BBDF80C501889FDF788FF04460028D2
:10C6C80000F0668100230360436017B1089A106088
:10C6D80000E00746069B13F001001ED0009B0020D7
:10C6E800E91889B20246FEF750F96060002800F0A8
:10C6F8004F81FEF7FEF9059B40441FFA80F843B1CD
:10C70800636801995868009BBDF80C20184419F01B
:10C7180019FE63685B68A36028E0BDF80010024654
:10C72800FEF733F96060002800F03281FEF7E1F986
:10C7380040441FFA80F8BBF1000F17D029460320A8
:10C748000122FEF722F9014630B900906068FEF731
:10C7580009F9009961601BE1019B08F10108436038
:10C76800A36060681FFA88F8FEF7D0F9B8F57A7FF9
:10C7780000F20E81A58160681421FEF7C7F80990C0
:10C78800002840F005816268308B5268C5EB0B0BBE
:10C7980022610892FCF7FCFF089A1FFA8BFB1080B5
:10C7A8002269308C0892FCF7F3FF089A50802269BE
:10C7B80004980892FCF7F2FF089A099B50602269D6
:10C7C8004FF6C0709374D374938909920893FCF759
:10C7D800DFFF089B034050460893FCF7D9FF089BEE
:10C7E800099A18439DF808309081A37323699889A2
:10C7F8000893FCF7D0FF079B00F03F001843FCF7B5
:10C80800C7FF089B049A9881BDF80C301A4404921B
:10C81800019A1A4413460192BBF1000F01D0224637
:10C828003EE7D6F874B0CDF80480BBF1000F00F0F5
:10C83800C080DBF800200AB19346FAE7BBF80C2069
:10C84800DBF8101002928889FCF7A5FF029A10F015
:10C85800030018BF0120C24200F0AD80DBF81020B1
:10C868009089FCF798FF830740F0A5801AF0030F22
:10C8780003D0BAF1010F40F09E80BBF80C10BA89C2
:10C888000A44318F8A4200F396809BF80E10BA7BD7
:10C89800914240F09080DBF810205068FDF70CF8CA
:10C8A800BBF80C203969024402924868FDF704F885
:10C8B800029A82427FD1009B7868C3F57F41EC31B0
:10C8C80009B2FEF723F8002862D1786842894AB98C
:10C8D800016808F1FF3879601FFA88F30260019354
:10C8E800FEF740F81AF0010F0CD0DBF810200120F9
:10C8F800B2F80C800092FCF74BFF009A40EA08005F
:10C9080090810DE07968DBF80400FEF7FFF8B9893B
:10C91800BBF80C200A44ABF80C203A68CBF800208E
:10C92800BC42384604BFBBF80C505C46FDF73CFDE2
:10C938001AF0030F1CBF09F101091FFA89F91AF04F
:10C94800010F1EBF96F8223043F0200386F82230EC
:10C95800B36E4B44B366B6F86E30C9EB0309BDF845
:10C968000430A6F86E90A6F870303DB32469E4B19F
:10C97800069B03F0020303F0FF05B3B90820A6895C
:10C98800FCF706FF3043A08118E000BFC826030863
:10C9980096F8223063F07F0386F822303FB138469C
:10C9A800FEF757FC03E0F62508E0002506E0FF2522
:10C9B80004E07767BCE7CBF80070B9E768B20BB062
:10C9C800BDE8F08F07B50B460122002100920191C6
:10C9D8000A46FFF722FE03B05DF804FB37B5047C76
:10C9E8001D46072C02D0023C022C06D8002332B187
:10C9F80000950193FFF711FE02E0F82000E01046D1
:10CA080040B203B030BDF7B504461421012000221E
:10CA1800FDF7BBFF054638B394F82230A06D23F02C
:10CA2800030384F82230FCF7B9FE69680246204601
:10CA3800FFF7BEFD2B89261D074600932146324687
:10CA480006232846FCF75FFF3882A27AE37A009231
:10CA580006220192214632462846FDF729F9284642
:10CA6800FDF780FF002000E0FE2040B203B0F0BDDB
:10CA78009D4B2DE9F7431B680446834200F02F8144
:10CA8800B0F85230B0F85C80456F984528BF98469A
:10CA980090F822309A0710D52DB9204603B0BDE88A
:10CAA800F043FFF7B0BF2B695868FCF705FFAB8967
:10CAB800E26C9B1A18444045EFD8A66F002E00F090
:10CAC800A8803368002B00F0A4801E46F9E72B6984
:10CAD8005868FCF7F1FEAB89E26C9B1A1844404594
:10CAE80000F2E3802B699889FCF755FEA36F002BB1
:10CAF80040F093802B686367237C022B0FD0D5F816
:10CB080010901020B9F80C70FCF742FE3843A9F8D1
:10CB18000C0094F8223023F0030384F82230606A72
:10CB28002F69FCF73BFEB860608D2F69FCF730FE7B
:10CB3800628D636AF8811344E362AB7B2F69DB077C
:10CB480003D56A48FCF72AFE7861274657F8043B64
:10CB5800002B74D0B4F93630013304BF0023E386C8
:10CB6800E36B3BB9624B1B68E3632B695868FCF7BE
:10CB7800A3FE20646868D5F8109043684289C3EB27
:10CB880009039BB2D21A42810289C0F80490D31AD1
:10CB98009BB200220381214689F8102089F81120D0
:10CBA80000933A460623FCF7AEFEA9F81000A27AD5
:10CBB800E37A009206220192686821463A46FDF718
:10CBC80077F82B695868FCF777FE2B690746988930
:10CBD800B5F80C90FCF7DFFD10F0030018BF01203A
:10CBE800A36D484438441B1A002B2B69B8BFA065B5
:10CBF8009889AF89FCF7CFFD10F0030018BF01201A
:10CC0800C74249D000232B60A36F03BBA5672E46FC
:10CC1800656F002D7FF45BAF5BE094F8222012F083
:10CC2800440F7FF467AF636F002B3AD0196800296F
:10CC38007FF460AF9989238F994232D35AE73846F7
:10CC4800FCF7D0FE0028BCD04368236082E72B693C
:10CC58005868FCF731FE336907465868FCF72CFE24
:10CC6800381A002816DA04F178073B681BB93B68C4
:10CC78002B603D6013E01B695868FCF71DFE2B69AB
:10CC880081465868FCF718FEC0EB09000028EEDA68
:10CC98003F68EAE73560BAE72846FEF7CBFA35463B
:10CCA800B5E712F0A00F7FF425AF94F89C6086B921
:10CCB8002B695868FCF700FEAB89E26C9B1A184494
:10CCC800B4F85C30984282BF0123C4F8986084F8B5
:10CCD8009C3094F8223003F07F0384F8223000203F
:10CCE80003B0BDE8F08300BF846F0020B4050402E0
:10CCF800706F00202DE9F74F81460E4690460120BF
:10CD0800142100221F46BDF830B0BDF834A0FDF74D
:10CD18003CFE0546002847D044685846FCF738FDD5
:10CD280020805046FCF734FD60804846FCF736FD0D
:10CD380060603046FCF732FDA0604FF6C070A689EF
:10CD4800FCF726FD06401420FCF722FD3043A081A5
:10CD580043F69820FCF71CFD0026E081A674E674D3
:10CD6800A089FCF718FD00F03F0040F4A040FCF754
:10CD78000FFD2B89A08126746674414600933A46BC
:10CD880028460623FCF7BFFD06232082414601936F
:10CD9800009628463A464023FCF78AFF284603B007
:10CDA800BDE8F04FFDF7DEBD03B0BDE8F08F826F40
:10CDB80010B592B111460B680BB11946FBE7446FE9
:10CDC8000C60426790F84A208367013280F84A2055
:10CDD800C363BDE81040FFF74BBE10BDF8B5866FC2
:10CDE8000446F6B1336800F1740583672B6853B9BC
:10CDF8002B6833602E6094F84A30013384F84A3047
:10CE08000023E363F8BD1B695868FCF755FD3369D7
:10CE180007465868FCF750FD381A0028E8DA2D68EC
:10CE2800E4E7F8BD836F10B504462BB390F82230C1
:10CE38005B0721D4FFF7D2FFB4F85230B4F85C2076
:10CE480093428BBF52085B08A4F85420A4F85430CE
:10CE5800228FB4F8541053009942B8BFA4F8543044
:10CE68001344B4F854201344A4F8523094F82230F0
:10CE780043F0040384F8223010BDF7B505461421A9
:10CE880001200022FDF781FD044618B3A86D2E1D70
:10CE98000138FCF783FC616802462846FFF788FBE7
:10CEA8002389074600932946324620460623FCF785
:10CEB8002AFD0021388206228DE80600EB7A2046FA
:10CEC80029463246FCF7F4FE204603B0BDE8F040A0
:10CED800FDF748BD03B0F0BD2DE9F341866F054667
:10CEE80016B9466F002E4AD033699889FCF753FC6F
:10CEF80010F0010007D0B389002B15BF00270127C8
:10CF08001521142101E00746152101200022FDF713
:10CF18003CFD044698B33369284661685A68FFF7B0
:10CF280047FB804667B186894FF6C070FCF730FC36
:10CF380006401120FCF72CFC3043A8F80C0003E055
:10CF4800B268636812781A7523892E1D00932946E2
:10CF5800324620460623FCF7D6FC0021A8F810002C
:10CF680006228DE80600EB7A204629463246FCF771
:10CF78009FFE204602B0BDE8F041FDF7F3BC02B0C9
:10CF8800BDE8F0812DE9F04F4568048985B0064673
:10CF980028888A46FCF7FFFBC0F303200230B4EB75
:10CFA800800F0BDB2888FCF7F6FBC0F30320810019
:10CFB80049423046FDF7AAFC044628B1304605B080
:10CFC800BDE8F04FFDF7CEBC05F1100B51465846B1
:10CFD8007768FCF789FE80463888FCF7DCFB8146D9
:10CFE8007888FCF7D8FB442810D1B9F1430F38D121
:10CFF800DAF82030002B34D05B68002B31D05A6827
:10D00800002A7DD0E9688A422BD179E03D4A214641
:10D01800D2F800E00392734613B35A8A82421CD1B5
:10D02800B8F1000F01D11A683AB1D5F810C01A68E2
:10D03800624502D0B8F1000F0FD024B91A7C12F063
:10D04800040F08BF1C469A8A4A4506D15A68002A26
:10D058004FD0D5F80CC062454BD01946DB68DBE7EA
:10D068002CB92B69DAF804209A42A7D10024FB884E
:10D0780053B133893046009305F10C015A46112308
:10D08800FCF741FC002899D130466FF00701FDF705
:10D098003DFC002892D16CB1A769002F8ED0CDF845
:10D0A8000090E0692146324605F10C03B84705B007
:10D0B800BDE8F08FB8F1000F80D14FF070402C69B7
:10D0C800FCF7FAFB04404FF06040FCF7F5FB8442A4
:10D0D8003FF474AF2888FCF75EFBC0F30320811C83
:10D0E80089003046FDF712FC30460321FCF710FB9F
:10D0F80064E729B1DA68CA60039AC3F80CE01360E0
:10D108001C46B4E7886F002070B5134C00232568CF
:10D118002E4626B1B04208BF0123F668F9E701B1EF
:10D12800096801608AB929464FF4805269B147F607
:10D13800FF76B24207D04E8A964203BF013292B2BE
:10D148002946C968F2E7F52004E042820BB9C560B8
:10D158002060002040B270BD886F00202DE9FF4795
:10D168009246428A04460F469846DDF8309032B11E
:10D1780038460821FDF7CAFB38B93D4610E001469C
:10D18800FFF7C2FF0028F3D054E001200821002255
:10D19800FDF7FBFB0546002847D03946FDF7C7FCDD
:10D1A800608A6E68FCF7F4FA30804046FCF7F0FAC3
:10D1B8000023B371F3712368708013B909F104086F
:10D1C8000AE0D9F80420934205D0BD422FD0284662
:10D1D800FDF7C8FB2BE0A0462889FCF7D9FAB080F8
:10D1E800237CDB070ED42B89284600934146524600
:10D1F8001123FCF788FB08B1F08003E04FF0FF3300
:10D20800B371F371A27AE37A009211220192CDF8F8
:10D218000890284641465246FCF7DAFCBD420446CF
:10D2280007D02846FDF79EFB03E0FF2002E0F72029
:10D2380000E0204640B204B0BDE8F087F7B50746E5
:10D2480010460E4614461D46FCF7CCFB38B100903C
:10D258003146384622462B46FFF780FF00E0FC2087
:10D2680040B203B0F0BD021D838AFFF7E7BF70B577
:10D278001646428A04460D4612B13DB12D6805E0B6
:10D288000146FFF741FF0028F7D011E0237C6560D5
:10D2980043F004032374074BA6821A68104618B19A
:10D2A800844204D0C068FAE7E2601C6000E0002015
:10D2B80040B270BD886F0020044B1B684360002398
:10D2C8008382037C23F0040303747047C426030895
:10D2D8008161C2617047094A1368834209D1C368F2
:10D2E800136008E0DA681AB1824204BFC268DA60E3
:10D2F800DB68002BF6D1FDF757B800BF886F002018
:10D30800074B10B55888FDF761F9044628B100218C
:10D3180020221CF013FAFF23E372204610BD00BF41
:10D32800C82603082DE9F043894630B1374A1378F7
:10D3380002EB0312947B022C07D000250A24344AFE
:10D34800AC46AE46274626460FE00468526894422B
:10D35800F3D11BE012F8018CB8F1000F08D11C467C
:10D3680001350A2D02F110022AD00A2CEBB2F1D0B5
:10D3780012F8018CB8F1010F11D148B1D0F8008032
:10D3880052F80B1C884503D1204A1370D8B239E0F3
:10D3980092F80080F045E3D31E46C646E0E7B8F1B0
:10D3A800020FDDD128B1D0F8008052F80B1C884557
:10D3B800EAD092F80080E04524BF1F46C446CFE774
:10D3C80063B20A2B02D119F0010F1AD019F0020F1B
:10D3D80017D1092B01DCE3B206E00A2F01D0FBB21A
:10D3E80002E00A2E0DD0F3B208491A018C18002663
:10D3F800A67308B1006860600A440020D0730B70FF
:10D40800C4E7FF2040B2BDE8F08300BFAC2B00208A
:10D41800BB2B00202DE9F0410746154698460C46DF
:10D4280009B9F6202BE00B68002BFAD008463946DC
:10D43800FCF75AFC0028F4D14FF070402668FCF73E
:10D448003BFA06404FF06040FCF736FA8642E8D0D7
:10D4580020464146FFF766FF002810DB094B010113
:10D468005A180220907317611A460620431ED8B234
:10D478002E5C53181C1826720028F7D1D87340B2B6
:10D48800BDE8F081AC2B00200A4B03F1A000DA7A4A
:10D49800997A0132D2B20229DA7201D1EF2A02E076
:10D4A800012903D1012A84BF00229A7210338342D2
:10D4B800EDD17047B02B002070B508460221164602
:10D4C8001D46FFF72FFF00280BDB074904010B1946
:10D4D8009B7B022B05D1043121440B1D336029604D
:10D4E80000E0FF2040B270BDAC2B002010B568B141
:10D4F8004A684368D2F81A104B4081680B4005D13E
:10D50800BDE8104002F11A01063283E710BD2DE98B
:10D51800F743884616460546002867D05389292BC5
:10D5280061D954680120E789FCF732F987425AD15A
:10D5380040F20460678AFCF72BF9874253D14FF415
:10D548000060278AFCF724F987424CD140F6060090
:10D55800A789FCF71DF9874245D127466B6857F81C
:10D568001C0FD4F82610019004F11602284643B186
:10D57800994206D101A90123FFF74CFF4FF0010999
:10D5880005E001A90023FFF745FF4FF00009A08A35
:10D59800FCF7FEF8012806D0022824D1284601A964
:10D5A800FBF770FB1FE0B9F1000F1CD00220FCF75D
:10D5B800EFF83B68A082C4F826306B68E361062365
:10D5C800013BDBB2E218917D82F82010E15418F893
:10D5D8000310917518F803109171002BF0D1AB6905
:10D5E8002846314698473046FDF7BCF903B0BDE8F8
:10D5F800F083F8B5002206460F4603202A21FDF7DE
:10D60800C4F9054600283BD044680120FCF7C0F85F
:10D618000623A082013BDBB2F01890F82B20E1181A
:10D628008A75194A12F803E01A44927981F820E0C1
:10D63800E25490F82B208A71002BEBD173680120FB
:10D64800E3613B68C4F82630FCF7A2F8E0814FF4A8
:10D658000060FCF79DF8208240F20460FCF798F81F
:10D66800608240F60600FCF793F8B369A08129466A
:10D678003046984704462846FDF774F9204600E0EE
:10D68800FF2040B2F8BD00BFF82603082DE9F0419D
:10D6980005460E46084629461746FCF725FB08B1FD
:10D6A800F6204DE04FF070403468FCF705F904406F
:10D6B8004FF06040FCF700F98442F1D03368002B4A
:10D6C800EED030460121FFF72DFE002838DB1E4C36
:10D6D8004FEA001804EB08039A7B0C330AB90122BD
:10D6E8009A7004EB08039B7B012B00D037B92846BE
:10D6F8003146FFF77EFF034617B300E0FF2304EB34
:10D708000802927B022A1AD17E680623013BDBB20B
:10D7180004EB08021A44127AF254EA1892F82B1011
:10D72800F2189171002BF1D14FF40060FCF730F83A
:10D73800AB69B08139462846BDE8F041184718461C
:10D7480040B2BDE8F08100BFAC2B00202DE9F341C9
:10D7580004460E4608460E211546FDF7D7F8002860
:10D7680058D128462146FCF7BFFA8046C0BB4FF087
:10D7780070402F68FCF7A0F807404FF06040FCF7B6
:10D788009BF8874228681AD101238DF800305E2360
:10D798008DF802308DF80180FCF78EF8C0F3064052
:10D7A8008DF803002868FCF787F8000A8DF8040054
:10D7B8002868FCF781F86A468DF8050011E063686F
:10D7C800A2684340134203D0E3682BB304F10C056D
:10D7D80020462946324602B0BDE8F041FFF756BF61
:10D7E800104A75680623013BDBB2D15CE954E118A5
:10D7F80091F82B00E9188871002BF4D14FF40060E0
:10D80800FBF7C6FF3146A8812046A36902B0BDE8F0
:10D81800F0411847FE2000E0FC2040B202B0BDE80D
:10D82800F08100BFFE26030838B54368044698898E
:10D838000D46FBF7ADFFB0F5006F0AD040F60603C2
:10D84800984211D1284605F12B012246FFF75FFEC9
:10D858000DE020466FF00D01FDF758F820B920467D
:10D868002946FCF7E1F802E02046FDF77BF80020A6
:10D8780038BD00BF2DE9F0410123ADF5006D002250
:10D8880013F080010DF580664DF8223046F823200C
:10D8980018BF1B2183EA430301324B40B2F5807F56
:10D8A800DBB2EDD101230022674C13F0800144F86C
:10D8B800223018BF1B21013281EA43030A2ADBB256
:10D8C800F2D1632384F82830002384F88B310120B7
:10D8D80056F82030C3F1FF035DF823707D0045EA58
:10D8E800E715EDB2690041EAD511C9B24A0042EA2A
:10D8F800D112D2B287F0630753007D4043EAD213B6
:10D9080069404A40DBB25340504A8354234483F869
:10D9180028010130B0F5807FDAD1B06B746A756B7D
:10D92800F66A0022494F12F807E01EF0800F14BF74
:10D938001B23002383EA4E034FEA0E21DBB241EAA0
:10D948000E41594083EA0E0341EA036307F5007E5E
:10D958004EF8223007F5C06E4FEA33634EF8223096
:10D9680007F5206E4FEA33634EF8223007F5606EF4
:10D978004FEA336307F580774EF82230BB5C91009D
:10D98800D3B10DF5806757F823704FF0FF0E00EB09
:10D99800070C27449CFBFEF897FBFEFECEEB0E2EF1
:10D9A800CEEB0707C8EB08285DF82770C8EB0C0C0E
:10D9B8005DF82CC03F0201E09C461F468CEA070E2A
:10D9C80083B10DF5806757F823704FF0FF0C2F4493
:10D9D80097FBFCFCCCEB0C2CCCEB07075DF8277015
:10D9E8003F0400E01F468EEA07077BB10DF5806E05
:10D9F8005EF823304FF0FF0E334493FBFEFECEEB70
:10DA08000E2ECEEB03035DF823301B067B40104F30
:10DA18000132CB5107F5806E4FEA336341F80E307F
:10DA28004FEA336307F5006E41F80E3007F540679B
:10DA38004FEA3363B2F5807FCB517FF473AF0DF5B6
:10DA4800006DBDE8F08100BF502C0020782C00202C
:10DA5800783E0020F8B5854E0446B36B0F46154650
:10DA68001BB9FFF707FF0123B363C02D07D0B5F536
:10DA7800807F06D0802D40F0F5800A2302E00C2339
:10DA880000E00E23236004F1080363606D11002297
:10DA9800AA4210DA07EB820188784E78000440EA3F
:10DAA800062017F82260C978304340EA016043F83D
:10DAB80022000132ECE722680C2A38D00E2A75D0F1
:10DAC8000A2A40F0D1800026694DDC6855F82610F6
:10DAD8001A6801365140C4F307222A4492F82800F4
:10DAE80005EB146292F82820414081EA0241E2B233
:10DAF8002A4492F828200A2E81EA0261C4F30742D8
:10DB0800154495F8282003F1100381EA022253F8FE
:10DB18000C1C1A6082EA010253F8081C5A6082EA57
:10DB2800010284EA02049A60DC60CDD19CE0002501
:10DB38004F4C586954F825101A6801354A40C0F30B
:10DB48000721214491F82810082D82EA010204EBEC
:10DB5800106191F8281003F1180382EA0142C1B25A
:10DB6800214491F8281082EA0162C0F307410C446D
:10DB780094F8281082EA012253F8141C1A6082EAE9
:10DB8800010253F8101C5A6082EA010253F80C1C77
:10DB98009A6082EA010253F8081CDA6082EA0102FC
:10DBA80080EA02001A615861C2D15DE00025304E5A
:10DBB800DC6956F825101A6801355140C4F307226C
:10DBC800324492F8280006EB146292F8282041406B
:10DBD80081EA0241E2B2324492F82820986881EA48
:10DBE8000261C4F30742324492F82820072D81EAE3
:10DBF80002215A68196281EA0201DA68596281EAE7
:10DC0800000182EA01029962D1B2DA62314491F8E4
:10DC18002800196903F1200381EA000106EB12606C
:10DC280090F8280081EA0061C2F307203044C2F36B
:10DC3800074290F82800324492F8282081EA00210F
:10DC480081EA024253F80C1C1A6182EA010253F875
:10DC5800081C5A6182EA010284EA02049A61DC61C2
:10DC6800A5D101E00348F8BD0020F8BD404E0020D2
:10DC7800502C002000F8FFFFF0B5C02AC7B00446BA
:10DC880006D0B2F5807F05D0802A65D10A2302E04C
:10DC98000C2300E00E23236004F108036360684648
:10DCA800FFF7D8FE002858D1009A019912018B1865
:10DCB8008A5804F11805A2605A68E2609A682261DD
:10DCC800DA6862612468013C002CA3F1100333DD9B
:10DCD800002653F8262022485FFA82FE00EB1267DE
:10DCE800864420499EF828C097F8287001EB8C0CD0
:10DCF80001EB8707D7F830EDDCF830718EEA070EB4
:10DD0800C2F307270744C2F3074297F82870024472
:10DD180092F8282001EB8707D7F8307501EB8201CC
:10DD2800D1F830298EEA07077A4045F826200136CF
:10DD3800042ECED11035C6E71A6868462A605A689C
:10DD480000216A609A68AA60DB684FF48C72EB6005
:10DD58001BF0F4FC002000E0034847B0F0BD00BF12
:10DD6800502C0020483D002000F8FFFF2DE9F04727
:10DD78009578547816782D04D0F804C045EA04251F
:10DD8800D478354345EA0464DCF800509779654057
:10DD9800547916793F0447EA0427D479374347EA88
:10DDA8000464DCF80470567A6740947A92F808E0C4
:10DDB800240444EA0624D67A44EA0E0444EA0666B1
:10DDC800DCF8084092F80DE07440967B360446EA89
:10DDD8000E2692F80CE0D27B46EA0E0646EA02626C
:10DDE800DCF80C600CF1100E564002684FEA62082D
:10DDF80008F1FF38002940F0F3817146B8F1000FAF
:10DE08008E46F54A01F120014FEA176040F3FD8084
:10DE18005FFA85FE02EB800002EB8E0ED0F830CD63
:10DE2800DEF83001C4F3074E8CEA000C51F8200CE0
:10DE380002EB8E0E8CEA000CC6F3072002EB800082
:10DE4800D0F830055FFA87F98CEA0000DEF830C9AF
:10DE580002EB890980EA0C0C200E02EB8000D0F856
:10DE680030EDD9F830015FFA84FA8EEA000E51F8E5
:10DE78001C0C02EB8A0A8EEA000EC5F3072002EB9F
:10DE88008000D0F83005C4F307248EEA0000C6F3FA
:10DE9800074E02EB8E0EDEF830E902EB840480EACE
:10DEA8000E0E300E02EB8000D0F8309DDAF830010B
:10DEB800F6B289EA000951F8180CD4F8304589EA15
:10DEC8000009C7F3072002EB8000D0F83005C7F33C
:10DED800074789EA0000C5F3074902EB8909D9F821
:10DEE80030992D0E80EA090002EB850502EB8609C0
:10DEF800D5F8306DD9F8305102EB87076E4051F8EC
:10DF0800145C4FEA106975406540D7F830695FFACC
:10DF18008CF44FEA1E6702EB840402EB87076E401D
:10DF2800D4F83051D7F8304D02EB8909654051F8E3
:10DF3800104C4FEA166A6C40C6F3072502EB8505BC
:10DF4800D5F83075C0F3074502EB8505D5F830598B
:10DF58007C4065405FFA8EF402EB8404D4F830719B
:10DF6800D9F8304D02EB8A0A674051F80C4C08F199
:10DF7800FF387C40CCF3072702EB8707D7F83075CA
:10DF88007C40C6F3074702EB8707D7F83079F6B22B
:10DF98006740C4B202EB8404D4F83091DAF8304D0B
:10DFA80002EB860689EA040951F8084CC0F30720F9
:10DFB80089EA0409CEF3072402EB8404D4F8304537
:10DFC80002EB800089EA0404CCF3074902EB8909D3
:10DFD800D9F830994FEA1C6C02EB8C0C84EA0904DE
:10DFE800D6F83091DCF8306DCEF3074E89EA060C8E
:10DFF80051F8046CD0F8300502EB8E028CEA060664
:10E00800D2F8302946405640F8E6E9B202EB8101E1
:10E0180002EB8000D1F830C1D0F8301DC4F30740BE
:10E028008CEA010CDEF8001002EB80008CEA010C8F
:10E03800C6F3072102EB8101D1F83015D0F8300979
:10E048008CEA010181EA000C4FEA1468F9B202EB8C
:10E05800810102EB8808D1F83001D8F8301D4FEA69
:10E0680016694840DEF8041002EB89094140C5F3FF
:10E07800072002EB8000D0F830054140C6F3074086
:10E0880002EB8000D0F83009F6B24840E1B202EB6A
:10E098008101D1F83081D9F8301D02EB860688EA73
:10E0A8000108DEF80810C4F3072488EA0108C7F35A
:10E0B800072102EB8101D1F8301502EB840488EACC
:10E0C8000101C5F3074802EB8808D8F830892D0EFE
:10E0D80002EB850981EA0808D6F83051D9F8301DD5
:10E0E800C7F307476940DEF80C5002EB87024D4042
:10E0F800D4F83015D2F83029384F4D4055405FFAE2
:10E108008CF23A4492F82841DEF8102007EB1061AF
:10E11800624091F82841C5F30721394482EA046234
:10E1280091F82841C8F30741394482EA042291F85A
:10E138002841DEF8141082EA0444C2B23A4492F844
:10E148002821514007EB186292F8282181EA0261E0
:10E15800CCF307223A4492F8282181EA0221C5F338
:10E1680007423A4492F8282181EA02415FFA88F28C
:10E178003A4492F82861DEF81820C8F3072872405C
:10E1880007EB156696F82861B84482EA0662C0F380
:10E1980007263E4496F82861C0F3074082EA062223
:10E1A800CCF307463E4496F8286107EB1C6C82EADC
:10E1B8000646EAB23A4492F82851DEF81C20074491
:10E1C8006A409CF8285197F8280182EA056298F875
:10E1D800285182EA0522ECE1483D0020502C00201D
:10E1E8007146B8F1000F8E464FEA176901F1200118
:10E1F8005FFA85FC4FEA16627B4840F3F78000EB34
:10E20800820200EB8C0CD2F828EEDCF828225FFAA8
:10E2180087FA8EEA020E51F8202C00EB8A0A8EEA61
:10E22800020EC7F3072200EB8202D2F8282600EB81
:10E2380089098EEA0202C4F3074E00EB8E0EDEF85F
:10E2480028EAD9F8289E82EA0E0E2A0E00EB8202EE
:10E25800D2F828CEDAF828225FFA84FA8CEA020C7F
:10E2680051F81C2C00EB8A0A8CEA020CC4F3072232
:10E2780000EB8202D2F82826240E8CEA0202C6F3AA
:10E28800074C00EB8C0CDCF828CA00EB840482EA0B
:10E298000C0CDAF82822D4F8284E89EA020951F839
:10E2A800182CC7F3074789EA0209C6F3072200EBCF
:10E2B8008202D2F82826F6B289EA0202C5F3074993
:10E2C80000EB8909D9F8289A00EB860682EA090941
:10E2D800D6F82822C5F30725624000EB850551F8DA
:10E2E800144CD5F8285600EB87075440D7F8282A4D
:10E2F8006C406240160E5FFA8EF400EB840400EB6B
:10E308008606D4F82852D6F8284E5FFA8CF66C4068
:10E3180051F8105C00EB86066540CCF3072400EB4F
:10E328008404D4F82846D6F828626540C9F307441F
:10E3380000EB8404D4F8284A4FEA1C6A65404FEA87
:10E348001E6400EB8404D4F8284E00EB8A0A86EA9F
:10E358000407C9F3072451F80C6C00EB8404D4F8C3
:10E3680028467E406640C2F3074400EB8404D4F894
:10E37800287A5FFA89F400EB84047740D4F828629D
:10E38800DAF8284E4FEA1969664051F8084C00EB54
:10E3980089097440C2F3072600EB8606D6F828667A
:10E3A800D2B27440CEF3074600EB8606D6F8286A48
:10E3B80000EB82027440D2F82862D9F8282ECEF3F6
:10E3C800072E724051F8046C00EB8E0E5640CCF3C9
:10E3D800074CDEF8282600EB8C005640D0F8282A97
:10E3E80008F1FF385640FCE6502C002000EB8C0C5E
:10E3F80000EB8202DCF82812D2F8282E00EB8909FB
:10E4080081EA020CC7F30721DEF8002000EB810146
:10E41800D1F828168CEA02024A40C4F3074100EBFF
:10E428008101D1F8281A82EA010CFAB2290E00EB10
:10E43800820200EB8101D2F82882D1F8282EC4F399
:10E44800072188EA020800EB8101DEF80420D1F8F0
:10E45800281688EA02024A40C6F3074100EB810108
:10E46800D1F8281AC7F3074782EA0108E2B200EB9D
:10E478008202D2F82812D9F8282E240E81EA02093D
:10E48800C6F30722DEF8081000EB8202D2F828262D
:10E4980089EA01015140C5F3074200EB8202D2F834
:10E4A800282AF6B200EB860600EB840481EA02090A
:10E4B800D4F8282ED6F82812C5F307255140DEF8DF
:10E4C8000C2000EB85054A4000EB8707D5F8281695
:10E4D800D7F8285A4A4055405FFA8CF2024492F81D
:10E4E8002840DEF8102000EB1561624091F82840C2
:10E4F800C8F30721014482EA046291F82840C9F36D
:10E508000741014482EA042291F82840DEF81410F9
:10E5180082EA04445FFA88F2024492F828205140C3
:10E5280000EB1C6292F8282081EA0261C9F30722F5
:10E53800024492F8282081EA0221C5F307420244E6
:10E5480092F8282081EA02415FFA89F2024492F89F
:10E558002860DEF8182000EB1969724000EB186695
:10E5680096F82860C8F3074882EA0662C5F30726CA
:10E57800064496F8286082EA0622CCF30746064449
:10E5880096F82860CCF3072C82EA0646EAB20244E1
:10E5980092F82850DEF81C2084446A4099F82850E4
:10E5A800404482EA05629CF8285090F8280082EAE4
:10E5B800052282EA0042200A5870200C9870080A46
:10E5C80019715871080C090ED971310A5972310C38
:10E5D8009972110A1C701E72240E360E1A73597322
:10E5E800110C120E9871DC70DE729973DA730020C8
:10E5F800BDE8F0872DE9F04F994685B013078046AE
:10E608008A4615460E9F0F9E93465CD100294FD12E
:10E618003A46AB1A3B44002B53DD1346EE46EA4616
:10E6280002F11004F446186859680833ACE803008E
:10E63800A342E646F6D1002133464046FFF796FB53
:10E64800731E09F1FF3106F10F0013F8012F11F8BD
:10E6580001EF83428EEA02021A70F6D15246CE4684
:10E668000DF1100C134603CB6345CEF80000CEF82D
:10E6780004101A460EF1080EF4D122461036C8E7E7
:10E6880019F80300CA5C4240E2540133102BF7D159
:10E698002246234640465146FFF768FB4B4604F1A5
:10E6A800100254F8041B944243F8041BF9D1103D9E
:10E6B800C5EB0B04002D07EB0401344401DD0023F6
:10E6C800DEE7002000E0024805B0BDE8F08F00BF9B
:10E6D800F0F7FFFF2DE9F04708ADE0CD82469846F8
:10E6E8001C6806EB020991B1013F24E02CB95046A1
:10E6F80001212A462B46FFF739FB2B5D16F8012B23
:10E70800534007F8013B2A55013404F00F044E45E5
:10E71800ECD112E02CB9504601212A462B46FFF7CE
:10E7280025FB2A5D16F8013B534007F8013F2B559E
:10E73800013404F00F044E45ECD1C8F80040002025
:10E74800BDE8F0872DE9F04FEFB00546002110A88D
:10E7580020221AF0F3FF0026771006F0010907F1CE
:10E76800020855B19F4BA04AA0484FEA8811B9F159
:10E77800000F18BF1A461BF047F818AC00211022EA
:10E7880020461AF0DBFF28A810A94FEA8812B9F131
:10E79800000F1BD1FFF770FA42F2107828A8002169
:10E7A80022462346FFF7E2FAB8F10108F6D12046DF
:10E7B8008F4901EB071110221AF02AFFB0B1002D82
:10E7C80000F00A818B481BF06BF805E1FFF742F96E
:10E7D80042F2107828A8012122462346FFF7C6FAFC
:10E7E800B8F10108F6D120468349E2E715B183481C
:10E7F8001BF056F80136062EAED115B10A201BF0D3
:10E8080017F84FF000094FEA690A09F001070AF101
:10E81800020645B1734B744A7948B101002F18BFFD
:10E828001A461AF0F1FF0DF1200800211022404687
:10E838001AF084FF0021102204A81AF07FFF00219B
:10E84800102220461AF07AFF28A810A9B20187B929
:10E85800FFF712FA42F210760094019428A80021DA
:10E8680010224346FFF7C6FE013EF5D12046654912
:10E878001EE0FFF7EFF842F2107B0121102208ABEF
:10E888000CAF04AE0094019428A8FFF7B3FE96E8F5
:10E898000F0087E80F0094E80F00BBF1010B86E832
:10E8A8000F0097E80F0084E80F00E6D1304656497C
:10E8B80001EB0A1110221AF0ABFE00287FF47FAF9B
:10E8C80015B14E481AF0ECFF09F10109B9F1060F2C
:10E8D80099D115B10A201AF0ABFF00274FEA670952
:10E8E80007F0010A5DB13F4B3F4A09F10201474871
:10E8F8008901BAF1000F18BF1A461AF085FF444B78
:10E9080008AE03F1100E324618685968083303C27E
:10E9180073451646F7D1364E09F1020B06F1D001C0
:10E9280001EB49114FEACB0210A817F00BFD0023A9
:10E9380028A810A94FEA8B120C93FFF78BF8BAF1AD
:10E94800000F1BD1A64606EB891606F5987306F547
:10E95800B876724618685968083303C2B3429646B7
:10E96800F7D108AB8DE818000021029428A84022AE
:10E978000CABFFF7AFFE204626491AE0A64606F57F
:10E98800F87306F50C76724618685968083303C29E
:10E99800B3429646F7D10121CDF800800194029444
:10E9A80028A840220CABFFF795FE20461A4901EB38
:10E9B800891140221AF02CFE00287FF400AF15B10F
:10E9C8000E481AF06DFF0137062F87D135B10A209E
:10E9D8001AF02EFF002002E0012000E028466FB068
:10E9E800BDE8F08FC2830308BE830308C68303080B
:10E9F800042703083D9C030834270308DB83030826
:10EA0800E28303086427030894270308F7830308AD
:10EA1800C4270308F4280308342803080023F0B5A2
:10EA28000360436000F10806F3540133B3F5807FB7
:10EA3800FAD100231C46C51D00F207109342A8BF57
:10EA4800002315F801EFCF5C74443C44E4B2375D11
:10EA580085422F7003F1010306F804E0EED1F0BD02
:10EA6800F0B50568446800F1080E00278F4215DAF2
:10EA78000135EDB21EF805603444E4B21EF804C056
:10EA88000EF805C00EF804606644F6B21EF806C01B
:10EA9800D65D8CEA0606DE550137E7E70560446077
:10EAA8000020F0BDF0B50646C7B0002401271EB10E
:10EAB8001B4839461AF0A8FE6B461A4D2A191068E9
:10EAC8005168082203C305F1180104A82144FFF77F
:10EAD800A5FF08210DEB01036A4604A8FFF7C0FF54
:10EAE80005F1300102A8214408221AF091FD0546DB
:10EAF80020B18EB10C481AF0D3FE0DE016B10B48C8
:10EB08001AF0CEFE0834182C07F10107CFD126B130
:10EB18000A201AF08DFE00E00125284647B0F0BD16
:10EB28000F840308342903083D9C0308DB8303088A
:10EB38002DE9F043002B7ED0DE00062496FBF4F48A
:10EB48006FF0050505FB0465022D03D0042D02D1E5
:10EB5800023400E003340D68AC4204DB01340C607D
:10EB68001020BDE8F083032693FBF6F6074606EB74
:10EB780046060024B4423D46964607F1040702F1D2
:10EB8800030229DA12F803ECDFF8B0804FEAAE0985
:10EB980012F8025C18F809900EF0030E12F801CC76
:10EBA80008EB0E1E07F8049C4FEA25191EF809E029
:10EBB80005F00F0507F803EC08EB85054FEAAC1ED6
:10EBC80015F80E500CF03F0C07F8025C18F80C50C2
:10EBD800033407F8015CCDE79C422A4627DA9EF801
:10EBE800002001349C42154FB8BF9EF801604FEADF
:10EBF800A20E17F80EE0A8BF002602F0030285F85F
:10EC080000E007EB02124FEA261E9C4212F80E2083
:10EC1800B8BF06F00F066A70B8BF17F8262005F1CE
:10EC28000303A8BF3D223D24AA705A1C1C70101A69
:10EC38000023086013701846BDE8F0837C29030898
:10EC48002DE9F04100241646A64627469F4225DABC
:10EC5800DD1B012D05DD35780D2D02D175780A2DC6
:10EC680019D035780A2D16D03D2D04D10EF1010E9C
:10EC7800BEF1020F60DC15F0800F5DD1DFF8C0C077
:10EC8800654495F840507F2D56D03F2D02D8BEF1EF
:10EC9800000F51D1013401370136D7E7002C48D095
:10ECA80006256C430B680734E410A34206DB0026F4
:10ECB80002F1FF3C03463446032508E00C601020AF
:10ECC800BDE8F0811CF801EFBEF10D0F08D107F186
:10ECD800FF3ECCEB0E0E9644BEF1000FF2DC26E0B0
:10ECE800BEF10A0FF3D0DFF858800134C6449EF80D
:10ECF80040E0BEF1400F08BF013D0EF03F0E042C6E
:10ED08004EEA8616E3D1002D0FDD340C012D1C7060
:10ED180001D1013309E0340A032D5C7003D00233BA
:10ED280000240225D3E79E7003330024CFE7181A86
:10ED380008600020BDE8F0811220BDE8F08100BF26
:10ED48007C29030830B50546A3B010B11A481AF05B
:10ED58005BFD8023019302A801A9184A4023FFF70D
:10ED6800E7FE28B9164802A958221AF051FC20B12A
:10ED7800F5B114481AF094FD1AE015B112481AF0CA
:10ED880043FD8023019302A801A90D4A5823FFF7E8
:10ED980057FF0028ECD1094802A940221AF038FC94
:10EDA80004460028E4D125B108481AF079FD00E0AE
:10EDB8000124204623B030BD218403083C2A0308DF
:10EDC8007C2A03083D9C03083A8403085A840308F4
:10EDD800A2F1300310B5DCB2092C88BFFF23036011
:10EDE800A2F14103052B9CBFA2F137030360A2F1F6
:10EDF8006103052B9CBF573A0260006888422CBF0C
:10EE08000620002010BD0023F0B516461D46854299
:10EE180016DAD6F800E0C3EB0E04346051F825701A
:10EE28000135BC422CBF4FF0000C4FF0010CE41B25
:10EE38009E452CBF63460CF1010346F8044BE6E7F8
:10EE480020EAE07002EB800243B11168C81A9942C7
:10EE580042F8040B2CBF00230123F5E7F0BDF0B501
:10EE6800864687B001930023039102920593BEF171
:10EE78000F0F40F3CA8003980299059A019B50F836
:10EE8800044B4FF000050E68E3FB0425B71845F165
:10EE9800000241F8047B50F8044B4FF000050E685F
:10EEA800E3FB0425B71845F1000241F8047B50F84C
:10EEB800044B4FF000050E68E3FB0425B71845F135
:10EEC800000241F8047B50F8044B4FF000050E682F
:10EED800E3FB0425B71845F1000241F8047B50F81C
:10EEE800044B4FF000050E68E3FB0425B71845F105
:10EEF800000241F8047B50F8044B4FF000050E68FF
:10EF0800E3FB0425B71845F1000241F8047B50F8EB
:10EF1800044B4FF000050E68E3FB0425B71845F1D4
:10EF2800000241F8047B50F8044B4FF000050E68CE
:10EF3800E3FB0425B71845F1000241F8047B50F8BB
:10EF4800044B4FF000050E68E3FB0425B71845F1A4
:10EF5800000241F8047B50F8044B4FF000050E689E
:10EF6800E3FB0425B71845F1000241F8047B50F88B
:10EF7800044B4FF000050E68E3FB0425B71845F174
:10EF8800000241F8047B50F8044B4FF000050E686E
:10EF9800E3FB0425B71845F1000241F8047B50F85B
:10EFA800044B4FF000050E68E3FB0425B71845F144
:10EFB800000241F8047B50F8044B4FF000050E683E
:10EFC800E3FB0425B71845F1000241F8047B50F82B
:10EFD800044B4FF000050E68E3FB0425B71845F114
:10EFE800000241F8047B50F8044B4FF000050E680E
:10EFF800E3FB0425B71845F1000241F8047B0592AC
:10F0080002910390AEF1100E31E7BEF1070F69DDF2
:10F0180003980299059A019B50F8044B4FF000059C
:10F028000E68E3FB0425B71845F1000241F8047B9C
:10F0380050F8044B4FF000050E68E3FB0425B718A1
:10F0480045F1000241F8047B50F8044B4FF00005ED
:10F058000E68E3FB0425B71845F1000241F8047B6C
:10F0680050F8044B4FF000050E68E3FB0425B71871
:10F0780045F1000241F8047B50F8044B4FF00005BD
:10F088000E68E3FB0425B71845F1000241F8047B3C
:10F0980050F8044B4FF000050E68E3FB0425B71841
:10F0A80045F1000241F8047B50F8044B4FF000058D
:10F0B8000E68E3FB0425B71845F1000241F8047B0C
:10F0C80050F8044B4FF000050E68E3FB0425B71811
:10F0D80045F1000241F8047B059202910390AEF1DC
:10F0E800080E92E7BEF1000F15DD03980299059A04
:10F0F800019B50F8044B4FF000050E68E3FB042514
:10F10800B71845F1000241F8047B0592029103907B
:10F118000EF1FF3EE6E7029A1168059B0B4442F8A0
:10F12800043B05998B422CBF002301230593002B38
:10F13800F2D107B0F0BD0FB482B002AA52F8043B76
:10F14800019202AA3BB1012119600021996059601E
:10F1580052F8043FF6E702B004B070470FB413B595
:10F1680004AB53F8044B01939CB1A06838B16268B2
:10F17800002192001AF0E2FAA06819F075FF012345
:10F18800236000236360A360019B1A1D01921C6821
:10F19800EAE702B0BDE8104004B070472DE9F0413D
:10F1A800456804468D420E461CDA8F00384619F031
:10F1B80053FF8046C8B13A4600211AF0BFFAA76843
:10F1C8006FB1AD0039462A46404617F0BBF83846BD
:10F1D80000212A461AF0B2FAA06819F045FF6660C5
:10F1E800C4F808800020BDE8F0810120BDE8F08166
:10F1F8008842F8B506460F461FD0496801398B008A
:10F20800002903DDBA68D258043BA2B13B684C1C04
:10F21800336030462146FFF7C1FF054678B972686A
:10F228002946B06892001AF089FAB068B968A20055
:10F2380017F088F803E00139E2E70020F8BD284616
:10F24800F8BD1FB503460A460068596801AC03C4F7
:10F2580011689868196051682060596091689960D0
:10F2680001AB03CB106018685160906004B010BD0A
:10F2780070B50E4601210446FFF790FF054688B990
:10F288006268A068920029461AF058FAA36886EACC
:10F29800E672002EA2EBE6721A60B4BF4FF0FF339D
:10F2A80001232360284670BD0023194670B54568C0
:10F2B800A94210DA826852F82140002224FA02F6A4
:10F2C800F60706D40132202A03F10103F6D10131F1
:10F2D800EEE7184670BD002070BD10B54368013BCD
:10F2E8009A00002B816802DD8C58043A1CB151F851
:10F2F80023201F2004E0013BF3E710F1FF3003D384
:10F3080022FA00F1C907F8D500EB4310013010BD0F
:10F3180008B5FFF7E2FF0730C01008BDF8B506468C
:10F328000D4617460024BC4201DA2B5D53B13B1B46
:10F338000333042193FBF1F13046FFF72FFF014619
:10F34800E8B901E00134EEE73046FFF791FF0146E6
:10F35800A8B97A1E9446A242C2EB0C030FDBAF5C3D
:10F368004FEAA30EB06803F00303DB0007FA03F3C8
:10F3780050F82E70013A3B4340F82E30EBE7084630
:10F38800F8BDF8B5144605460F46FFF7C1FF84429D
:10F39800064617DB2246384600211AF0CFF93C44CE
:10F3A8000023F21A002A0BDDAA68981003F0030163
:10F3B80052F82020C900CA4004F8012D0133F0E7B3
:10F3C8000020F8BD0820F8BD2DE9F04106464FF0B1
:10F3D80020080C4691FBF8F501F01F07FFF77DFFA9
:10F3E80073682044B0EB431F02DC002D0DDC0AE0FB
:10F3F80000F11F0191FBF8F13046FFF7CFFE00281E
:10F40800F3D0BDE8F081E7B918E06FF00301694374
:10F418007268531E9200AB42A2F1040205DBB06889
:10F42800013B841864588450F5E79A00002BEADB06
:10F43800B16800208850013B043AF7E70020BDE896
:10F44800F081D6F804C0AB0000206545F6DAD6F89E
:10F4580008E0C7F120025EF80340013504FA07F11D
:10F4680001434EF8031024FA02F00433EDE7F0B537
:10F47800202491FBF4F4002C01F01F0105DC79B382
:10F48800436800265A1E9B0017E0456800222B1B84
:10F498009A4207DA8668171956F8277046F82270D4
:10F4A8000132F5E723EAE3739A00AB42E7DA8468AE
:10F4B8000026A65001330432F7E7002AA3F104031B
:10F4C8000EDBD0F808E0C1F120045EF80370013AC1
:10F4D80027FA01F535434EF8035007FA04F6ECE72E
:10F4E8000020F0BDF0B54368013B9A00002B03DB18
:10F4F8008468A458043A24B14A681C46013A950025
:10F5080006E0013BF2E78E687759043D1FB9013ADE
:10F51800002AF8DA19E0002B02DA4FF0FF30F0BDCC
:10F52800934210DC9A42F8DC9B00002C09DB8268CD
:10F53800D158F258914206D8A3F10403EDD3013C07
:10F54800F3E70020F0BD0120F0BDD843C00FF0BDA7
:10F558002DE9F04F8B46914687B0109F80467A6818
:10F56800B8680021920004931AF0E8F8BB68D9F84B
:10F5780004400193DBF80430019DA342A8BF234651
:10F588000293631C9B0003934FF0000AA245D8F82E
:10F59800080021DADBF8081050F82AC00B682E683A
:10F5A8002A4603FB0C66049B02985E436346CDF82B
:10F5B80014C0FFF754FC2A4633462046D9F80810F1
:10F5C800FFF74DFCDDF814C0039A45F804CB00237F
:10F5D800AB500AF1010AD9E7019B621C24EAE471E5
:10F5E800920003EB810116F0ADFE49464046FFF755
:10F5F80079FF00282046A7BFD9F80810D8F80820B6
:10F60800D8F80810BA6807B0BDE8F04FFFF7FBBBA1
:10F61800F0B54368013B9A00002B03DB8468A458CB
:10F62800043A24B14A681D46013A940006E0013BB9
:10F63800F2E78E683759043C1FB9013A002AF8DA14
:10F6480026E0002B046801DA624224E0934201DDDF
:10F65800026820E09A42F7DC221E096801DD0029D1
:10F6680014DB002901DC9B000DE0002CFBDA4FF0D5
:10F67800FF3210E08168CF58F1588F420BD8A3F1C0
:10F688000403E1D3013D002DF4DA03E0012202E096
:10F69800002BDDDA00221046F0BD1FB581EAE173C8
:10F6A800A3EBE17300290093B4BF4FF0FF330123AC
:10F6B800019301A901230293CDF80CD0FFF7A8FF0D
:10F6C80005B05DF804FB90422DE9F0410446174669
:10F6D80006D0884205D0FFF78BFD064608B14AE000
:10F6E8000F467D680123013D2360AB00002D03DB3D
:10F6F800BA68D258043B62B12046691CFFF74EFD38
:10F708000646002837D1D7F808E0A368074601461F
:10F7180001E0013DEAE7A94213DC186801313844E9
:10F728001860DEF80020024443F8042B5EF804CB8E
:10F7380062452CBF00220122B8422CBF1746571C35
:10F74800E9E74FEA8108B7B162684D1C914206DBD0
:10F7580020462946FFF722FD60B9A36843441A688A
:10F7680029463A44BA421A602CBF0027012708F1FB
:10F778000408E8E706463046BDE8F081F0B50546DE
:10F7880085B008460F4611461646FFF7ABFE00281F
:10F798002EDB01A80021FFF7CEFCB54206D101A857
:10F7A8002946FFF725FD0446E0B901AEBD4205D163
:10F7B8007068012301382B6083000BE02846394626
:10F7C800FFF716FD044668B9F2E7B268D258043B61
:10F7D80012B901380028F8DA0130B168AA68FFF7D1
:10F7E80012FB002401A80021FFF7B8FC204600E026
:10F7F8000A2005B0F0BDF8B50C68136805466343E8
:10F808000E46174612D508461146FFF76BFE00282C
:10F81800284604DB31463A46FFF7B0FF08E0394690
:10F828003246FFF7ABFF28B9644202E0FFF74BFF0F
:10F8380000B92C60F8BDF8B50C6813680546634339
:10F84800002B0E46174612DD08461146FFF74AFE02
:10F858000028284604DB31463A46FFF78FFF08E0C8
:10F8680039463246FFF78AFF28B9644202E0FFF7BB
:10F878002AFF00B92C60F8BD1FB582EAE273A3EB3A
:10F88800E273002A0093B4BF4FF0FF3301230193C2
:10F8980001AA01230293CDF80CD0FFF7ACFF05B005
:10F8A8005DF804FB1FB582EAE273A3EBE273002A5A
:10F8B8000093B4BF4FF0FF330123019301AA012342
:10F8C8000293CDF80CD0FFF7B6FF05B05DF804FB46
:10F8D8002DE9F0470646884686B01746684603A9CC
:10F8E8000022FFF728FC464507D168463146FFF756
:10F8F8007FFC8246002847D1E846BE4207D103A8CC
:10F908003146FFF775FC824600283DD103AFD8F891
:10F918000450013DAB00002D04DBD8F80820D25874
:10F92800043B1AB17C68013CA30006E0013DF2E704
:10F93800BA68D258043B12B9013C002CF8DA2919EC
:10F9480030460231FFF72AFCA1468246E0B951460B
:10F958003046FFF78DFC8246B0B90135A400B9F1F5
:10F96800000F0CDBB268BB6822441B592846D8F844
:10F978000810FFF774FA09F1FF39043CEFE7D8F8EB
:10F9880000203B685343336003A869460022FFF711
:10F99800E5FB504606B0BDE8F0871FB5012300928D
:10F9A80001AA01930293CDF80CD0FFF791FF05B09F
:10F9B8005DF804FB2DE9F0438B1E0E2B85B006463F
:10F9C800894690467AD801A80021FFF7B4FB404643
:10F9D8001AF038FAB9F1100F054636D183001F33F3
:10F9E8002021304693FBF1F1FFF7D8FB04460028AD
:10F9F8005ED121463046FFF73BFC0446002857D12C
:10FA0800013DA946002DC5EB090727DB07D198F86A
:10FA180000302D2B03D14FF0FF33336048E06846A8
:10FA2800102118F80520FFF7D3F900283FD1B26854
:10FA3800F810009B07F0070752F82010BF00BB40E2
:10FA48000B4342F82030013DDCE730460021FFF748
:10FA58000FFC044660BB0746AF4201DB002427E0E9
:10FA68003FB998F800302D2B03D14FF0FF333360A6
:10FA78001BE06846494618F80720FFF7A9F904462D
:10FA8800B0B901A831464A46FFF787FF044678B95E
:10FA980033683046012B01A9009A02D1FFF7ECFE2A
:10FAA80001E0FFF7FFFE044610B90137D4E704462A
:10FAB80001A80021FFF752FB204600E0042005B012
:10FAC800BDE8F0832DE9F0411446ADF5816D02AD36
:10FAD8004FF4806280460E462846002119F02EFE1B
:10FAE800284640F2FF31224618F060FB18B328463A
:10FAF8001AF0A8F9431EEA5C0A2A02BF1846002237
:10FB0800EA54431EEA5C0D2A02BF18460022EA5452
:10FB18002C18671EAF4206D301A8314614F8012CF1
:10FB2800FFF756F928B1404631462246FFF742FF13
:10FB380002E03C46EDE702200DF5816DBDE8F0815D
:10FB48002DE9F04F82469BB00F461846002191469A
:10FB58000693FFF7A2FD002800F0A281002417AD4C
:10FB68000BA80EA911AA14AB00950194FFF7E3FAAC
:10FB780048460699FFF7B6FCA04217DABAF1000F1B
:10FB880001D14FB910E021465046FFF771FB0446FA
:10FB9800002840F07981F4E738464946FFF728FB0A
:10FBA8000446002840F0708100207AE10BA84946FD
:10FBB800FFF71EFB0446002840F066810EA8069950
:10FBC800FFF716FB0446002840F05E81D9F80410C0
:10FBD800012311A802310E930B93FFF7DFFA0446B5
:10FBE800002840F05181214611A8FFF741FB044647
:10FBF800002840F0498114A80221FFF7CFFA0446F3
:10FC0800002840F0418128460321FFF7C7FA04463F
:10FC1800002840F039810EA8FFF75FFBA24B034094
:10FC2800002BBEBF03F1FF3363F01F0301331F2B0B
:10FC380011D0C3F11F030BA819460393FFF7C4FBA8
:10FC4800002840F020810EA80399FFF7BDFB00288B
:10FC580040F0198101E0002303930F9B0C9E05934C
:10FC680006F1FF38013BC3EB08054FEA451B0EA818
:10FC780059460493FFF7A8FBAD000BA80EA9FFF7A0
:10FC8800C7FC002809DB13990BA84A5901324A51CD
:10FC980001460EAAFFF7CFFDEFE70EA85946FFF77A
:10FCA800E6FB049B06F180469B000793043B0993FF
:10FCB800059B023EC3F1010508EB050303F18045EE
:10FCC800013B013D5B01AD000593B600049B9845DF
:10FCD80040F3B5800D9B10990798321D089208587B
:10FCE8009A58824204D3139B4FF0FF325A5129E0AD
:10FCF8004FEA104BB2FBFBFE0BFB1E229B591FFA6F
:10FD080080FC190C41EA02420CFB0EF18A4204D233
:10FD1800024482420EF1FF3EF8D2521AB2FBFBF1C6
:10FD28000BFB11220CFB01FC9BB243EA0242624529
:10FD380004D20244824201F1FF31F8D2139B41EA16
:10FD48000E415951139AA6F1040B535901335351DB
:10FD5800139A14A853590021013B5351FFF788FA0D
:10FD6800002840F09080049A169B002AC8BF099981
:10FD7800109AC8BF505807991860525814A85A606A
:10FD8800139B01465A59FFF708FE0146002878D10F
:10FD980017A8FFF76DFA002875D1B8F1010FC8BF91
:10FDA8000D9A199BC8BF52F80B000D9A1860B8F14C
:10FDB800000FCCBF915900215960089914A85258D6
:10FDC80017A99A60FFF724FC0028C1DC139B14A82C
:10FDD8000EA95A59FFF7E1FD002854D114A8059936
:10FDE800FFF7F2FA00284ED10BA8014614AAFFF734
:10FDF80022FD0146002844D10BA8FFF74EFC00283D
:10FE080015DA14A80EA9FFF7F3F900283BD114A8B6
:10FE18000599FFF7D9FA002835D10BA8014614AA8D
:10FE2800FFF7E9FC78BB139A5359013B5351059BE3
:10FE380008F1FF38203B043D0593043E46E7BAF13C
:10FE4800000F0AD0504611A9FFF7D2F9069BD9F83E
:10FE580000201B685343CAF80030AFB103990BA8C0
:10FE6800FFF705FB0BA93846FFF7C2F9D9F80030B0
:10FE780038463B600021FFF710FC28B901233B609E
:10FE880002E00C4600E0044617AB00930023019300
:10FE98000BA80EA911AA14ABFFF760F9204600E0E1
:10FEA8000C201BB0BDE8F08F1F0000801FB5002B91
:10FEB80083EAE374A4EBE374B4BF4FF0FF33012388
:10FEC80001930123029301AB0094CDF80CD0FFF706
:10FED80037FE04B010BD70B504460E46104600212A
:10FEE8001546FFF7DAFB002820DB002021463246C2
:10FEF8002B46FFF725FED0B920460021FFF7CDFBA2
:10FF080000280BDA204621462A46FFF774FCF2E760
:10FF1800204621462A46FFF78EFC40B9204629464E
:10FF2800FFF776FB0028F3DA002070BD0A2070BDC9
:10FF38002DE9F04F1E469B68ADF5517D1F6881463F
:10FF4800FB070D46049240F1B78107A80AA90022D1
:10FF5800FFF7F1F800214FF4407210A819F0EEFBFA
:10FF68000498FFF7BAF9B0F5287F0ADAEF280BDC16
:10FF78004F280CDC1728CCBF4FF003084FF00108BE
:10FF880007E04FF0060804E04FF0050801E04FF0E5
:10FF980004087368484603F1010A5146FFF7FEF862
:10FFA8000446002840F0688113A85146FFF7F6F888
:10FFB8000446002840F060810AA84FEA4A01FFF78A
:10FFC800EDF80446002840F05781DA9B0BB19B6896
:10FFD8001BBB07A80121FFF74BF90446002840F096
:10FFE8004B81716807A88901FFF7EEF904460028DC
:08FFF80040F0428107A8014618
:020000040801F1
:100000003246FFF76CFF0446002840F03981DA9B46
:1000100073B1DA9A07AB03CB106018685160906037
:1000200006E0DA9A07AB1068516803C3906818605D
:1000300031462846FFF7F0FA0028294613A803DBCB
:100040003246FFF74CFF01E0FFF7D6F8BA1C02F08A
:10005000040207EB420107FB01F3C3F1020301FBBA
:1000600003F207FB02F5C5F1020502FB05F307FBEE
:1000700003F5023D5D430AAF13A807A932462B469C
:100080000097FFF769FA484607A9FFF7B5F8044655
:10009000002840F0F58006AB4FF0010A0F9300975F
:1000A00048460DA932462B46CDF818A0CDF834A00D
:1000B000CDF838A0FFF750FAD04507D1049B0027B0
:1000C0005B68BC460393BA46BB466BE008F1FF3B56
:1000D0000AFA0BF710AB4FF00C0A0AFB073A7168EB
:1000E00050460131FFF75EF8002840F0C8805046C6
:1000F00013A9FFF781F8002840F0C180A4460AAB9D
:1001000000935046514632462B46CDF80CC0FFF7BF
:1001100023FADDF80CC00CF1010CDC45EFDB0137F4
:100120004FF00C0C10AB0CFB073A4FF0010B0BFA25
:1001300008FB5F45C2DA716850460131CDF80CA06A
:10014000FFF730F8002840F09A805046AAF10C01E1
:10015000FFF752F80AF10C0A002840F090800AAB31
:100160000093039813A932462B46FFF7F5F90137A0
:10017000DFE703934FF0200A049B039A9B680AF180
:10018000FF3A53F8223023FA0AF313F0010317D091
:100190000CF1010CCCEB08029340C44543EA0B0B75
:1001A0001FD00227BAF1000FE6D1039B039A013B4F
:1001B000002ADED1012303FA08F3049392464DE0AE
:1001C000002FEFD0012FE3D10AAB009348464946F8
:1001D00032462B46CDF814C0FFF7BEF9DDF814C047
:1001E000E0E74FF0000C0AAF009748464946324618
:1001F0002B46CDF814C0FFF7AFF9DDF814C00CF1B1
:10020000010CC445EFD110AB0C2101FB0B31009761
:10021000484632462B464FF0000BFFF79DF9012769
:10022000DC46BFE72B460097484649463246CDF8A4
:100230000CC0FFF791F9049B4FEA4B0B13EA0B0F2D
:10024000DDF80CC008D00097484613A932462B466B
:10025000FFF782F9DDF80CC00AF1010AE2450AAFA6
:10026000E0DB012306930D930E9306AB0F930097EB
:1002700048460DA932462B46FFF76EF900E00446CA
:10028000012308F1FF3203FA02F603FA08F5AE4241
:1002900008DA10AB0C2000FB06300021FEF762FFED
:1002A0000136F4E7DA9B13A80AA91BB10022FEF776
:1002B00059FF03E007AADA9BFEF754FF204600E04F
:1002C00004200DF5517DBDE8F08F002AF0B52DD04A
:1002D0002EDB012A01D1002325E0022A04D18B68FC
:1002E0001B6803F001031EE04D6800236F1EAD0084
:1002F000002FA5F1040511DB8C68013F6459260C21
:1003000046EA0343B3FBF2F602FB1633A4B244EA17
:100310000343B3FBF2F402FB1433E9E70968002955
:1003200001DA03B1D31A03600020F0BD0C20F0BD48
:100330000A20F0BD8B1E0E2B73B504460E461546E3
:1003400026D8214601A83246FFF7BFFF014608BB69
:10035000204622463346FFF7ADFD0146D0B9204680
:10036000FFF79FF938B9019B2A68092B0AD8511C5D
:100370002960303309E0204631462A46FFF7DAFF8C
:1003800048B9F0E7511C296037331370002002E0B0
:10039000042000E0084602B070BD2DE9F0431D4680
:1003A0008B1E0E2B85B007468846164667D8FEF78B
:1003B00098FFB8F1030F04DD4010B8F1100F08BF2B
:1003C00040102B680330834202DA2860082057E08F
:1003D00001A800210096FEF7B2FE3B68013301BF81
:1003E000009B5A1C00922D2208BF1A70B8F1100F02
:1003F00024D17C680021013C4FEA8409002C30DBC9
:100400004FF00308BA684FEAC80352F80920DA40EF
:1004100012F0FF0203D111B918EB040F07D11A49EA
:10042000009819F099FB009B01211844009018F1E5
:10043000FF38E7D2013CA9F10409DFE701A83946FA
:10044000FEF7DAFE0446A0B9019B01A8013308BFFC
:10045000012341466A4608BF0193FFF76BFF04463C
:1004600038B9009B00245A1C00921C70009B9E1BF4
:100470002E6001A80021FEF775FE204600E0042052
:1004800005B0BDE8F08300BF628403082DE9F043A6
:10049000ADF60C0D02AD14460F464FF4006200217C
:1004A00006462846984619F04DF940F2FE7321465B
:1004B000019338462A4601ABFFF76FFF044670BB35
:1004C000194B002E08BF1E46304619F0BFFC81466E
:1004D000284619F0BBFC0D232B540A222B18074683
:1004E0005A70B8F1000F13D0304601214A464346F6
:1004F00018F0DCFB484501D0022011E00237284605
:1005000001213A46434618F0D1FBB842F4D106E047
:10051000064831462A4619F07BF9404600E020465D
:100520000DF60C0DBDE8F08325A3030867840308CE
:100530002DE9F04107460E461846002115461C4697
:10054000FFF7AFF80028DDF8188008DBCDF8188039
:10055000384631462A462346BDE8F041ECE4042003
:10056000BDE8F08170B50C468AB004A900230646A8
:10057000154601A807AAFEF7E2FD214604A8FEF7EA
:100580003BFE0446002861D107A82946FEF734FE49
:10059000044600285AD104A8FEF78AFE054607A89B
:1005A000FEF786FE8542A8BF054604A82946FEF749
:1005B00062FF0446002849D107A82946FEF75BFFE1
:1005C0000446002842D101230793049304A8002184
:1005D000FFF767F878B304A8FEF76AFE014604A89F
:1005E000FEF749FF044688BB07A8FEF761FE0146F7
:1005F00007A8FEF740FF044640BB04A807A9FFF781
:100600000BF8002808DB04A8014607AAFFF7BAF890
:100610000446D8B904A807E007A8014604AAFFF7D2
:10062000B1F8044690B907A80121FEF724FF04465B
:100630000028CBD00AE007A82946FEF7C9FE0446E9
:1006400020B9304607A9FEF7D7FD044607A804A93C
:1006500001AA0023FEF786FD20460AB070BD2DE9F1
:10066000F04FA5B007900691104600211546FFF700
:1006700018F8002840F3408109AB009321AB0493A4
:100680000CAE00230FAC0DF1480B0DF160080DF11D
:100690006C090DF1780A0593304621465A4615AB90
:1006A000CDF80480CDF80890CDF80CA0FEF747FDFA
:1006B00009A806992A46FFF755FF0746002840F08B
:1006C000098109A80121FEF7ECFF002840F0018113
:1006D000304606992A46FFF702FC0746002840F0FC
:1006E000F98020463146FEF787FD0746002840F096
:1006F000F18040462946FEF77FFD0746002840F07E
:10070000E98048462946FEF777FD0746002840F075
:10071000E18058460121FEF7AFFD0746002840F072
:10072000D980394615A8FEF7A7FD0746002840F0F6
:10073000D18039465046FEF79FFD0746002840F01D
:10074000C98021A80121FEF797FD0746002840F047
:10075000C180119B1B68D8074CD420460121FEF7AD
:100760008AFE0746002840F0B580149B1B68DB0713
:1007700010D4179B1B68DF070CD412A80121FEF7C9
:100780007AFE0746002840F0A58015A80121FEF753
:1007900072FEDAE712A8014618AAFFF730F80746FA
:1007A000002840F0978015A801463246FFF747F829
:1007B00007460028E1D08DE01BA80121FEF75BFE73
:1007C0000746002840F08680209B1B68D90716D476
:1007D000239B1B68DA0712D41EA80121FEF74BFEEB
:1007E0000746002876D121A80121FEF744FE0746DE
:1007F00000286FD11D9B1B68DB07DDD510E01EA80C
:10080000014618AAFEF7FBFF0746002862D121A87F
:1008100001463246FFF713F807460028DCD059E0BE
:1008200020461BA9FEF7F8FE00281FDB20462146C4
:100830001BAAFFF704F8074600284BD112A801466F
:100840001EAAFEF7FCFF0746002843D115A8014663
:1008500021AAFEF7F4FF074600283BD120460021DD
:10086000FEF71FFF00287FF474AF18E01BA80146B5
:100870002246FEF7E4FF074660BB1EA8014612AA07
:10088000FEF7DDFF074628BB21A8014615AAE0E7D1
:100890001EA801462A46FEF7B2FF0746D0B91EA899
:1008A0000021FEF7FEFE0028F2DB06E01EA801464E
:1008B0002A46FEF7C4FF074660B91EA82946FEF780
:1008C000ABFE0028F2DA07981EA9FEF795FC074652
:1008D00000E00E2709AB009315AB019300230593AD
:1008E00021A8CDF808B00394049651464A464346E1
:1008F000FEF738FC384600E0042025B0BDE8F08F54
:100900002DE9F04F95B00391002105469346FEF77F
:10091000C8FE002800F0FE8028460121FEF7C1FE37
:10092000002800F0F78028460221FEF7BAFE0028D2
:1009300000F0F18011AB009305AE00230193304627
:100940000EAB08A90BAAFEF7FAFB2B680293012352
:100950002B60AB681B68DB0740F1DC806F4F57F8FA
:10096000044F002C14DD28462146FEF79AFE00288D
:100970000CDD224604A82946FFF7A7FC0446002800
:1009800040F0BB80049B002BE9D1C3E00020C2E013
:10099000304629460122FEF789FF0446002840F030
:1009A000AC803046FEF784FC3146824608A8FEF74C
:1009B00023FC0446002840F0A08008A85146FEF71A
:1009C0005AFD0446002840F098802846FEF789FC2E
:1009D00040F21353984211DC40F2513398420FDC3D
:1009E00040F2892398420DDCB0F5AF7F0CDAF9288C
:1009F0000CDC9528CCBF12271B2708E0022706E055
:100A0000032704E0042702E0082700E00C274FF04A
:100A100000080EA86968FEF7C5FB044600286CD1E3
:100A2000DDF840904C460F9AC9EB0403B3EB820FFC
:100A300005DA5846039B984704F8010BF3E70EA824
:100A4000FEF74FFC04463046FEF74BFC211A0131FD
:100A50000EA8FEF710FD044600284ED1109A0EA8ED
:100A60001368014643F00303136011AB009308AA17
:100A70002B46FFF75DFD044600283ED10EA8314607
:100A8000FEF7CAFD20B908F10108B845C1D134E02C
:100A90000EA80121FEF705FE0028F4D04FF0010951
:100AA000D14505DB0EA83146FEF7B6FDD8B123E0EF
:100AB0000EA83146FEF7B0FD0028F3D00EA90BA812
:100AC0000A46FEF709FFA8B90EA80BA92A46FFF7A8
:100AD00006FA78B90EA80121FEF7E3FD0028E1D05F
:100AE00009F10109DCE70EA80121FEF7DAFD002873
:100AF000C9D101E0044600E00E24029B11A82B603E
:100B00000023019300960EA90BAA08ABFEF72AFB5F
:100B1000204600E00E2015B0BDE8F08FD42A03086F
:100B200002292DE9FF4705460E4690461F4678DD0F
:100B300001A80021FEF703FB06F11F012846491119
:100B4000FEF730FB0446002865D121462846FEF713
:100B500093FB044600285ED1D5F808A0D1466A6808
:100B6000CAEB0903B3EB820F04DA0C98B84709F813
:100B7000010BF4E72846FEF7B4FBB042014604DA65
:100B80002846711AFEF724FC0DE008DCAA681368F9
:100B900043F003031360B8F1000F0ED015E02846B0
:100BA000891BFEF768FCA8BBF0E70E2832D1284667
:100BB00029460222FEF764FE60BB284639460C9A9D
:100BC000FFF79EFE0028F0D125E001A8294601226A
:100BD000FEF76CFEF0B901A80121FEF74CFCC8B984
:100BE000284639460C9AFFF78BFE28B901A83946EA
:100BF0000C9AFFF785FE70B10E280BD101A829468B
:100C00000122FEF73DFE28B9284629460222FEF7BA
:100C100037FEDFE7044601A80021FEF7A3FA2046CD
:100C200000E0042004B0BDE8F0872DE9F04F9BB050
:100C300017AB05AE02930DF12C0A00230DF1440809
:100C400014AD039308A952460EAB0446CDF80080BC
:100C500030460195FEF773FA304610217E4AFEF7C2
:100C6000ADFE0746002840F0DC8008A810217B4A32
:100C7000FEF7A4FE0746002840F0D380504610211E
:100C8000774AFEF79BFE0746002840F0CA800EA870
:100C900031465246FEF720FE0746002840F0C1804C
:100CA000284610216F4AFEF789FE0746002840F0CB
:100CB000B88014B16C4818F0ABFD0EA82946FEF7B9
:100CC000ABFC30B1002C00F09E80684818F0ECFDC1
:100CD00099E014B1664818F0E7FD0EA84146324687
:100CE0005346FEF731FF0746002840F09A80284619
:100CF0001021604AFEF762FE0746002840F091800E
:100D000017A810215C4AFEF759FE0746002840F05C
:100D1000888014B1594818F07BFD0EA82946FEF7CB
:100D20007BFC0028CED1404617A9FEF775FC0028B1
:100D3000C8D114B14E4818F0B7FD002300930EA897
:100D4000314608AA0BABFFF7F3FB0746002868D132
:100D5000284610214A4AFEF731FE0746002860D196
:100D600014B1484818F054FD0EA82946FEF754FC6B
:100D70000028A7D114B13E4818F096FD0EA83146C0
:100D80005246FFF76CFC074600284AD1284610213E
:100D90003D4AFEF713FE0746002842D114B13B48F6
:100DA00018F036FD0EA82946FEF736FC002889D13A
:100DB0002CB12F4818F078FD354818F029FDDFF8E0
:100DC000DC904FF0000B0EA859F8081CFEF754FAFF
:100DD000074630BB404659F8041CFEF74DFA07465B
:100DE000F8B930460EA94246FFF7BCFB0746C0B92A
:100DF0003046D9F80010FEF754FC30B11CB125483C
:100E0000594618F005FD012022E00BF1010BBBF162
:100E1000030F09F10C09D6D144B1154818F044FD6F
:100E200004E01CB11C48394618F0F2FC08AB0193F1
:100E300000230393CDF800A0029617A82946424646
:100E40000EABFEF78FF914B10A2018F0F5FC384606
:100E50001BB0BDE8F08F00BF6C840308ED8403086D
:100E60006E850308CF850308AE8603083D9C030802
:100E7000DB830308C8860308EC8603084B87030856
:100E800065870308C4870308DE8703083F880308D3
:100E9000598803087688030884880308802D03088E
:100EA0000B6870B504684968634040681E4CDDB249
:100EB00048402544190E665C95F80011C3F30745B8
:100EC0002544C3F3072395F80052234493F80033D5
:100ED00041EA066141EA054141EA032104EB10635E
:100EE00093F80052C3B2E35C43EA0563C0F30745DD
:100EF0002544C0F3072095F80053204490F80001E2
:100F000043EA054343EA002381EA3361106883EA38
:100F1000314381EA3321434083EA3123136053682C
:100F20005940516070BD00BF9C2D03082DE9F04F62
:100F30001446C3B00EAF051D40220646884638460B
:100F4000002118F0FFFB284600214FF4887218F0AA
:100F5000F9FBC02C09D0B4F5807F06D0802C40F07E
:100F6000078203233360002302E00423336001235C
:100F7000082294FBF2F201930023934204DA18F85A
:100F80000310F9540133F8E7C02C02D0A04B002223
:100F90000AE00DF147030DF14F0113F8012FD24381
:100FA0008B421A72F9D1F1E7197813F8010C090490
:100FB00041EA006198780833014313F8070C41EACD
:100FC000002102A8815013F8041C00EB020E13F854
:100FD000050C090441EA006113F8020C08320143D0
:100FE00013F8030C302A41EA0021CEF80410DBD1BB
:100FF0000DF1780840224046002118F0A3FB3A4644
:101000000023517817F82300090441EA0061D078E1
:101010000432014312F8020C41EA002148F823107F
:101020000133082BEDD11DAB21AF043319691A68C8
:10103000BB4282EA01021A62F7D126A802A928AAB5
:10104000FFF72EFF04A928A826AAFFF729FF25AB42
:10105000984629A953F8040F53F8202C8B4282EAB2
:1010600000021A60F6D126A806A928AAFFF718FFE1
:1010700028A808A926AAFFF713FF802C12DD3B46FB
:10108000043319691A68434582EA01021A62F7D1EA
:101090002AA80AA92CAAFFF703FF2CA80CA92AAAA0
:1010A000FFF7FEFE1E9B5B4A2E931F9B91462F93DC
:1010B000209B01203093219B3193019B4FEA031C1D
:1010C0002EAB19460CF1FF38904418F8012F42B3AB
:1010D000C0EB00122F9F02F01F02C2F1200E27FA70
:1010E0000EFB2E9F07FA02FA8BEA0A070F61309F68
:1010F00027FA0EFB2F9F07FA02FA8BEA0A074F61C5
:10110000319F27FA0EFB309F07FA02FA8BEA0A0793
:101110008F612E9F319E27FA0EF706FA02F2574092
:10112000CF610130052801F11001CED101993A4A71
:101130004FF0500808FB0128002118F90100421C5B
:1011400018BF53F8212001F1010118BF45F82020F4
:101150001429F2D1802C0DDC269A0CF1070A2E926C
:10116000279ACA442F92289A19463092299A012028
:10117000319253E01946229A0CF1030A2E92239AD7
:10118000CA442F92249A01203092259A31921AF85B
:10119000012F2AB3C0EB00122F9F02F01F02C2F1F1
:1011A000200E27FA0EFB2E9F97408BEA07070F6150
:1011B000309F27FA0EFB2F9F97408BEA07074F615E
:1011C000319F27FA0EFB309F97408BEA07078F610C
:1011D0002E9F319E27FA0EF706FA02F25740CF6192
:1011E0000130052801F11001D1D1002108EB0102E5
:1011F00092F91400471C1CBF2EAA52F8212001F1BD
:10120000010118BF45F820201429EFD1A4E700BF41
:101210009D310308CC310308EC3103081AF8012F83
:101220002AB3C0EB00122F9F02F01F02C2F1200E62
:1012300027FA0EFB2E9F97408BEA07070F61309F1E
:1012400027FA0EFB2F9F97408BEA07074F61319FCC
:1012500027FA0EFB309F97408BEA07078F612E9F7E
:10126000319E27FA0EF706FA02F25740CF6101309D
:10127000052801F11001D1D1002108EB010292F9FA
:101280002800461C1CBF2EAA52F8212001F10101A2
:1012900018BF45F820201429EFD1802C0ADC0199D1
:1012A000354A0E46142303FB01220C235E43002320
:1012B000B6004CE02A9A0CF10B0C2E922B9AE144CA
:1012C0002F922C9A012130922D9A319219F8012FE8
:1012D00032B3C1EB01122F9802F01F02C2F12004B9
:1012E00020FA04FE2E9800FA02F78EEA0700186131
:1012F000309820FA04FE2F9800FA02F78EEA0700D1
:101300005861319820FA04FE309800FA02F78EEA0C
:10131000070098612E98E040319C94406040D8616D
:101320000131052903F11003D0D1002308EB03029A
:1013300092F93C20541C1CBF2EA951F8231003F134
:10134000010318BF45F82210142BEFD1A7E7D1569F
:10135000481C1EBF55F8210006EB8301491903F113
:10136000010318BFC1F88000142BF0D1002000E069
:10137000024843B0BDE8F08F8C32030800F6FFFF4F
:10138000F0B5C02AC7B0054608D0B2F5807F05D0B9
:10139000802A48D103230360002402E004232B6049
:1013A000012401A8FFF7C2FD00283DD1230101AAB5
:1013B000303302EB830359681A696960996805F153
:1013C0001406A960D9682A61E960E10001F11604F8
:1013D000A6461F1F1C350C3B9A68013C45F8082C9B
:1013E000DA6805F1080545F80C2CA3F10803F3D1E0
:1013F0006FF0070202FB01F3B03BFA1852F8081C29
:10140000FB5806EBCE0046F83E1052F8041C8360F1
:1014100053684160C360214601A84FF48A7218F0F6
:1014200091F9204600E0014847B0F0BD00F6FFFF0B
:10143000F0B51D46537914791B0443EA0463D4794B
:10144000117A23439479167B43EA0424537A92F861
:1014500000E01B0443EA0163D17A85B00B43917A23
:10146000076843EA0121537B1B0443EA0663D67BEA
:101470003343967B43EA06235678360446EA0E6EDB
:10148000D67892784EEA060646EA0222466872400C
:10149000009282685440C2680194514002690291EE
:1014A000534000F114040393002F43D068462146B3
:1014B00002AAFFF7F5FC02A804F108016A46FFF74B
:1014C000EFFC684604F1100102AAFFF7E9FC02A84C
:1014D00004F118016A46FFF7E3FC684604F12001B5
:1014E00002AAFFF7DDFC013F02A804F128016A46C9
:1014F000FFF7D6FC0FB930341CE0009B226B403460
:1015000003EA0201019A82EAF17254F80C1C01927A
:101510000A435340009354F8042C039B43EA02010E
:10152000029A4A4054F8081C02920A4083EAF27375
:101530000393B9E72068029B61685840039BA26847
:101540005940009BE4685A40019BE8706340040ED8
:101550002C70040C6C70040A080E2871080C687159
:10156000E971080A110E2972110C6972EA72110AE6
:101570001A0E2A731A0CA8716A7300201A0AAC702A
:10158000A972AA73EB7305B0F0BD2DE9F04F99462F
:1015900085B0130780468A4615460E9F0F9E9346D8
:1015A0005CD100294FD13A46AB1A3B44002B53DDA6
:1015B0001346EE46EA4602F11004F44618685968EC
:1015C0000833ACE80300A342E646F6D100213346D7
:1015D0004046FFF72DFF731E09F1FF3106F10F00A2
:1015E00013F8012F11F801EF83428EEA02021A70FC
:1015F000F6D15246CE460DF1100C134603CB63458F
:10160000CEF80000CEF804101A460EF1080EF4D100
:1016100022461036C8E719F80300CA5C4240E2547B
:101620000133102BF7D12246234640465146FFF79F
:10163000FFFE4B4604F1100254F8041B944243F899
:10164000041BF9D1103DC5EB0B04002D07EB040181
:10165000344401DD0023DEE7002000E0014805B04E
:10166000BDE8F08FF0F5FFFF2DE9F04708ADE0CDC4
:10167000824698461C6806EB020991B1013F24E0BE
:101680002CB9504601212A462B46FFF7D1FE2B5D8F
:1016900016F8012B534007F8013B2A55013404F09A
:1016A0000F044E45ECD112E02CB9504601212A46D8
:1016B0002B46FFF7BDFE2A5D16F8013B534007F8A5
:1016C000013F2B55013404F00F044E45ECD1C8F80E
:1016D00000400020BDE8F0872DE9F04FEFB006464E
:1016E000002111A8202218F02DF84FF000084FEA31
:1016F000680908F0010B09F102074EB19A4B9B4AA9
:101700009B48B901BBF1000F18BF1A4618F080F8CA
:10171000FB000393BB010293964B4FEA491903EB7D
:10172000090A0027944C07EB090104EB4101039AD5
:1017300011A814F00BFE29A811A9029ABBF1000F01
:101740001CD1FFF71DFE0AEB070305AC03F11005E2
:10175000224618685968083303C2AB421446F7D1D1
:10176000864B09AC3B4403F11005224618685968C2
:10177000083303C2AB421446F7D11BE0C0343C44EB
:10178000FFF7D4FB04F1100505AB1A462068616829
:10179000083403C2AC421346F7D10AEB070309AC85
:1017A00003F11005224618685968083303C2AB429A
:1017B0001446F7D105AC5946224629A819AB09AD04
:1017C000FFF736FE19A82946102217F025FF30B181
:1017D000002E00F0C2806A4818F066F8BDE01037AD
:1017E000202F9FD116B1674818F05EF808F1010864
:1017F000B8F1060F7FF47BAF16B10A2018F01CF881
:101800004FF000084FEA680B08F001095EB1564B33
:10181000564A0BF102015C488901B9F1000F18BF6B
:101820001A4617F0F5FF594B274603F1100CE64610
:101830003A4618685968083303C263451746F7D11A
:101840002F46524B03F1100C3A461868596808337A
:1018500003C263451746F7D10BF102070EEB4B119C
:10186000FA0011A814F072FDBA0129A811A9B9F162
:10187000000F02D1FFF784FD01E0FFF757FB444B57
:101880004FF0300A0AFB0B3A00270DF1340EB9F184
:10189000000F1ED194E80F008EE80F00A6460AEB59
:1018A000070303F1100C724618685968083303C225
:1018B00063459646F7D1AE46364B3B4403F1100CD8
:1018C000724618685968083303C263459646F7D1D3
:1018D0001DE095E80F008EE80F00A6462D4B3B4417
:1018E00003F1100C724618685968083303C2634547
:1018F0009646F7D1AE460AEB070303F1100C724689
:1019000018685968083303C263459646F7D10DF14C
:10191000640BCDF804B0494610220DAB009429A801
:10192000FFF733FE58462946102217F075FE83460E
:1019300000287FF44DAF1037302FA6D116B11148D3
:1019400017F0B2FF08F10108B8F1060F7FF45AAFA3
:101950002EB10A2017F070FF01E04FF0010B58463E
:101960006FB0BDE8F08F00BFC2830308BE830308D9
:10197000AA880308B432030814330308D4330308D5
:101980003D9C0308DB830308C4880308F433030881
:1019900064340308F43403080FB413B5094C04ABE2
:1019A00053F8042B204640F2FF1101931CF0F4FA87
:1019B0002046002384F8FF3102B0BDE8104004B097
:1019C000704700BF7C4E002070B516468269ADF5A9
:1019D000027D04460D468AB10093869B40F2FF11BA
:1019E0000193084A334602A818F06AF800238DF8DC
:1019F0000732A06AA369294602AA98470DF5027D1D
:101A000070BD00BFDE88030870B50D468169ADF575
:101A1000047D16460446899A99B10093889B0292E8
:101A20000193039240F2FF11074A334604A818F0CD
:101A300047F800238DF80F32A06AA369294604AA4B
:101A400098470DF5047D70BDEC8803082DE9F0453D
:101A50001E468369ADF5057D82460D4690468E9FF4
:101A6000002B54D0002F52DB8C9B40F2FF110193CE
:101A7000294A43460096029704A8002418F020F84B
:101A80008DF80F42DAF81830DAF82800294604AA4F
:101A90009847BC4233D0B4F5805F31D023071AD1C8
:101AA00034B1DAF81830DAF8280029461B4A98478A
:101AB00040F2FF111A4A43460096019404A817F019
:101AC000FFFF00238DF80F32DAF82800DAF818301B
:101AD000294604AA98478D9B40F2FF111B5D114ACD
:101AE00004A817F0EDFF00238DF80F32DAF8280074
:101AF000DAF81830294604AA98470134C9E734B106
:101B0000DAF81830DAF828002946044A98470DF523
:101B1000057DBDE8F08500BF0F8903083089030803
:101B200032890308EE9903082DE9F04F9B4683693B
:101B3000ADF5077D04460F469246DDF84482002B42
:101B40006DD0B8F1000F6AD0D8F80460013EB30040
:101B5000002E04DBD8F80820D258043BB2B1909B89
:101B6000CDF800B00193731C5B01029306A85346A5
:101B700040F2FF112C4A002517F0A2FF8DF81752F2
:101B8000A369A06A394606AA984727E0013EDFE725
:101B9000AB0727D04FEA890C4FF00309D8F808307B
:101BA0004FEAC90253F80C3040F2FF11D340DBB2C8
:101BB0001E4A06A8CDF814C017F082FF00238DF846
:101BC0001732A06AA369394606AA09F1FF39984776
:101BD000B9F1FF3FDDF814C0E0D10135B6EB0509DE
:101BE000D6D517E025B1A369A06A3946104A9847AF
:101BF0005346CDF800B006A840F2FF110D4A17F089
